:020000040800F2
:1000000000200010F5FD0208F15702086D4D0008B0
:10001000ED570208E9570208E55702080000000002
:10002000000000000000000000000000E15702088E
:10003000DD57020800000000D9570208710F0008C0
:100040005DFE02085DFE02085DFE02085DFE02081C
:100050005DFE02085DFE02085524000881250008A7
:100060004525000809250008CD240008F13B0008BB
:10007000E13B0008D13B0008C13B0008B13B000850
:100080009D3B0008893B00085DFE02085DFE0208FA
:10009000715B02085DFE02085DFE02089124000803
:1000A0005DFE0208E953000889530008F95300086F
:1000B000D9530008C9530008B95300085DFE02086F
:1000C0005DFE02085DFE02085DFE02085DFE02089C
:1000D0005DFE02089D10000821100008A50F000811
:1000E000192400085DFE0208C95702085DFE0208D7
:1000F000995300085DFE0208A95300085DFE02083E
:100100000000000000000000000000005DFE02088A
:100110005DFE02085DFE0208392E01081D2E010851
:10012000753B0008613B00084D3B0008393B000867
:10013000253B00085DFE02080000000000000000F2
:100140005DFE02085DFE02085DFE02080000000080
:10015000000000000000000000000000000000009F
:1001600000000000000000005DFE02085DFE0208C5
:100170005DFE02080000000000000000000000001A
:08018000000000005DFE020812
:1001880070B4EFF31186502383F31288436B1A6817
:10019800D20720D45D686DB9446A826A944217D048
:1001A80081691144D9600ED9A21A5A60846200226A
:1001B80080F850201A6842F00102F1B21A6081F307
:1001C800118870BC704701698A1A5A608562EEE727
:1001D800012380F85030F1B281F3118870BC704768
:1001E800436A8269D154436A0169426B01338B4285
:1001F80028BF00234362002A2FD0EFF31181502338
:1002080083F31288436B1A68D2072CD470B45E68E3
:100218006EB9456A826A954217D084691444DC60D5
:100228000ED9AA1A5A608562002280F850201A68EE
:1002380042F00102C9B21A6081F3118870BC70479C
:100248000469A21A5A608662EEE7012380F85030EA
:10025800C9B281F3118870BC7047C26C136843F04F
:10026800800313607047C9B281F31188704700BFDB
:10027800026B10B462B1036CC2684469D11A013BC5
:10028800615C5DF8044B08BF13460364C8B270474D
:10029800016A4369C4685B5C0131A14228BF114609
:1002A80001625DF8044BD8B2704700BF436B13B1CD
:1002B80090F850007047836A406A181AB0FA80F0C4
:1002C80040097047416A836A99420AD3CB1A416B45
:1002D800026961B14968501E0B4483420AD2C01AB0
:1002E800704702691144CB1A416B0029F2D1501EA4
:1002F800C01A704700207047036B43B1026C5B68FB
:1003080093422FBF981AC0689B1AC0187047C269D9
:10031800036A9A422FBFD01AC0688018C01A704763
:100328000A4B30B503F1140493F900205D78072ACD
:10033800C8BF143A811804330D7313F8025C85544E
:1003480013F8012C0A76A342EED130BD1C2803080D
:1003580003682DE9F041DF691FB13B46BDE8F04174
:100368001847002A164611DD04460D460E4400E0E3
:1003780023689B68204698470028F9D0236815F819
:10038800011B1B6820469847AE42F1D1BDE8F081B9
:1003980000232222027043708370C370704710B527
:1003A800074B03F10C0193F900205C788454024454
:1003B8009C78D470DC78947104338B42F3D110BDEF
:1003C80030280308002870B51EDB0928044620DD04
:1003D800012303EB83035B00B0FBF3F2092AF8D88F
:1003E8007BB10E4EB4FBF3F00928CCBF5722302264
:1003F800A6FB03E5024403FB1044EB0801F8012BBC
:10040800F0D100230B7070BD2D230B7040420131D9
:10041800DBE7303001F8010BF3E700BFCDCCCCCCE3
:10042800884230B44FF001042ED301FB04F4B0FB32
:10043800F4F58D42F9D284B1AAB901E0B0FBF4F524
:10044800092DCCBF572230222A4404FB150003F89B
:10045800012BB4FBF1F4002CF0D100221A7030BC4F
:100468007047B0FBF4F5092DCCBF372230222A445F
:1004780004FB150003F8012BB4FBF1F4002CF0D1B8
:1004880000221A7030BC70470546002AEBD1D7E726
:1004980003685A1C02601970704700BF2DE9F047C5
:1004A800089C2578002B804689460CBF4FF0200A0F
:1004B8004FF0300A661C35B3002A29DD334601E0C7
:1004C800024698B113F8011B501E0029F8D1971E57
:1004D80060B13D46013D51464046C8476B1C002B64
:1004E800F8DC257827EAE770013055B1041B294666
:1004F8004046C847301916F8015B002DF7D1BDE812
:10050800F087BDE8F087002A04DC2846BDE8F087BC
:100518000020EBE7571EDCE783684268D0ED037ADA
:1005280000EB83010133934281ED040A836004BF29
:100538000023836000EB830393ED047A036870EE75
:10054800277A9A42C0ED037A77EEC77AC0ED037A2C
:100558000CDA013307EE103AF8EEC76AB7EE007A04
:1005680087EEA60A036030EE070A704707EE102AE6
:10057800B8EEC77A87EE870A704700BF90ED057A14
:1005880090ED004AD0ED066AD0ED014AD0ED047A2C
:1005980090ED035AD0ED025AA4EE007AB0EE406A0C
:1005A800B0EE470AB0EE667AA6EE247A67EEC07A15
:1005B800A0EE457AE6EE257A80ED057AC0ED067A5A
:1005C800704700BFD0ED057A90ED013AD0ED003AC2
:1005D800D0ED064A90ED024A90ED077A90ED035A65
:1005E80090ED086AD0ED045AC0ED067AF0EE406A44
:1005F80027EE830AC0ED056AA3EEA60A80ED087A05
:10060800A4EE240AA5EE470AA5EEC60A80ED070A5D
:10061800704700BFD0ED007A90ED017A30EE670A9E
:10062800E7EE007AB0EE670AC0ED007A704700BFC7
:10063800704700BF0A44914214D030B40139551EA6
:1006480041F2210211F8014F082380EA0420040432
:100658004CBF82EA40004000013B80B2F7D18D4296
:10066800F0D130BC704700BF4FF4006383827047FD
:100678004FF40063838270474FF48053838270473E
:1006880070B5044682B01430E56D06236A464321EE
:10069800A847B0B19DF804009DF800609DF80110CE
:1006A8009DF802509DF803209DF8053041EA062187
:1006B80043EA002342EA0522A187E287A4F84030F2
:1006C800012002B070BD00BF70B5044682B008308A
:1006D800656A06236A463B21A847A8B19DF804002D
:1006E8009DF800609DF801109DF802509DF80320C8
:1006F8009DF8053041EA062143EA002342EA052233
:10070800E18222836383012002B070BD50F8043C6B
:10071800012280F84520103803B11847704700BF00
:1007280010B490E80600047B40690223A3404B60A4
:1007380013685DF8044B4FF6FE710B4013601FE51C
:1007480070B40468037B2268022101FA03F31A4299
:1007580013D042690A49582000FB02124FF6FE7670
:1007680050685289C5680068296831402960C168A5
:10077800D24392B20A40C260636070BC704700BF47
:100788004C4B002030B4094B1C7864B1084B002551
:1007980003EBC4041A6899885562D068083301438A
:1007A800A342D160F6D130BC704700BF0C4E002088
:1007B800104E002010B40268047B11680223A34085
:1007C800194209D00649406800240C7001684FF6A8
:1007D800FE742140016053605DF8044B704700BF10
:1007E8002741002030B50446C06C61710368A268D7
:1007F80023F00103036087B0A379009213F0040289
:100808003DD04FF4805213F00203019244D1029379
:100818004FF480630022039311F00103059237D14E
:10082800049308238D07694648BF04931FF0ACFE64
:100838006079E36CA17900F00202002A15BF4FF439
:1008480040324FF480324FF40034002410F0010F8E
:10085800586808BF2246CC074CBF024320EA020270
:100868005A609A6809074CBF42F0080222F0080251
:100878009A601A6842F001021A6007B030BD13F09E
:10088800020301920BD04FF4005513460295C1E7BD
:10089800042304930C23C5E74FF40053B7E70293EE
:1008A800B8E700BF10B50446C06CA160036823F028
:1008B80001030360A37986B013F00402009141D0CC
:1008C8004FF4805213F00203019244D102934FF483
:1008D800806362790393D1074FF000030493059373
:1008E80045BF0423049308230C236946920748BF95
:1008F80004931FF049FE6079E36CA17900F00202CD
:10090800002A15BF4FF440324FF480324FF40034C0
:10091800002410F0010F586808BF2246CC074CBFCE
:10092800024320EA02025A609A6809074CBF42F063
:10093800080222F008029A601A6842F001021A605E
:1009480006B010BD13F00203019207D04FF4005116
:1009580013460291BDE74FF40053B7E70293B8E797
:100968002DE9F341056906460F467DBBD0F80080A6
:10097800C8F30A0323B30023D6F80080019323F0B9
:100988007FFC042819D1224C236943F00103236119
:10099800BBB2A8F8003023F073FC04282ED108F16C
:1009A80002030193019B3F0C1F8023F069FC23691C
:1009B800042823F00103236125D06FF0010505E029
:1009C80023F05EFC042805D04FF0FF35284602B01E
:1009D800BDE8F0810E4C236943F002032361C4F89B
:1009E8001480236943F04003236123F049FC236901
:1009F800042823F002032361BDD0E5E7236923F02F
:100A080001032361D9E7336804333360DEE700BFAD
:100A180000200240F8B504460D468E180027B5425E
:100A280001D12069F8BDE368591CE160234415F839
:100A3800012B1A720429F2D1A1682046FFF790FF12
:100A4800E7602061EBE700BF70B582B004466946F5
:100A5800143025F0FDFCB0B19DF805009DF801604B
:100A68009DF802109DF803509DF804209DF806306B
:100A780041EA062143EA002342EA0522A187E287E8
:100A8800A4F84030012002B070BD00BF2DE9F04F3E
:100A9800013085B0C3B203930B4602918B4C8C4E48
:100AA800002B00F099808B4D8B4FDFF8309225F0AA
:100AB800A9FE4FF4FA7A4FF0100C4FF47A70D9F877
:100AC8000430C3F30803002B40F0DE80EFF31183FA
:100AD800002B40F0D9802968A26800BF2B68994292
:100AE800F9D1D7F800E000FB0EF39B1AB3FBFEF335
:100AF80000FB01314FF0010E0191D9F80430C3F326
:100B08000803002B40F08780EFF31183002B40F09F
:100B180082802B68A16800BF2A689342F9D1D7F870
:100B280000B000FB0BF2521AB2FBFBF200FB0323EE
:100B3800019A9B1AB3F57A7FDFD3BAF1010ABED1C5
:100B4800039B002B40F0BD804FF47A7ADFF88C913C
:100B580050464FF0100CD9F80430C3F30803002BAB
:100B680075D1EFF31183002B71D12968A26800BFFA
:100B78002B689942F9D1D7F800E000FB0EF39B1AD5
:100B8800B3FBFEF300FB01314FF0010E0191D9F8E0
:100B98000430C3F3080313BBEFF31183FBB92B68CD
:100BA800A16800BF2A689342F9D1D7F800B000FBCA
:100BB8000BF2521AB2FBFBF200FB0323019A9B1AB9
:100BC800B3F57A7FE3D3BAF1010AC4D1029B013BA2
:100BD8000293002B7FF467AF05B0BDE8F08FEFF309
:100BE80011888CF31288A1682368DB0344BFC6F818
:100BF80000E0A1682B6832685FFA88F888F31188EA
:100C0800D7F800801A4400FB08F35B1AB3FBF8F32B
:100C180000FB0233D2E7EFF311888CF31288A16846
:100C28002368DB0344BFC6F800E0A1682B6832687C
:100C38005FFA88F888F31188D7F800801A4400FB17
:100C480008F35B1AB3FBF8F300FB023370E7EFF32A
:100C580011828CF31288D4F808E02368D90303D5ED
:100C680001233360D4F808E02B683168D2B282F3EC
:100C780011883A68194400FB02F3A3EB0E03B3FB97
:100C8800F2F300FB01317FE7EFF311828CF3128856
:100C9800D4F808E02368D90303D501233360D4F8D6
:100CA80008E02B683168D2B282F311883A68194497
:100CB80000FB02F3A3EB0E03B3FBF2F300FB0131DD
:100CC80018E7184625F01EFC3EE700BF10E000E0DC
:100CD80024710020287100202C71002000ED00E014
:100CE800204B5B68C3F3080330B4BBB9EFF311833F
:100CF800A3B91D4B1D4C1868A16800BF1A68904223
:100D0800F9D11B4B1C684FF47A7202FB04F3591A91
:100D1800B1FBF4F130BC02FB00107047EFF3118215
:100D2800102383F3128811498C680B6813F4803FF1
:100D3800104B02D0012018608C680B49D2B20D68A4
:100D4800186882F311880A4B19684FF47A7228449C
:100D580002FB01F31B1B30BCB3FBF1F302FB0030B9
:100D6800704700BF00ED00E02871002010E000E0AF
:100D78002C710020247100202DE9F84F8046FFF7E0
:100D8800AFFF254E2549DFF8A0E0254A254D8446CA
:100D980010274FF47A740120DEF80430C3F30803F7
:100DA800D3B9EFF31183BBB90B68D2F808A000BF21
:100DB800D1F800904B45F7D1D6F800B004FB0BF9F9
:100DC800A9EB0A09B9FBFBF904FB0393A3EB0C039A
:100DD8004345E1D3BDE8F88FEFF3118A87F3128812
:100DE800D2F808B01368DB0344BF2860D2F808B013
:100DF8000B68D5F800905FFA8AFA8AF31188D6F85A
:100E080000A0994404FB0AF3A3EB0B03B3FBFAF32A
:100E180004FB0933DAE700BF2C7100202871002099
:100E280010E000E02471002000ED00E02DE9F04F13
:100E3800DFF830C1474A4849484E494D8046102797
:100E480018F1FF38C0F08480DCF80430C3F30803DD
:100E5800002B5CD1EFF31183002B58D10B689468F9
:100E680000BF08688342F9D1D6F800904FF47A7031
:100E780000FB09FEAEEB040EBEFBF9FE00FB03EE21
:100E8800DCF80430C3F308034FF47A740120FBB98B
:100E9800EFF31183E3B90B68D2F808A000BFD1F8CB
:100EA80000904B45F7D1D6F800B004FB0BF9A9EB3D
:100EB8000A09B9FBFBF904FB0393A3EB0E03B3F593
:100EC8007A7FBDD2DCF80430C3F30803002BDFD0EF
:100ED800EFF3118A87F31288D2F808B01368DB039E
:100EE80044BF2860D2F808B00B68D5F800905FFAC4
:100EF8008AFA8AF31188D6F800A0994404FB0AF309
:100F0800A3EB0B03B3FBFAF304FB0933D5E7EFF3C9
:100F1800118487F31288D2F808901368D80303D590
:100F280001232B60D2F808900B682868E4B284F398
:100F38001188D6F800A04FF47A7400EB030E04FB76
:100F48000AF3A3EB0903B3FBFAF304FB0E3E97E79E
:100F5800BDE8F08F10E000E0287100202C7100201F
:100F68002471002000ED00E030B4EFF3118310226B
:100F780082F312880649074C0A680748013200259F
:100F88000A602560DBB2026883F3118830BC7047C1
:100F9800287100202471002010E000E01D4B70B57E
:100FA8009C68E36C226BDD69C2B1636B2BB12B07C4
:100FB80002D5E36C08221A6270BD2A06F7D5A26A28
:100FC800616A8A421FD0511CA069A162825C2069B3
:100FD800E66C81423285EAD3A362E8E7A906E4D544
:100FE800E26A1AB1988C80B29047DEE7E1699B8C7F
:100FF8006069DBB24E1CE6614354E169E3689942DB
:1010080028BFE261D1E7E26C136823F08003136024
:10101800CDE700BFF82900201D4B70B55C68E36C74
:10102800226BDD69C2B1636B2BB12B0702D5E36C70
:1010380008221A6270BD2A06F7D5A26A616A8A4236
:101048001FD0511CA069A162825C2069E66C8142B4
:101058003285EAD3A362E8E7A906E4D5E26A1AB1C1
:10106800988C80B29047DEE7E1699B8C6069DBB2BF
:101078004E1CE6614354E169E368994228BFE26186
:10108800D1E7E26C136823F080031360CDE700BF5B
:10109800F82900201D4B70B51C68E36C226BDD69D4
:1010A800C2B1636B2BB12B0702D5E36C08221A621D
:1010B80070BD2A06F7D5A26A616A8A421FD0511C00
:1010C800A069A162825C2069E66C81423285EAD31C
:1010D800A362E8E7A906E4D5E26A1AB1988C80B25F
:1010E8009047DEE7E1699B8C6069DBB24E1CE661E4
:1010F8004354E169E368994228BFE261D1E7E26CB1
:10110800136823F080031360CDE700BFF82900209F
:1011180003685B6A03B11847704700BF03681B6A1E
:1011280003B11847704700BF03682DE9F041DF6934
:101138001FB13B46BDE8F0411847002A164611DDAD
:1011480004460D460E4400E023689B6820469847F5
:101158000028F9D0236815F8011B1B68204698471A
:10116800AE42F1D1BDE8F08103689B69184700BF22
:1011780003685B69184700BF0368DB68184700BF4E
:1011880003689B68184700BF03685B68184700BF7F
:1011980003681B68184700BF014B1868F8E700BFD1
:1011A8008C780020054B53F8203033B11A689B889F
:1011B800918A0B4218BF1B0493617047F47000209A
:1011C80003682DE9F04F03F13845644EAD0A012458
:1011D800755D05F01F066D09022D04FA06F400F08E
:1011E800A280032D00F0A480012D52D08088B0FA8F
:1011F80080F4C4F11F04A4B2E50803EB850504F0EC
:1012080007042E6AA4000F27A74026EA07062E62C5
:101218002E6A01F0030702FA04F47A1E3443012A05
:10122800C1F3810CC1F300182C62C1F3411135D907
:10123800C60700F19780850700F1A380440700F1F5
:10124800B180020700F1BF80C60600F1CD80850697
:1012580000F1DB80440600F1E980020600F1F78026
:10126800C60500F10581850500F11381440500F1EB
:101278002181020500F12F81C60400F13D8185041A
:1012880000F14B81440400F15981020455D4BDE8B2
:10129800F08F334D6E6934436C61A7E70024224612
:1012A8004FF0010E4FF0030904E00132102A04F157
:1012B8000204ECD00EFA02F636EA0005F5D1D3F8AE
:1012C80008A009FA04F5ED430AEA050AC3F808A0DC
:1012D800D3F808B00CFA04FA4AEA0B0AC3F808A0D3
:1012E800B3F804A01FFA8AFA2AEA06069E80B3F821
:1012F80004A008FA02F646EA0A06B6B29E801E68FC
:101308002E401E60D3F800A007FA04F646EA0A0643
:101318001E60D3F80CA001FA04F605EA0A0A46EAA8
:101328000A05DD60C1E70E4DAE693443AC615DE787
:101338000B4DEE693443EC6158E71A6822F04042DD
:101348001A601A6842EA87771F60DA6822F040421A
:1013580042EA8171D960BDE8F08F00BF104F0308E1
:10136800001002401A6822F003021A601A683A4311
:101378001A60DA6822F003020A438507DA607FF50B
:101388005DAF1A6822F00C021A601A6842EA8702F6
:101398001A60DA6822F00C0242EA81024407DA6035
:1013A8007FF54FAF1A6822F030021A601A6842EAD5
:1013B80007121A60DA6822F0300242EA0112DA6093
:1013C80002077FF541AF1A6822F0C0021A601A6856
:1013D80042EA87121A60DA6822F0C00242EA8112F1
:1013E800C606DA607FF533AF1A6822F440721A60D5
:1013F8001A6842EA07221A60DA6822F4407242EA5E
:1014080001228506DA607FF525AF1A6822F440626A
:101418001A601A6842EA87221A60DA6822F440627F
:1014280042EA81224406DA607FF517AF1A6822F48F
:1014380040521A601A6842EA07321A60DA6822F4DF
:10144800405242EA0132DA6002067FF509AF1A68B3
:1014580022F440421A601A6842EA87321A60DA684F
:1014680022F4404242EA8132C605DA607FF5FBAEDB
:101478001A6822F440321A601A6842EA07421A606F
:10148800DA6822F4403242EA01428505DA607FF5E3
:10149800EDAE1A6822F440221A601A6842EA8742BE
:1014A8001A60DA6822F4402242EA81424405DA608E
:1014B8007FF5DFAE1A6822F440121A601A6842EA11
:1014C80007521A60DA6822F4401242EA0152DA60DE
:1014D80002057FF5D1AE1A6822F440021A601A6834
:1014E80042EA87521A60DA6822F4400242EA8152DC
:1014F800C604DA607FF5C3AE1A6822F040721A603B
:101508001A6842EA07621A60DA6822F0407242EA10
:1015180001628504DA607FF5B5AE1A6822F0406290
:101528001A601A6842EA87621A60DA6822F0406232
:1015380042EA81624404DA607FF5A7AE1A6822F0B5
:1015480040521A601A6842EA07721A60DA6822F092
:10155800405242EA0172DA6097E600BF036803F17D
:1015680038422DE9F04F920A584DAA5C02F01F0547
:1015780052090124022A04FA05F400F08C80032A97
:1015880000F08E80012A3CD001F003077A1E012A60
:10159800C1F3810CC1F300188088C1F3411135D91A
:1015A800C60700F19780850700F1A380440700F182
:1015B800B180020700F1BF80C60600F1CD80850624
:1015C80000F1DB80440600F1E980020600F1F780B3
:1015D800C60500F10581850500F11381440500F178
:1015E8002181020500F12F81C60400F13D818504A7
:1015F80000F14B81440400F15981020455D4BDE83F
:10160800F08F334A55692C435461BDE700242246C4
:101618004FF0010E4FF0030904E00132102A04F1E3
:101628000204ECD00EFA02F636EA0005F5D1D3F83A
:1016380008A009FA04F5ED430AEA050AC3F808A068
:10164800D3F808B00CFA04FA4AEA0B0AC3F808A05F
:10165800B3F804A01FFA8AFA2AEA06069E80B3F8AD
:1016680004A008FA02F646EA0A06B6B29E801E6888
:101678002E401E60D3F800A007FA04F646EA0A06D0
:101688001E60D3F80CA001FA04F605EA0A0A46EA35
:101698000A05DD60C1E70E4A95692C43946173E73A
:1016A8000B4AD5692C43D4616EE71A6822F0404290
:1016B8001A601A6842EA87771F60DA6822F04042A7
:1016C80042EA8171D960BDE8F08F00BF104F03086E
:1016D800001002401A6822F003021A601A683A439E
:1016E8001A60DA6822F003020A438507DA607FF598
:1016F8005DAF1A6822F00C021A601A6842EA870283
:101708001A60DA6822F00C0242EA81024407DA60C1
:101718007FF54FAF1A6822F030021A601A6842EA61
:1017280007121A60DA6822F0300242EA0112DA601F
:1017380002077FF541AF1A6822F0C0021A601A68E2
:1017480042EA87121A60DA6822F0C00242EA81127D
:10175800C606DA607FF533AF1A6822F440721A6061
:101768001A6842EA07221A60DA6822F4407242EAEA
:1017780001228506DA607FF525AF1A6822F44062F7
:101788001A601A6842EA87221A60DA6822F440620C
:1017980042EA81224406DA607FF517AF1A6822F41C
:1017A80040521A601A6842EA07321A60DA6822F46C
:1017B800405242EA0132DA6002067FF509AF1A6840
:1017C80022F440421A601A6842EA87321A60DA68DC
:1017D80022F4404242EA8132C605DA607FF5FBAE68
:1017E8001A6822F440321A601A6842EA07421A60FC
:1017F800DA6822F4403242EA01428505DA607FF570
:10180800EDAE1A6822F440221A601A6842EA87424A
:101818001A60DA6822F4402242EA81424405DA601A
:101828007FF5DFAE1A6822F440121A601A6842EA9D
:1018380007521A60DA6822F4401242EA0152DA606A
:1018480002057FF5D1AE1A6822F440021A601A68C0
:1018580042EA87521A60DA6822F4400242EA815268
:10186800C604DA607FF5C3AE1A6822F040721A60C7
:101878001A6842EA07621A60DA6822F0407242EA9D
:1018880001628504DA607FF5B5AE1A6822F040621D
:101898001A601A6842EA87621A60DA6822F04062BF
:1018A80042EA81624404DA607FF5A7AE1A6822F042
:1018B80040521A601A6842EA07721A60DA6822F01F
:1018C800405242EA0172DA6097E600BF10B5040997
:1018D800013C052C17D80D4B33F8142000F00F00ED
:1018E80042FA00F313F001030DD0012303FA00F0CC
:1018F800013810402EF066FA054A064B125D104476
:1019080003EBC00010BD002010BD00BFFC4303085E
:10191800084403082C4900202DE9F04F4A484B4B56
:101928004B4C4FF090414FF0010A4FF002094FF035
:1019380004084FF0080C4FF0100E20274026802591
:1019480030F8022B12F0010F03D01960A3F804A09D
:10195800083312F0020F03D01960A3F8049008337B
:1019680012F0040F03D01960A3F80480083312F0B2
:10197800080F03D01960A3F804C0083312F0100F41
:1019880003D01960A3F804E0083312F0200F02D046
:1019980019609F80083312F0400F02D019609E80B2
:1019A800083312F0800F02D019609D80083312F4BA
:1019B800807F05D04FF4807B1960A3F804B008330A
:1019C80012F4007F05D04FF4007B1960A3F804B02F
:1019D800083312F4806F05D04FF4806B1960A3F8B8
:1019E80004B0083312F4006F05D04FF4006B19608F
:1019F800A3F804B0083312F4805F05D04FF4805B7D
:101A08001960A3F804B0083312F4005F05D04FF44E
:101A1800005B1960A3F804B0083312F4804F05D0B6
:101A28004FF4804B1960A3F804B00833D20B04D0EC
:101A38004FF4004219609A80083301F58061A14291
:101A48007FF47EAFBDE8F08FFC4303082C490020EB
:101A580000180048002867D003682DE9F04F03F10B
:101A680038445C4EA40A0125345D04F01F0664095D
:101A7800022C05FA06F558D0032C00F0A580012C9D
:101A880058D08088B0FA80F4C4F11F04A4B2E508E5
:101A980003EB850504F007042E6AA4000F27A7406E
:101AA80026EA07062E622E6A01F00307A2407C1E72
:101AB8003243012CC1F3810CC1F300182A62C1F32F
:101AC80041113CD9C60700F18980850700F195804E
:101AD800440700F1A380020700F1B180C60600F1B7
:101AE800BF80850600F1CD80440600F1DB80020648
:101AF80000F1E980C60500F1F780850500F1058150
:101B0800440500F11381020500F12181C60400F1AA
:101B18002F81850400F13D81440400F14B810204CA
:101B280000F15981BDE8F08F70472B4CA669354309
:101B3800A561A6E7284C666935436561A1E70024DD
:101B480022464FF0010E4FF0030904E00132102A3B
:101B580004F10204E6D00EFA02F636EA0005F5D1E1
:101B6800D3F808A009FA04F5ED430AEA050AC3F810
:101B780008A0D3F808B00CFA04FA4AEA0B0AC3F82A
:101B880008A0B3F804A01FFA8AFA2AEA06069E807B
:101B9800B3F804A008FA02F646EA0A06B6B29E802E
:101BA8001E682E401E60D3F800A007FA04F646EA25
:101BB8000A061E60D3F80CA001FA04F605EA0A0A20
:101BC80046EA0A05DD60C1E7034CE6693543E5618D
:101BD80057E700BF104F0308001002401A6822F0B0
:101BE80003021A601A683A431A60DA6822F003029C
:101BF8000A438507DA607FF56BAF1A6822F00C029A
:101C08001A601A6842EA87021A60DA6822F00C023F
:101C180042EA81024407DA607FF55DAF1A6822F074
:101C280030021A601A6842EA07121A60DA6822F06B
:101C3800300242EA0112DA6002077FF54FAF1A68F4
:101C480022F0C0021A601A6842EA87121A60DA683B
:101C580022F0C00242EA8112C606DA607FF541AF7F
:101C68001A6822F440721A601A6842EA07221A6057
:101C7800DA6822F4407242EA01228506DA607FF5CA
:101C880033AF1A6822F440621A601A6842EA87225F
:101C98001A60DA6822F4406242EA81224406DA6075
:101CA8007FF525AF1A6822F440521A601A6842EA92
:101CB80007321A60DA6822F4405242EA0132DA60E6
:101CC80002067FF517AF1A6822F440421A601A68B4
:101CD80042EA87321A60DA6822F4404242EA8132E4
:101CE800C605DA607FF509AF1A6822F440321A6037
:101CF8001A6842EA07421A60DA6822F4403242EA75
:101D080001428505DA607FF5FBAE1A6822F44022AD
:101D18001A601A6842EA87421A60DA6822F4402296
:101D280042EA81424405DA607FF5EDAE1A6822F492
:101D380040121A601A6842EA07521A60DA6822F4F6
:101D4800401242EA0152DA6002057FF5DFAE1A68F6
:101D580022F440021A601A6842EA87521A60DA6866
:101D680022F4400242EA8152C604DA607FF5D1AE1D
:101D78001A6822F040721A601A6842EA07621A600A
:101D8800DA6822F0407242EA01628504DA607FF57F
:101D9800C3AE1A6822F040621A601A6842EA876283
:101DA8001A60DA6822F0406242EA81624404DA602A
:101DB8007FF5B5AE1A6822F040521A601A6842EAF6
:101DC80007721A60DA6822F0405242EA0172DA6059
:101DD80002047FF5A7AE1A6822F040421A601A681A
:101DE80042EA87771F60DA6822F0404242EA81714E
:101DF800D960BDE8F08F00BF002852D0036803F116
:101E080038422DE9F04F920A504DAA5C02F01F05A6
:101E180052090124022A04FA05F443D0032A00F0E7
:101E28009080012A43D001F003077A1E012AC1F3EA
:101E3800810CC1F300188088C1F341113CD9C60751
:101E480000F18880850700F19480440700F1A280A2
:101E5800020700F1B080C60600F1BE80850600F1D9
:101E6800CC80440600F1DA80020600F1E880C6055D
:101E780000F1F680850500F10481440500F1128126
:101E8800020500F12081C60400F12E81850400F1CD
:101E98003C81440400F14A81020400F15881BDE804
:101EA800F08F70472A4A95692C439461BBE7284A0A
:101EB80055692C435461B6E7002422464FF0010EC1
:101EC8004FF0030904E00132102A04F10204E6D0BD
:101ED8000EFA02F636EA0005F5D1D3F808A009FA99
:101EE80004F5ED430AEA050AC3F808A0D3F808B0D8
:101EF8000CFA04FA4AEA0B0AC3F808A0B3F804A0DB
:101F08001FFA8AFA2AEA06069E80B3F804A008FA9D
:101F180002F646EA0A06B6B29E801E682E401E6089
:101F2800D3F800A007FA04F646EA0A061E60D3F8BA
:101F38000CA001FA04F605EA0A0A46EA0A05DD6079
:101F4800C1E7034AD5692C43D4616CE7104F0308F5
:101F5800001002401A6822F003021A601A683A4315
:101F68001A60DA6822F003020A438507DA607FF50F
:101F78006CAF1A6822F00C021A601A6842EA8702EB
:101F88001A60DA6822F00C0242EA81024407DA6039
:101F98007FF55EAF1A6822F030021A601A6842EACA
:101FA80007121A60DA6822F0300242EA0112DA6097
:101FB80002077FF550AF1A6822F0C0021A601A684B
:101FC80042EA87121A60DA6822F0C00242EA8112F5
:101FD800C606DA607FF542AF1A6822F440721A60CA
:101FE8001A6842EA07221A60DA6822F4407242EA62
:101FF80001228506DA607FF534AF1A6822F4406260
:102008001A601A6842EA87221A60DA6822F4406283
:1020180042EA81224406DA607FF526AF1A6822F484
:1020280040521A601A6842EA07321A60DA6822F4E3
:10203800405242EA0132DA6002067FF518AF1A68A8
:1020480022F440421A601A6842EA87321A60DA6853
:1020580022F4404242EA8132C605DA607FF50AAFCF
:102068001A6822F440321A601A6842EA07421A6073
:10207800DA6822F4403242EA01428505DA607FF5E7
:10208800FCAE1A6822F440221A601A6842EA8742B3
:102098001A60DA6822F4402242EA81424405DA6092
:1020A8007FF5EEAE1A6822F440121A601A6842EA06
:1020B80007521A60DA6822F4401242EA0152DA60E2
:1020C80002057FF5E0AE1A6822F440021A601A6829
:1020D80042EA87521A60DA6822F4400242EA8152E0
:1020E800C604DA607FF5D2AE1A6822F040721A6030
:1020F8001A6842EA07621A60DA6822F0407242EA15
:1021080001628504DA607FF5C4AE1A6822F0406285
:102118001A601A6842EA87621A60DA6822F0406236
:1021280042EA81624404DA607FF5B6AE1A6822F0AA
:1021380040521A601A6842EA07721A60DA6822F096
:10214800405242EA0172DA6002047FF5A8AE1A68CA
:1021580022F040421A601A6842EA87771F60DA68FC
:1021680022F0404242EA8171D960BDE8F08F00BF99
:1021780010B1036882881A85704700BF10B10368E0
:1021880082889A61704700BFF8B50468037B2268AB
:1021980002259D402A420DD1216804229A4011420D
:1021A80018BF62602168082202FA03F3194218BFB7
:1021B8006360F8BD1749184A0B684FF6FE7633403E
:1021C8000B6013899F07FCD5134B1A891606FCD49C
:1021D8001B89D90718D4014610480F4A0368104EC6
:1021E8004FF6FE773B40036065609388306823F0C4
:1021F80003031B041B0C9380FFF7C0FF094A0C68FC
:102208000B7B00211170C7E7034B9A891A89D20703
:10221800E1D5FAE708040240003C00401C040240F3
:10222800144800202139002038B100298388026829
:1022380014BF002110218B40936170470E4B1B88FF
:1022480001463BB90D4B0E4A1B7810680BB981F05B
:102258000101E9E70B4B5A691AB118B91A681060FD
:1022680058747047084A18681188084A92FBF1F2B6
:10227800012102605974704700710020027100202A
:1022880004710020087100202071002020A107009F
:1022980010B40A4B0A4A1C7801238340234052F8A1
:1022A800200029B9B3FA83F149095DF8044BBBE76B
:1022B800191C18BF01215DF8044BB5E7F370002025
:1022C800F470002030B1036882881B8A1A4214BF58
:1022D80001200020704700BF38B590F8593003B985
:1022E80038BD04461846FFF7F1FA0546FFF7EAFF3E
:1022F80001460028F4D1D5B12023E871AB712846F6
:10230800FFF77AFD2146104B41F8103F284624F08C
:102318003FF8AB88B3FA83F3C3F11F035A1CDFD02D
:1023280001229A4009490B6813430B6038BD2946BE
:10233800FFF762FD2146044B41F8103F284624F080
:1023480027F80122EEE700BF150700080004014046
:1023580038B5044600F11405FFF7BEFF236E80224E
:102368006B21284698476420FEF760FD236E0722FC
:102378006821284698476420FEF758FD236E0022FE
:102388006B21284698476420FEF750FD236E0122F2
:102398006B21284698470F20FEF748FD94F85320F4
:1023A800236E032A8CBF1A2218221B21284698471D
:1023B8000F20FEF73BFD236E18221C212846984764
:1023C8000F20FEF733FD236E94F852201A21284679
:1023D80098470F20FEF72AFD236E94F85420192100
:1023E800284698476420FEF721FD236E10223721E6
:1023F800284698470F20FEF719FD2846236E01222C
:10240800382198470F20BDE83840FEF70FBD00BFC0
:102418002DE9F0410B4E346873691C400FD0DFF88A
:1024280028800127B4FA84F3C3F11F0307FA03F5E0
:1024380058F8230003689847AC437561F2D1BDE8AA
:10244800F08100BF00040140AC7000202DE9F0418C
:102458000B4E346873691C400FD0DFF828800127C1
:10246800B4FA84F3C3F11F0307FA03F558F82300FD
:1024780003689847AC437561F2D1BDE8F08100BFAD
:1024880000040140AC7000202DE9F0410B4E346887
:1024980073691C400FD0DFF828800127B4FA84F351
:1024A800C3F11F0307FA03F558F823000368984798
:1024B800AC437561F2D1BDE8F08100BF0004014072
:1024C800AC7000202DE9F0410B4E346873691C4054
:1024D8000FD0DFF828800127B4FA84F3C3F11F0373
:1024E80007FA03F558F8230003689847AC43756169
:1024F800F2D1BDE8F08100BF00040140AC700020BB
:102508002DE9F0410B4E346873691C400FD0DFF899
:1025180028800127B4FA84F3C3F11F0307FA03F5EF
:1025280058F8230003689847AC437561F2D1BDE8B9
:10253800F08100BF00040140AC7000202DE9F0419B
:102548000B4E346873691C400FD0DFF828800127D0
:10255800B4FA84F3C3F11F0307FA03F558F823000C
:1025680003689847AC437561F2D1BDE8F08100BFBC
:1025780000040140AC7000202DE9F0410B4E346896
:1025880073691C400FD0DFF828800127B4FA84F360
:10259800C3F11F0307FA03F558F8230003689847A7
:1025A800AC437561F2D1BDE8F08100BF0004014081
:1025B800AC7000200B490C4A0C4808B58B6943F0F5
:1025C80001038B61136843F4805313600021402298
:1025D80030F06BF8064B4FF0FF321A60C3F8032057
:1025E80008BD00BF0010024000000140AC70002090
:1025F800EC7000202DE9F041044618460D461646B9
:1026080098462CF015FF2768E6722844A0722946E0
:102618007D69434632462046AC46BDE8F0416047F6
:10262800036810B504461B689847236820469B68D2
:102638009847A37B0133A37310BD00BF10B503688F
:1026480004469B689847FF2301226373227310BDD9
:1026580008B5FFF73BF940B12C2282710022C27104
:102668002021BDE80840FFF7C7BB08BD40F2E933A9
:1026780000E09BB10289013B12F0020F9BB2F8D037
:10268800017340F2E93300E043B10289013B12F0E3
:10269800010F9BB2F8D0007BC0B270470C4A904241
:1026A80009D00C4B984210D003F58063984201D0B2
:1026B800FF2070470223084A02EB03135A890132AC
:1026C80092B25A815889C0B270470123F3E700BF1C
:1026D8000030014000380040B07D0020F8B50446C5
:1026E800806816461F4610B1036882881A8541F033
:1026F80080016068FFF7BAFF65684FF0000CAB898E
:102708004FF47A714FF6FF734FF0FF0E674502D111
:1027180031E099421BD02889013910F0020089B2B2
:10272800F7D085F80CE04FF47A7102E091B2994243
:102738000DD0288910F0010001F1FF32F6D02A7B74
:10274800D2B20EB1327001360CF1010CDEE70E4B3D
:102758009D4208D0A3F578439D4213D003F58063CA
:102768009D4208D10220094B03EB00104389013335
:102778009BB243814389A36813B11A689B8893610C
:102788000120F8BD0120EEE700300140B07D0020B7
:1027980038B583680446154613B11A689B881385B3
:1027A8006068FFF763FF29466068FFF75FFFA3686B
:1027B80013B11A689B889361012038BD10B504468F
:1027C80080692BF01DF80120FEF7D6FA2046FFF7A6
:1027D800BFFD10226A2104F11400FFF7D9FF64201D
:1027E800FEF724FBA0692AF0F9FF0120BDE810409C
:1027F800FEF7C2BAF8B5434E0446FFF76DFD3778C9
:10280800C7B104F11405A0692BF00EF894F8522012
:102818001A212846FFF7BCFF0120FEF7ADFAA06990
:102828002AF0DCFF2046FDF72BFF94F93E300133F8
:102838005FD0F8BD04F11405A0692AF0F5FF8022E5
:102848006B212846FFF7A4FF9620FEF7EFFA032234
:1028580068212846FFF79CFF9620FEF7E7FA032237
:102868006B212846FFF794FF0F20FEF785FA102208
:102878006A212846FFF78CFF0F20FEF77DFA3A46BB
:102888006C212846FFF784FF0F20FEF775FA94F8AD
:10289800542019212846FFF77BFF0F20FEF76CFA1A
:1028A80018221B212846FFF773FF0F20FEF764FA52
:1028B80010221C212846FFF76BFF0F20FEF75CFA59
:1028C800102237212846FFF763FF0F20FEF754FA3E
:1028D800012238212846FFF75BFF0F20FEF74CFA4C
:1028E800A0692AF07BFF0120FEF746FA0123337026
:1028F80089E794F93C3001339BD10620BDE8F840C4
:1029080002F034BFA81B0020F8B505015A4C5B4BF8
:10291800625961199A4204EB050704BF01230B733E
:102928000646387A2AF0E0FB3B7A03F01F015B0980
:102938000122022B02FA01F278D0032B71D0012B6D
:1029480067D0631901361879FEF7C0FFF6B207465B
:1029580010B11223C671837163195879FEF7B6FF57
:1029680010B11323C671837163199879FEF7AEFF0E
:1029780010B11423C671837166190E21F279384695
:10298800FFF768F87079FEF7A1FFF2790E21FFF7DB
:1029980061F8B079FEF79AFFF2790E21FFF75AF83D
:1029A8006359374A934251D0344A934259D0354AF1
:1029B800934240D02C44227B002A2FD101200224AC
:1029C8009A8822F480521204120C9A80998889B24B
:1029D80041F4805199801A8802F4415242F44572B8
:1029E800024322431A809A8822F470621204120C5D
:1029F80042F4E0629A809A8B22F400621204120C6C
:102A080007219A8319821A8892B242F040021A80EA
:102A1800F8BD1D4B996A0A439A6292E70020044662
:102A2800CEE7194B19690A431A618AE7164BD96828
:102A38000A43DA6085E702F5EA32116941F4004198
:102A48001161116921F400411161B3E702F5604297
:102A5800D16841F48051D160D16821F48051D160AE
:102A6800A8E702F5EC32116941F48041116111695E
:102A780021F4804111619DE7B07D002000380040BD
:102A880000300140003C004000100240427A02B988
:102A9800704710B504460368406804F10A01984776
:102AA8000023637210BD00BF437A5A1C0344D2B29C
:102AB80042729972037A934200D802B9704710B5EE
:102AC80004460368406804F10A01984700236372CA
:102AD80010BD00BF30B40B4D002305F1200101E00B
:102AE800272B0CD011F8132082424FEA430403F13C
:102AF8000103F5D12C4494F8210030BC7047002024
:102B080030BC70471C28030870B5448806460D463B
:102B1800C4F30B042246002128462FF0C6FD336972
:102B2800094A934209D3094A934206D222462846C3
:102B38001946BDE870402DF0A1BA23B121462846B8
:102B4800BDE87040184770BDD08D0308C48E0308D7
:102B5800064B07498B4202D30023184670471A8850
:102B6800C2F30B029042F8D01433F3E770890308DC
:102B7800D08D0308024A136823EA000010607047EA
:102B880048820020F8B5174D2B78A32B28D16B78F5
:102B9800BE2B25D1022229464FF6FF70FDF74AFDCC
:102BA800114FAC1C22884AB1A618BE4218D2052A79
:102BB80016D92146FDF73EFD3446F3E721460222A9
:102BC800FDF738FD0222A118FDF734FD0634074B46
:102BD800641B1C8041F60F53C31A58425841F8BD74
:102BE8000020F8BD00F0030800000408702E002043
:102BF8002DE9F04FDFF848914C4F8BB00326A7EB37
:102C080009071822002104A82FF04FFD484BCDF8E2
:102C1800109005971A69120604D5464A5A6002F1BF
:102C280088325A6001228DF824203422DA60424B1F
:102C3800424C1B88ADF800300222694604A8FDF713
:102C4800E9FE022269464FF6FF70FDF7F3FCDFF854
:102C5800F4A080464FF0000B544536D30AAC00254B
:102C680024F8245D0222214604A8FDF7D3FE02229F
:102C780021464046FDF7DEFC40BAC043ADF80800E7
:102C8800022202A904A8FDF7C5FE079860B106ABA9
:102C9800C0F10402294618442FF007FD069904A83C
:102CA800FDF75EFE079508909DF82430089A23B139
:102CB8001F490B6943F080030B61013E2DD0002AA8
:102CC8009FD1FFF75FFF50B32CE065888DF80DB0FA
:102CD800C5F30B05AB1DADF808302388C3F30B0211
:102CE800ADF80A201B0B062202A904A88DF80C30A7
:102CF800FDF790FE062202A94046FDF79BFC61689D
:102D080080462A4604A8FDF785FE616840462A46A3
:102D1800FDF790FC143480469EE7002AD1D00520A8
:102D280002F024FD0BB0BDE8F08F00BF00000408DE
:102D380000200240230167458A2803087089030898
:102D480000F00308D08D03080378202B024600F119
:102D58000100F9D0092BF7D02D2B2CD02B2B03BF3A
:102D68005378B7EE000A0246B7EE000AA3F1300125
:102D7800C8B209289FED467A10D8F2EE046A07EE29
:102D8800901AF8EEE77A12F8013FE7EE267AA3F1F7
:102D98003001C8B20928B0EE677AF0D92E2B4CD092
:102DA80003F0DF03452B0BD0F7EE007A67EE276AB6
:102DB80020EE260A70475378BFEE000A0246D5E790
:102DC80010B451782D2959D02B290ABF9178501C5D
:102DD800901C0024A1F13003092B53D8002303EBE6
:102DE800830301EB430310F8011FA1F13002092A04
:102DF800A3F13003F3D9B3F59A7F28BF4FF49A7340
:102E0800072B42D9DFED236A1A46F7EE007A083A13
:102E1800072A67EEA67AFAD803F007032BB1F2EE79
:102E2800046A013B67EEA67AFBD124B3C7EE276A92
:102E38005DF8044B20EE260A70475378A3F1300161
:102E4800C8B2092802F10102AAD8F2EE046AF0EE2B
:102E5800665A07EE901AF8EEE77A12F8013F87EE05
:102E6800A66AA3F13001C8B2092866EEA56A37EE52
:102E7800067AEED994E767EE276AD9E7901C91782D
:102E88000124A7E7F7EE007ACFE7F7EE007AC5E767
:102E98000000000020BCBE4CB5EEC00ADFED317A60
:102EA800F1EE10FACCBF30EE270A30EE670ADFEDFC
:102EB8002E7A20EE270A30B5FDEEC07A87B017EEDD
:102EC800904A054684EAE470002303A9A0EBE47065
:102ED80001930093029321F099FC002CACBF2023AE
:102EE8002D2303A88DF800302CF0A2FA012803A99D
:102EF80024D002282DD0032805BF30236846684611
:102F08008DF801302FF0F7FB68462CF091FA033862
:102F1800C4B22246694628462FF04BFC00232B55A5
:102F280028462CF085FA2E22431C2A540DEB040166
:102F3800E8182FF0FDFB284607B030BD302368465F
:102F48008DF801308DF802308DF803302FF0D3FB67
:102F5800DAE7302368468DF801308DF802302FF01B
:102F6800CAFBD1E76F12033A00007A442DE9F04119
:102F7800064615460846B6FBF2F43CB905FB146450
:102F8800124B1B5D00F8013BBDE8F081B4FBF2F782
:102F980067B90E4B05FB174705FB1464DA5D00F8AB
:102FA800012B1B5D00F8013BBDE8F081B7FBF2F88F
:102FB800B8F1000F02D04046FFF7D8FF05FB18789C
:102FC800024B13F8082000F8012BE3E7C04F030871
:102FD80030B402681146531C036011F8024B0160BB
:102FE800D31C517803609378151D05601B0443EAD0
:102FF8000123D078234343EA006030BC704700BF08
:103008000368591C1A46016012F8021B02605878BE
:1030180041EA0020704700BF03685A1C0260187814
:10302800704700BF38B50446006815462DF026F8ED
:1030380022682A44226038BD036810B40A0A5C1C5E
:1030480004601A7003685A1C026019705DF8044B1A
:10305800704700BF03685A1C026010B419700368F7
:103068000A0A5C1C04601A7003680A0C5C1C046081
:103078001A700368090E5A1C026019705DF8044B37
:10308800704700BF03685A1C026019700368090A78
:103098005A1C0260197070472DE9F047002488B067
:1030A80080460F461E46A14605AD531C0393117872
:1030B80039B3252933D1931CCDF810900393507858
:1030C80030284ED04FF0000AA0F13003DBB2092BB4
:1030D80042D96C2819D0642800F0938024D8252878
:1030E8001CD063D9582876D063281BD13178404644
:1030F800B847039A531C0393117804360134002906
:10310800D7D1204608B0BDE8F087039B5A1C03922C
:103118001B78642B7CD02AD8252B54D125214046F6
:103128000134B847039AC0E7732833D044D97528C7
:103138004FD106F1040E30682B4600220A2176464C
:10314800FDF76EF9049A0095534639464046FDF757
:10315800A5F9039A0444A8E704AA03A924F0DAF815
:10316800B7E7D31C039390784FF0010AACE7732BB1
:1031780010D05BD9752B3AD0782B96D1A3F1580291
:10318800B2FA82F2306852092B4610210436FDF754
:1031980047F9D7E73368049A009339460023404635
:1031A800FDF77CF904360444039A7EE70028B9D178
:1031B800204608B0BDE8F0876E28B3D1039A33687B
:1031C80004361C6071E72AD9582BD7D0632B8DD0D1
:1031D8006BE77828A6D1A0F15802B2FA82F23068DB
:1031E80052092B461021FDF71BF90436AAE706F110
:1031F800040E30682B4600220A217646FDF710F9A6
:10320800A0E7331D306829461E46FDF7DBF899E72D
:10321800331D306829461E46FDF7D4F892E7002B87
:103228007FF443AF204608B0BDE8F0876E2BC6D0C8
:103238003BE700BF0EB400B584B005AB019053F86E
:10324800042B0649039301A8FFF726FF019B0022E0
:103258001A7004B05DF804EB03B0704799040008D5
:103268000FB430B583B006AB0A490B4853F8042BAA
:10327800096800680193FFF70FFF084C05462068AE
:10328800FDF776FF0028FAD0284603B0BDE83040A5
:1032980004B07047EC290020F02900208C78002029
:1032A800DFED2B7AB4EEE70AF1EE10FA4ADDDFED36
:1032B800296A9FED297A01E0B0EE670AB4EEC70AE1
:1032C800F1EE10FA70EE667AF6DC9FED247AF4EEF1
:1032D800C77AF1EE10FA38D5DFED1E6A9FED207A35
:1032E80001E0F0EE407AF4EEC77AF1EE10FA37EE2C
:1032F800A60AF6D4DFED1B7AB4EEE70AF1EE10FA6F
:1033080014DDDFED137A37EEC00A60EE006A9FED38
:10331800166A9FED167ADFED167AA6EE867A20EE0B
:10332800266AE6EE877AA6EE270A7047DFED117A5D
:10333800B4EEE70AF1EE10FA44BFDFED087A37EE93
:10334800C00AE2E7F0EE407ABFE7B0EE670AD1E7DD
:10335800DB0F4940DB0FC940E4CB1641DB0F49C006
:10336800E4CB16C1DB0FC93F92E741B99730083C5F
:1033780015A82ABEDB0FC9BF09B909E0194690FB99
:10338800F1F301FB13030846002BF7D108467047F9
:103398000146FBE710B507EE901A2DED028BB8EE4B
:1033A800678ADFED217A28EE008A044628EE278A0C
:1033B800B0EE480A2DF0B8F8F0EE408AB0EE480AB0
:1033C8002DF014F8F7EE007A9FED187AF0EE675AB0
:1033D800E8EE875A0023A361B0EE676AC7EEA56AD4
:1033E80063612362E361A8EEC76ABDEC028B77EEE6
:1033F800C07AB6EE007AF8EE005A27EE877A20EE09
:10340800250A27EE267A26EE266A67EEA67A20EEA9
:10341800260A84ED046AC4ED017A84ED007A84ED0D
:10342800027A84ED030A10BD27D4D236F304353F5F
:1034380010B44C09012250F8243001F01F0102FA9F
:1034480001F10B4340F824305DF8044B704700BF8E
:103458004B0901F01F0150F82320012303FA01F161
:10346800114214BF18460020704700BF2DE9F84FDD
:10347800294A137803F0FF04002BFAD1DFF8A8904B
:10348800DFF8A880D9F80000244F254D012388F8DB
:103498000030FEF76DFE05202AF040F920462AF09C
:1034A8003DF906202AF03AF920462AF037F93E7805
:1034B800042046F001062AF031F930462AF02EF9A8
:1034C8002B8893B1DFF868A0164E1AF804B00720CD
:1034D8002AF024F958462AF021F91AF804202B88F2
:1034E80032550134A4B2A342EFD807202AF016F9C6
:1034F800FF202AF013F93C7804202AF00FF920461F
:103508002AF00CF9D9F80000FEF738FE002388F8F5
:103518000030BDE8F88F00BF21390020353B00207E
:1035280008020020443B0020144800202D3B0020C6
:10353800243900202DE9F041474E3068FEF718FE87
:10354800464B1B78012B78D05FD3022B0AD1DFF8CA
:103558002C81082388F800300D254FF4C373404FA1
:103568003B8010E0DFF814813D4F98F8003003F0FD
:103578004003002B14BF4FF4F0734FF4C3733B8028
:1035880014BF10250D25002404F11000C0B22AF044
:10359800C5F8013401202AF0C1F8A3B2AB42F3D335
:1035A80098F800402F4D00202AF0B8F820462AF05D
:1035B800B5F82D4B1C7802202AF0B0F820462AF0E6
:1035C800ADF82A4B1C7803202AF0A8F820462AF0E8
:1035D800A5F8274B1C78042004432AF09FF82046BE
:1035E8002AF09CF83068FEF7C9FD3A882148002186
:1035F8002FF05BF82B7833B11F4B1B7833B30023C4
:103608002B70BDE8F081BDE8F081A0202AF086F893
:1036180000202AF083F800F00603022BDFF85C8014
:1036280007D000F00500012803D1482388F80030AE
:1036380008E0082388F800308EE7DFF84080482348
:1036480088F8003010254FF4F07388E7FFF70EFF75
:1036580000232B70BDE8F081144800201848002092
:1036680008020020000000201F48002020480020F9
:10367800353B0020443B00202D3B00200A0200205F
:103688002DE9F0472A4F2B4D2B4C82463868894646
:10369800FEF76EFD0120FDF7C9FB0026A8464AFA91
:1036A80006F3DA0720683DD5FEF768FD2868FEF7BF
:1036B80065FD0120FDF7BAFB2868FEF759FD0136C4
:1036C8000120FDF7B3FB042EE9D12068FEF756FD73
:1036D8002868FEF753FD0120FDF7A8FB2868FEF7D0
:1036E80047FD0120FDF7A2FB002529FA05F3DB07BA
:1036F80020681AD5FEF742FDD8F80000FEF73EFD17
:103708000120FDF793FBD8F80000FEF731FD0135E5
:103718000120FDF78BFB142DE7D13868BDE8F04791
:10372800FEF72CBDFEF724FDC0E7FEF721FDE3E719
:10373800202A0020242A00201C2A002010B54FF43B
:103748007A7444434FF4C8710020FFF799FF282189
:10375800B4FBF1F101F03F014FF420630120B4FB09
:10376800F3F441EAC411BDE8104089E7F0B55B4BBA
:103778005B4A97B01968914200AF00F0A38059499D
:10378800594A00234FF47000C1F888003B607B6001
:10379800136843F48033136003E03B68B3F5A04F2C
:1037A80009D0136803F400337B603B6801333B6046
:1037B8007B68002BF1D04C4B1B6813F4003318BF07
:1037C80001237B607B68012B52D0464C464B474A0D
:1037D800E260474A596A11605A6A42F080725A6236
:1037E8005A6942F4FC025A610025032207F10801D4
:1037F800012341F6FF764FF09040FD60BE603A73BA
:10380800BB731EF05BFC4FF6FF7307F108013948E4
:10381800BB601EF053FC07F108013748374E1EF015
:103828004DFC07F1080136481EF048FC07F1080175
:1038380034481EF043FC07F1080133481EF03EFCF3
:1038480007F108001EF04AFABB683049304AA1FB6C
:10385800031330499B0CF0204FF0070E5C370B60C8
:10386800566084F823009560C2F800E0BD46F0BDBC
:10387800294A1D4B122111605A685A605A685A60C9
:103888005A6842F480625A605A6822F47C125A607C
:103898005A6842F4E8125A601A6842F080721A6054
:1038A8001A689201FCD559680F4A21F00301596042
:1038B800596841F002015960536803F00C03082B62
:1038C800FAD182E700221A6062B6144B1B6883F3B0
:1038D8000888134B1B689847FEE700BFFC9F002031
:1038E800EFBEADDE00ED00E0001002400005FA0575
:1038F8006051002000040048000800483F190100FA
:10390800000C0048001000480014004883DE1B43E8
:1039180010E000E02C7100200020024000D8FF1FBA
:1039280004D8FF1F064A00235168814202F11C0295
:1039380004D001330C2BF7D100207047D8B2704760
:10394800A000002070B50F4C0F4DC0EBC00004EB79
:103958008004686926693043686182B09209667B91
:10396800A1600025012101A863618DF804608DF82C
:1039780005208DF806508DF807101EF0CBF802B020
:1039880070BD00BFA000002000100240074BC0EB34
:10399800C00030B403EB8000054C056963692B4314
:1039A80063610176427630BC704700BFA0000020FA
:1039B800001002402DE9F04F554C54F8204083B0D8
:1039C800002C60D0656D1F469046524B6A68E264D1
:1039D800A160236004F15A014FF4807304F5AD72BD
:1039E8006161A261E36023610646287E29F07CFBC1
:1039F800E86858B1FFF796FF721CD2B20C21FFF7A6
:103A0800C5FFE36CEA6822632433A364A86890B115
:103A1800FFF788FF721C8146D2B20B21FFF7B6FF71
:103A28002346EA7E3C494846FFF78CFFE36CAA68C8
:103A380062632833636494F85900FDF747FF8146B1
:103A480094F85800FDF742FF3A07824695F819B0F6
:103A58001DD5B9F1000F1AD017F0110F4FF00B0355
:103A680006F1010614BF4E213E2189F8063089F877
:103A780007605A464846FDF7EDFFFB0743D5236B21
:103A88006BB3636B5BB3204603B0BDE8F08F17F0F0
:103A9800010F0CBF2E274E2718F0020F0DD0B9F1D9
:103AA800000F0AD00B22731C89F8062089F807300A
:103AB80048465A463946FDF7CDFF18F0010FDED0CB
:103AC800BAF1000FDBD001360C238AF807605A469A
:103AD80039468AF806305046FDF7BCFFCFE72B7F02
:103AE800AA7E8DF804209B090021012201A88DF8E7
:103AF80005308DF806108DF807201EF00BF82046CB
:103B080003B0BDE8F08F4846FEF732FBB7E700BFC9
:103B1800F82900208C280308290700080348D0F852
:103B28003C3113B100F59A7018477047A000002087
:103B38000348D0F8203113B100F58C70184770474E
:103B4800A00000200348D0F804310BB1FC3018471E
:103B5800704700BFA00000200348D0F8E8300BB140
:103B6800E0301847704700BFA00000200348D0F895
:103B7800CC300BB1C4301847704700BFA0000020FC
:103B88000348D0F8B0300BB1A8301847704700BFD1
:103B9800A00000200348D0F894300BB18C301847AF
:103BA800704700BFA00000200248836F0BB170303F
:103BB80018477047A00000200248C36D0BB154306D
:103BC80018477047A00000200248036C0BB138303A
:103BD80018477047A00000200248436A0BB11C3008
:103BE80018477047A00000200248836803B11847AF
:103BF800704700BFA00000201749184B184A194801
:103C080010B4D1F8884044F47004C1F888401C68A6
:103C180044F001041C605C6822405A601A6822F073
:103C2800847222F480321A601A6822F480221A60A0
:103C38005A6822F4FE025A60DA6A22F00F02DA6247
:103C48001A6B002410404FF0006218639C608A6071
:103C58005DF8044B704700BF00ED00E00010024023
:103C68000CC07FF8CCFC00FF38B50B4C23688BB137
:103C78005A68821A002A054604DA0CE05A68AA1A19
:103C8800002A07DB9A68226018461A68904723685A
:103C9800002BF3D138BD38BD283100200B4B002252
:103CA80010B4027203F17804012102E0072A09DC4A
:103CB8009979890702D51979815401329C4203F117
:103CC8001403F3D15DF8044B704700BF184F030885
:103CD8002B230370704700BF012310B41321102455
:103CE800122244704171C2700370037183705DF8D1
:103CF800044B704708B511F00BFA024B024ADA6020
:103D0800FEE700BF00ED00E00400FA05024A034B9D
:103D18001278197819F0E8BAC01E0020C11E0020D8
:103D28002DE9F0470569C3681D4028D00F460646AF
:103D38004FF000484FF00009B5FA85F328FA03F26E
:103D4800D2431B3B32611540042B16D8DFE803F041
:103D58003129211903007B6A002B32D003F1FF3A85
:103D68001FFA8AFAC7F824903C6A34B123682046BF
:103D7800514698476468002CF8D1002DDCD1BDE885
:103D8800F0873868716B036889B29847002DD3D1E2
:103D9800F5E77868B16B036889B29847002DCBD1F5
:103DA800EDE7B868F16B036889B29847002DC3D175
:103DB800E5E7F868316C036889B29847002DBBD1F4
:103DC800DDE7F36A1FFA83FACEE700BF2DE9F04F6B
:103DD8002DED028BA0F10A0389B00C46E72B00F207
:103DE8006486DFE813F01C0162066206620662065A
:103DF800620662066206620662066206620662067B
:103E0800620662066206620662066206620662066A
:103E18006206620662068005620662066206700530
:103E28006206620662065B066206CD056206B40596
:103E38006206A80562069F05620635066206210627
:103E48006206620662061A061206620638036206EF
:103E58006206310362060903620662066206F6021A
:103E68006206620662066206D7026206FC00620605
:103E780031046E0162066206620662066206620626
:103E880062062D01620603046206CF036206590327
:103E98006206450362066206620662061E05E304C0
:103EA800DC04AB04E800620662065B0236026206C6
:103EB800FF01E3016206620662066206D801620635
:103EC8006206B701620662066206A8019101C30292
:103ED80081026206620662067202620662068B044C
:103EE800620662066206620662066206620662068A
:103EF80062066206620662066206620662061E05BF
:103F08006206620662066206620662066206620669
:103F18006206620662066206620662066206620659
:103F28006206620662066206620662066206620649
:103F38006206620662066206620662066206620639
:103F48006206620662066206620662066206620629
:103F58006206620662066206620662066206620619
:103F68006206620662066206620662066206620609
:103F780062066206620662066206620662066206F9
:103F880062066206620662066206620662066206E9
:103F980062066206620662066206620662066206D9
:103FA80062066206620662066206620662066206C9
:103FB800620680045604AC4E337853B1AB4F0025EB
:103FC80037F8021F2046FFF75DF833780135AB421A
:103FD800F6DC012009B0BDEC028BBDE8F08FA24EE3
:103FE8003378002BF5D0A24F0025B846236817F880
:103FF8001520591C21601A7098F8011001EB8101F5
:1040080001EB810101F2EE2189B22046FFF73AF86F
:1040180033780135AB4208F10208E7DCD9E7954D62
:1040280028462BF005FA0028D3DD2B4605442268E4
:1040380013F8011B501C9D4220601170F7D1C8E78E
:1040480019F036F9FF28064600F01E8608A9002553
:1040580001F8125D0DF10D008DF80D5019F028F8DA
:1040680008A800F8115D19F017F808A800F8105D05
:1040780019F006F808A820F8085D18F0F5FF23687D
:104088005A1C22601E7023689DF80D20591C21605F
:104098001A7023689DF80E20591C21601A70236835
:1040A8009DF80F20591C21601A7023689DF8102074
:1040B800591C21601A702046BDF81810FEF7E2FF5F
:1040C80087E70B686C4E01255A1C0A601D700B6847
:1040D800B278591921601A7025F0A8F82368674A40
:1040E80067495F1927601870B1F90010B2F900002C
:1040F800FFF742F923685A19226018703188204660
:10410800FEF7C0FF284665E70A685E4B5E491878E7
:10411800551C2560107022685878551C2560107051
:1041280022689B78501C206013702046C988FEF7CF
:10413800A9FF01204EE7544D08462988FEF7A2FF43
:1041480069882046FEF79EFF2046A988FEF79AFF59
:1041580001203FE74D4D05F16006A9882046FEF78E
:1041680091FFE9882046FEF78DFF29892046FEF752
:1041780089FF2368AA7A591C21601A702368EA7A91
:10418800591C21601A7055F80C1B2046FEF762FF77
:10419800B542E2D11DE73E4952232268501C2060F7
:1041A800137011F8013F002BF7D112E739480023AB
:1041B8002268056803EB4301561C6D5C2660157088
:1041C800026825680A446E1C527826602A700268C4
:1041D80025680A4401339278691C0A2B21602A70E9
:1041E800E6D1F6E62C4D0B682A68591C1278216036
:1041F8001A702B6822689978531C23600023117069
:104208002A6821681A4401335279481C032B20601C
:104218000A70F5D123682A68591C127A21601A702D
:1042280023682A68591CD27821601A7023682A6882
:10423800591C127921601A702B6820465989FEF79B
:1042480021FF2A682368527A591C21601A702A684B
:1042580007E100212046FEF7FDFE20460021FEF77B
:1042680011FF0120B6E600BF54300020664300204D
:10427800AC3200205841002040430020BC77002089
:10428800BE7700202C780020DC2C0020307A00201B
:10429800B428030870410020FC380020A84D0846C7
:1042A8002988FEF7EFFE69882046FEF7EBFEB5F990
:1042B8000430A44AD91782FB0323C1EBA30120468B
:1042C80089B2FEF7DFFE012084E69F4D0846298A61
:1042D800FEF7D8FE698A2046FEF7D4FE2046A98A52
:1042E800FEF7D0FE012075E6DFF894E20027FEB263
:1042F800714600232268501C206016702268501CEA
:1043080020601370226811F8010F0133551C062B29
:1043180025601070EED10137062F0EF1060EE6D19A
:104328008A4900232268501C206017702268501C9C
:1043380020601370226811F8010F0133551C0B2BF4
:1043480025601070EED12368814A581C072120602F
:10435800197023680021581C20601970236892F88E
:10436800F020591C216001201A7033E60B68794A45
:1043780079491078794A5D1C256018702368897816
:10438800581C2060197023689278591C21600120FC
:104398001A701FE60B68724D591C2A7921601A7031
:1043A80023686A79591C21601A7029882046FEF70B
:1043B80069FE2368AA79591C21601A706988204609
:1043C800FEF760FE2368EA79591C216001201A7003
:1043D80000E60B6800255A1C0A6020461D70294615
:1043E800FEF738FE29462046FEF734FE20462946C9
:1043F800FEF730FE0120EDE50B685A4A5A4D117858
:104408005A4A581C2060197011682046FEF722FE8F
:104418002368574A591C127A21601A702988204645
:10442800FEF730FEA9882046FEF72CFE2989204693
:10443800FEF728FE00212046FEF724FE2046002134
:10444800FEF720FE0120C5E5084608224849FEF788
:10445800E9FD0120BEE50B68464A581C91782060AA
:10446800197023685278591C216001201A70B1E52F
:104478000B68394A4049D078384A5D1C2560187065
:1044880023684979581C206019702368D278591C10
:10449800216001201A709DE500212046FEF7F2FDFB
:1044A80000212046FEF7EEFD00212046FEF7EAFD3A
:1044B8002368324D00265A1C22601E7023682A6821
:1044C800591C92F82C2021601A7023682A68591CFC
:1044D80092F8362021601A7023682A68591C92F8CD
:1044E800372021601A7023685A1C22601E702368C6
:1044F8005A1C22601E7023685A1C22601E702B688A
:104508002046598FFEF7BEFD2B682046198FFEF70F
:10451800B9FD23682A68591C92F82E2021601A7068
:1045280023685A1C22601E702B682046598EFEF79D
:10453800A9FD2B682046998EFEF7A4FD012049E5C8
:104548005041002067666666244B00200741002022
:1045580024400020544E0020347800204478002065
:10456800F42C0020A8340020282A002048820020AB
:104578000C500020507800204C450020704100204D
:10458800E3400020AE4E0B687279AE4D591C216095
:104598001A702B682046198CFEF774FD2B6820468C
:1045A800D98BFEF76FFD71892046FEF76BFDB18947
:1045B8002046FEF767FD2B682046598CFEF762FD02
:1045C8002B682046998CFEF75DFDF1892046FEF7A1
:1045D80059FD318A2046FEF755FD2A68236892F86E
:1045E8002620591C216001201A70F3E4944EF378B8
:1045F800002B00F03B830B680822591C21601A70BD
:1046080023680122991821601A7023688E4D591C5D
:104618002A7921601A702368AA78591C21601A70B7
:1046280029882046FEF72EFDE9892046FEF72AFD57
:104638002368F279591C21601A702368EA78591C9A
:10464800216001201A70C5E40A68804D511C0123BD
:104658002160137095F824207D49002A40F0498391
:104668002268501C20601370236841F2B4105A1C51
:10467800085C226041F27812187089582046890A2D
:10468800FEF7E8FCA96A20464908FEF7E3FC01208A
:10469800A0E4704B03F1700522681978501C206063
:1046A800117022685978501C20601170226899781E
:1046B800501C206011702268D978501C206011703D
:1046C80022681979501C2060117022685979501C91
:1046D80020601170226899790733501C9D42206030
:1046E8001170D9D175E45C4D0846E989FEF7CAFC1A
:1046F8002046A989FEF7C6FC01206BE40B68574FDA
:10470800591C3A7821601A703B78002B3FF461AC51
:104718000025EEB230461DF044FD23684278591C4E
:10472800216030461A701DF03CFD01892046FEF7D5
:10473800A9FC3B780135AB42EBDC4AE4484D494ED5
:104748009FED498ADFF84881DFED488A05F12007A7
:104758000EE0FCEEE77ACDED017ABDF804102046B4
:104768000435FEF78FFCBD4206F118063FF431AC64
:10477800717C0029F3D03E4BD5ED007A1B78012BD4
:10478800E7D13C4B1B68DB0440F16882F5EE407AC8
:10479800F1EE10FA40F0918240F2DC51DFE7084672
:1047A80010223549FEF73EFC012013E4334B9B8A67
:1047B800B3F5006F00F26682B3F5806F00F27B827A
:1047C800B3F5007F34BF012702272D4D05F10C06F4
:1047D80055F8041B91FBF7F1204689B2FEF752FC0D
:1047E800B542F5D1274D284F05F10C06B5EC010A65
:1047F800D7ED087A80EE270A2BF04AFE81B22046D0
:10480800FEF740FCB542F1D1204D05F10C0655F8F4
:10481800041B204689B2FEF735FCB542F7D1FFF7F5
:10482800D8BB00258146DFF86C80DFF86CB00595B1
:1048380004950695079501214FF6FF7A34E000BFED
:10484800544E002070410020244B0020806E002030
:10485800CC590020247B002034780020AA45002071
:104868001C330020644A00200000404200E08244DB
:10487800484B0020784E00200C330020D4770020CD
:104888000C7800206C4E0020047E0020502D002063
:10489800DB9B9141E42803084C41002001350B2D96
:1048A80000F0238118F9011F4F1C4AFA05F3F5D0CF
:1048B800DE07F3D5BBF800302B41D807EED506A8A4
:1048C800FEF7B6FDEAE7A84D08462988FEF7DAFBA9
:1048D800A9882046FEF7D6FB20462989FEF7D2FB99
:1048E8000120FFF777BBA14D05F15006287826F087
:1048F800F9FA2368027A591C21601A7023686A78C9
:10490800591C21601A702368AA78591C21601A70F2
:104918002368EA780435591CAE4221601A70E5D143
:10492800FFF757BB0B68924A591C527D2160012042
:104938001A70FFF74FBB8F4D05F1800655F8041F1D
:104948002046FEF787FBAE42F8D1FFF742BB8A4DFF
:1049580005F14006B5F880102046FEF793FB236862
:1049680095F88220591C21601A70236895F88320D5
:104978000435591CAE4221601A70EBD1FFF729BBF0
:104988007B4D0B682A7A591C21601A70A98B204626
:10499800FEF778FB298B2046FEF774FB698B2046CF
:1049A800FEF770FB2368EA7C591C21601A70A98CF9
:1049B8002046FEF767FBE98C2046FEF763FB236879
:1049C800AA7F591C21601A70236895F82020591C69
:1049D80021601A70698C2046FEF754FB2368EA7A36
:1049E800591C21601A70E9682046FEF733FB2368DA
:1049F8002A7C591C21601A70236895F82120591CBB
:104A0800216001201A70FFF7E5BA0B680122991896
:104A1800216010461A70FFF7DDBA08460021FEF73C
:104A280019FB0120FFF7D6BA544D554E05F1300752
:104A380095F90210534B93F906208A4203F10803B3
:104A480036D09E42F7D10835BD42F1D1FFF7C1BA41
:104A58004D4B03F15A0522685979501C206011709A
:104A680022681978501C2060117022685978501CEF
:104A78002060117022689978501C2060117022689B
:104A8800D978501C20601170226819790633501C9F
:104A98009D4220601170DED1FFF79BBA0B683B4A3C
:104AA800581C117820601970DBE40020FFF792BAD7
:104AB80023685A1C2260197029882046FEF7E2FAFA
:104AC8002368EA78591C21601A7023682A79591CCE
:104AD80021601A702368AA79591C21601A7023680A
:104AE8006A79591C21601A70ADE7DFF8ACA000257F
:104AF8004FF008080135C5F1200208FA02F2A5F1C5
:104B080020032AFA05F6164328FA03F31E43252D37
:104B180006F001024FF000030BD01343EAD0E8B2CD
:104B280017F012FA0028E5D0294606A8FEF780FCFF
:104B3800E0E7174B1B78DA0700F1AD800025154E2A
:104B48002F4602E00135252D28D029463046FEF7AC
:104B58007FFC0028F6D0294606A8FEF779FC002835
:104B680077D10137EEE700BF282A0020AC340020B7
:104B78000C5000202040002024400020284800201D
:104B8800E84F0020B84F0020082B0020A834002050
:104B98009C4500200479002090E33FF46B4B6C4D5A
:104BA800B3F850102046FEF76DFA00212046FEF7B4
:104BB80069FA684B19684B0103F02002C1F34003FE
:104BC8001343C1F3800243EA4203C1F3C00243EA3C
:104BD8008203C1F3401243EAC20301F010011943F2
:104BE8002046FEF74FFA04A904222046FEF71AFAD7
:104BF80023682978584A581C20601970118864293C
:104C0800A8BF64212046FEF73DFAB9F1960F47D0B8
:104C180000212046FEF736FA2168B7F1190348BF8C
:104C2800A7F11203A3F3C4034A1C226020461A46C4
:104C38000B7005A9FEF7F6F92368484A581C10219D
:104C48002060197020461188FEF704FA0120FFF74A
:104C5800C1B9394604A8FEF7EBFB82E7F4EEC87A3F
:104C6800F1EE10FA4DDA4FF47A7178E50B68B17805
:104C78003B4A581C2060197023681278591C21601F
:104C88001A70C2E40827A0E523685A1C2260012094
:104C98001E70FFF79FB9069B43F0010306934DE78B
:104CA80023680322591C21601A7023686A78591CEA
:104CB80021601A70B0E7042787E5F4EEC87AF1EEB0
:104CC80010FA3FF569ADF4EEE87AFDEEE77AF1EE19
:104CD80010FA17EE901A2BD86FF4F973303903FBDA
:104CE80001F140F2E73391FBF3F101F2DB5189B2B4
:104CF80035E54B78022B16D0032B0CBF0423012378
:104D0800AEE4FDEEE77A40F2E73217EE903A303B38
:104D180002FB03F388FB0312D917C1EB622101F2EE
:104D2800E93189B21BE5042A34BF0223032397E43F
:104D380040F2F313A1F5836103FB01F140F2E7337D
:104D480091FBF3F101F2DD5189B208E51802002068
:104D580074410020A0430020722E0020A4430020AC
:104D68002878002008B501210220FDF791FA094BA7
:104D78001B7803F00503052B08D000210120FDF75F
:104D880087FA00210846FDF783FAFEE710F052FA89
:104D9800F3E700BFF4290020022828BF022010B43E
:104DA800084C094B207000EB8002C0EBC202074997
:104DB8005DF8044B013003EB4203C0B20B6023F0F3
:104DC800ADB900BF7441002004810020704100206B
:104DD80008B513F0A3FEFDF70BFFBDE8084013F07C
:104DE80085BE00BF38B5434B5A899989914224BF83
:104DF80000225A81198ADA89914224BF0022DA8175
:104E0800DA788AB3072A2FD03B493C4D91F85700EE
:104E1800012400210A282C709C70D9713DD00C28DF
:104E280065D0DFED377A8ABB364C9FED370AA2781A
:104E3800002918BFF0EE407A062A04D8334901EB5E
:104E4800820191ED0F0A217959B3013A032A4DD80D
:104E5800F7EE007A87EE800A2BF01AFB2388984237
:104E680028BF1846208038BDD97921B19878042800
:104E7800B8BF04209870204890F857000A280CD032
:104E88000C28CED1DFED227A002ACDD0072ACBD04C
:104E98000A282CD1DFED1F7AC6E70A20DFED1E7A3B
:104EA800C1E79B78154A07EE103A1178B8EEC77A31
:104EB80027EE277A07EE901AF8EEE77A67EE877AF8
:104EC800B4EEE70AF1EE10FA10DDC0EE077AFDEE57
:104ED800E77A17EE903A102BA8BF1023012BB8BF22
:104EE8000123DBB28B4238BF0B46137038BDDFEDB0
:104EF8000B7A99E7544E0020047E00202878002081
:104F08006F120339244B00206F120338B4280308AA
:104F18000AD7A3390F506E3A5304E9386F12833A0F
:104F280038B50C4C0C4DAC4206D26168204614349E
:104F3800FDF7EAFDAC42F8D3084A094B094C146066
:104F4800002209491A705A7008480860BDE83840BC
:104F580017F0F2BF70890308D08D03087041002054
:104F68007441002004810020FC3800200C820020BD
:104F780008B5FFF7D5FF13F0D1FDFDF739FEBDE801
:104F8800084013F0B3BD00BFF0B50C292BD8DFE8FB
:104F980001F06F2A2A2A4C2A2A2A2B2A2A2A0700B1
:104FA800046AB2F80CE097881668674D24F48054B8
:104FB8000462036A4468C16923F4005343EA0E3368
:104FC80021F4E641A84243EA073341EA062100F00A
:104FD800B58005F50065A84200F0B080926844608D
:104FE800C16102640362F0BD046A96899588D2F8AB
:104FF80000E0554F24F480740462036A4468C16970
:1050080023F4007343EA062321F07301B84243EA0C
:10501800052341EA0E017ED04C4DA8427BD0926810
:105028004460C161C2630362F0BD046A96899588D1
:10503800D2F800E0444F24F010040462036A446884
:10504800816923F0200321F0807143EA061321F4DB
:10505800E641B84243EA051341EA0E2148D03B4DE8
:10506800A84245D092684460816182630362F0BDC2
:10507800046A9389B2F804E01768334E24F00104F7
:105088000462056A4468816943EA0E0321F48031A9
:1050980025F002059BB221F07301B04243EA0503F3
:1050A80041EA070114D0294DA84211D005F5406501
:1050B800A8420DD005F58065A84209D005F58065A0
:1050C800A84205D092684460816142630362F0BDE2
:1050D800D689158A578A23F0080333433D43D68877
:1050E80024F4407423F00403ADB233432C43E9E7BE
:1050F800D589178AD68823F0800343EA051324F458
:105108004064558A23F0400344EA870443EA0613BF
:1051180044EA8504A6E7D589178AD68823F400636C
:1051280043EA052324F44054558A23F4806344EA6F
:10513800071443EA062344EA051470E7158A24F4A1
:10514800804444EA851449E7002C014000340140BA
:105158002DE9F04FF022002183B07948794CDFF82F
:105168000892794D794E7A4FDFF800822DF09DFA3A
:1051780078487949DFF8F8E1DFF8F8C100221359D7
:10518800834200F0C280B3F1804F00F0CA80AB4286
:1051980000F0C980B34200F0C880BB4200F0C7806D
:1051A800734500F0C680634500F0C580434500F0B4
:1051B800C480DFF8C4A153457AD00AF5806A534504
:1051C80008BF092375D014328C2AD8D15D4C634DA1
:1051D800634E614F04F18C0802E01434A04564D09A
:1051E800A379002BF9D023794FEA131909F1FF3974
:1051F800B9F1050F03F00F03EFD835F8190040FA9D
:1052080003F2D207E9D54FF0010A0AFA03F3013B8A
:1052180018402AF0D7FD16F809305249184411EB06
:10522800C002DAD051F83000DFF850E1217A00F1FD
:1052380038439B0A1EF8033003F01F0E5B09022B4C
:105248000AFA0EFA63D0032B66D0012B58D0938844
:105258000093B3FA83F3C3F11F039BB2DA0800EBA0
:10526800820203F00703D2F820E09B004FF00F0CF6
:105278000CFA03FC2EEA0C0EC2F820E0D2F820E06B
:1052880001FA03F343EA0E0313626946002302227C
:1052980014348DF804208DF805308DF806308DF81B
:1052A80007301CF00BFFA0459AD103B0BDE8F08F82
:1052B800082309EBC3034FF0010B93F85CA00AF035
:1052C8001F034FEA5A1ABAF1020F0BFA03F311D06F
:1052D800BAF1030F08D0DA457FF475AFD1F814A0FE
:1052E80043EA0A034B616EE7D1F81CA043EA0A03BC
:1052F800CB6168E7D1F818A043EA0A038B6162E73B
:105308007B694AEA03037B61A1E70023D1E7BB6914
:105318004AEA0303BB619AE7FB694AEA0303FB61B4
:1053280095E70123C5E70223C3E70323C1E7042365
:10533800BFE70523BDE70623BBE70723B9E700BF9F
:1053480030710020184F0308000400400008004096
:1053580000100040002C014000100240FC430308EC
:10536800084403082C490020B428030800400140E1
:10537800001400400034014000440140104F03086D
:1053880001490248FEF7CCBCF871002000480140F2
:1053980001490248FEF7C4BCD07100200034014026
:1053A80001490248FEF7BCBCD0710020003401401E
:1053B80001490248FEF7B4BCA8710020000800406B
:1053C80001490248FEF7ACBC80710020000400408F
:1053D80002494FF08040FEF7A3BC00BF587100207F
:1053E80001490248FEF79CBC30710020002C0140A6
:1053F80001490248FEF794BC30710020002C01409E
:105408002DE9F04104684E4DA30AAB427AD00AD97F
:105418004C4DAB425FD00535AB4277D0073DAB4230
:105428005DD0BDE8F081B3F5801F67D0013DAB4288
:1054380059D14FF0700E022647794FEA970C002990
:1054480068D0B000634685190227D4F80C809F40C5
:105458000CEB4503BFB23C4D03F1040C47EA0807C7
:1054680045F8231045F82C20E760EFF3118150220E
:1054780082F31288821905EBC2021369002B34D01B
:1054880013620433821905EBC202576917B11F6012
:1054980053690433821905EBC202976917B11F607B
:1054A80093690433821905EBC202D76917B11F60EB
:1054B800D36904330027CAB21F6082F311883044CD
:1054C80005EBC000036A9BB9E3684FF6FE72134010
:1054D800E360BDE8F0814FF0C00E0426ACE74FF062
:1054E800200E0026A8E7BDE8F08105EB0E03C9E70A
:1054F800E36843F00103E360BDE8F0814FF0480E34
:10550800012699E74FF0980E032695E74FF0E80E2D
:10551800052691E7BF08022306FA03F0BB40DB43E8
:10552800E768094D9BB23B4087190CEB470CE360D9
:105538000CF1040345F82C1045F8232095E700BF2B
:10554800020010004D0010003071002030B50368D3
:105558005C4D18885C4CB4FBF2F20139013AAB425D
:1055680094B283B089B282B266D05848834263D07D
:10557800B3F1804F60D0A0F5983083425CD000F53D
:105588008060834258D0524883425BD000F58060E7
:1055980083427DD022F4407200F58C3092B283426F
:1055A8001A80D9621C850ED0484A93420BD002F566
:1055B8004062934207D002F58062934203D002F51D
:1055C8008062934201D100221A8601225A611A8808
:1055D8003C4992B242F001028B421A8062D0B3F188
:1055E800804F61D03B4A934260D002F5806293427B
:1055F8005ED002F5006293425CD002F5806293426D
:105608005AD002F59032934258D002F54062934244
:1056180056D002F5806293421ED002F58062934212
:1056280008BF092219D002A84FF0012340F8043D11
:105638001CF070FA03B030BD254822F07002834296
:1056480092B2A3D101201A80D9621C8558611A88A8
:1056580092B202431A80C5E708221F4B03EBC2032C
:1056680001A893F85D408DF80440012300228DF8CD
:1056780005308DF807308DF806201CF04BFA1B2CEE
:10568800D8D1164B019301A81CF044FA03B030BDE1
:1056980001201A80D9621C8558611A8892B2024387
:1056A8001A809CE70022D8E70122D6E70222D4E735
:1056B8000322D2E70422D0E70522CEE70622CCE770
:1056C8000722CAE7002C014000A24A040034014026
:1056D8000010004000040040B4280308190100012C
:1056E800204B98422DD0B0F1804F2CD0A3F59433A5
:1056F80098422AD003F58063984228D003F50063C6
:10570800984226D003F58063984224D003F590335D
:10571800984222D003F54063984220D003F5806375
:10572800984207D003F58063984208BF092202D047
:105738000020704708220C4B03EBC20393F85C006F
:1057480070470022F7E70122F5E70222F3E7032278
:10575800F1E70422EFE70522EDE70622EBE707224F
:10576800E9E700BF002C0140B42803082DE9F04FF9
:10577800013085B0C3B203938E4D8F4F8F4C904E3E
:105788000A230293DFF8409221F03CF84FF4FA7AAA
:105798004FF0100C4FF47A70D9F80430C3F30803B3
:1057A800002B40F0C880EFF31183002B40F0C3803A
:1057B8002968A26800BF2B689942F9D1D7F800E0A0
:1057C80000FB0EF39B1AB3FBFEF300FB01314FF015
:1057D800010E0191D9F80430C3F30803002B40F0FF
:1057E8008E80EFF31183002B40F089802B68A1682D
:1057F80000BF2A689342F9D1D7F800B000FB0BF23A
:10580800521AB2FBFBF200FB0323019A9B1AB3F571
:105818007A7FDFD3BAF1010ABED1039B002B40F097
:10582800C4804FF47A7ADFF8A09150464FF0100CFC
:10583800D9F80430C3F30803002B40F09980EFF344
:105848001183002B40F094802968A26800BF2B6860
:105858009942F9D1D7F800E000FB0EF39B1AB3FB8D
:10586800FEF300FB01314FF0010E0191D9F804302D
:10587800C3F308033BBBEFF3118323BB2B68A16879
:1058880000BF2A689342F9D1D7F800B000FB0BF2A9
:10589800521AB2FBFBF200FB0323019A9B1AB3F5E1
:1058A8007A7FE3D3BAF1010AC2D1029B013B02938A
:1058B8007FF468AF4349444B4448454A0860DA607E
:1058C80005B0BDE8F08FEFF311888CF31288A1685A
:1058D8002368DB0344BFC6F800E0A1682B68326880
:1058E8005FFA88F888F31188D7F800801A4400FB1B
:1058F80008F35B1AB3FBF8F300FB0233CDE7EFF3D1
:1059080011888CF31288A1682368DB0344BFC6F8AA
:1059180000E0A1682B6832685FFA88F888F311887C
:10592800D7F800801A4400FB08F35B1AB3FBF8F3BE
:1059380000FB023369E7EFF311828CF31288D4F885
:1059480008E02368D90303D501233360D4F808E0BD
:105958002B683168D2B282F311883A68194400FB87
:1059680002F3A3EB0E03B3FBF2F300FB01312EE7C6
:10597800EFF311828CF31288D4F808E02368D90376
:1059880003D501233360D4F808E02B683168D2B21C
:1059980082F311883A68194400FB02F3A3EB0E0363
:1059A800B3FBF2F300FB01315DE7184620F0AAFDD6
:1059B80037E700BF287100202C71002010E000E0BC
:1059C80024710020FC9F002000ED00E0EFBEADDE5A
:1059D8000400FA052DE9F047B14FB24E13F09EF8D6
:1059E800BE421ED2DFF84483DFF84493444625883C
:1059F80062197DB14A450DD2052D0BD933886188CE
:105A0800C3F30B03994200F0FA8014462588621903
:105A1800002DEFD1716830461436FDF775F8BE4297
:105A2800E4D3A14A1378A3F1170102290FD99F499A
:105A380011F83300002840F00481D8000144497867
:105A480029B19B4911F83330002B00F02281994C81
:105A58006378022B84BF002363702378022B84BFF2
:105A680000232370944B9A78042A00F0098132B9F4
:105A78001A88B2F5F07F84BF4FF4F0721A808F4D08
:105A88008F4A2B681A40002A00F00681D80700F1D7
:105A9800F280590400F1EA801A0700F1E2809B04C1
:105AA80000F1D880874D2B685A8C998C914224BF7D
:105AB80000225A84FFF796F91EF05CF910B9824863
:105AC80021F080FC8020FDF755F84FF40070FDF7B9
:105AD80051F84FF40030FDF74DF84FF40010FDF782
:105AE80049F84FF00070FDF745F84FF08060FDF77A
:105AF80041F84FF00060FDF73DF86378022B06D8B7
:105B0800724A734903EB430302EB83030B60237868
:105B1800022B07D803EB83016E4AC3EBC10302EBE8
:105B280043032B6016F088FA002130226A482CF0D3
:105B3800BCFD286826F0FAFF684B2E6803F1500177
:105B480002E0043399427AD01A78002AF9D19C7875
:105B5800D8788442F5D26249624B91F804E06248F1
:105B6800624D5C6B624B2860C827642111FB0E7183
:105B7800DFF8C0E159605F4F30F8061C5E4DAEF8A3
:105B8800001000219960D960196159619961D96142
:105B980083F8201083F821103A702E600CB114F0AD
:105BA80043FE564B9FED565A1B88564A9FED566A40
:105BB8005579564C56495748086006EE903AF8EE23
:105BC800E66A1388C5EE265A07EE103A538812790A
:105BD800C4ED005A07EE903AB8EEC77A4E4BF8EE8D
:105BE800E77A1D725A7227EE067A67EE867ABDE862
:105BF800F04783ED017AC3ED007A12F077BF63793D
:105C08009B077FF402AF716894F804A03046FCF754
:105C18007BFF3388BAEB133F04D01436BE42FFF43F
:105C2800E5AEFEE673887068AA1FC3F30B039A42B9
:105C380004F10601A8BF1A462AF020FAEDE701226E
:105C480089E7D8000C186468002C7FF4F7AE172495
:105C58001470F3E63148FCF78DFF4020FCF78AFF0B
:105C680020E72F48FCF786FF2B6818E72D48FCF73C
:105C780081FF2B6810E72C48FCF77CFF2B6808E7AE
:105C88009A8AB2F57A7FBFF4FAAE4FF47A729A82A2
:105C9800F5E618231370DAE643F001032B60F5E606
:105CA800D08D030870890308A834002048440308ED
:105CB800A04D030874410020244B00204882002096
:105CC8000960000270410020284800200C82002052
:105CD800FC3800200481002080210020AC34002002
:105CE800F42C0020D47700203A780020DC780020BB
:105CF800843F002005020020B4210020D41F00208A
:105D0800C0C9FB48E41B002017B7D138D81F0020B2
:105D1800D42A00203661023DB02A00200940000242
:105D280001600002092000020860000202F0030876
:105D3800000004083838002008B512F0EFFEFCF720
:105D480057FF12F0D3FEFFF745FE0120BDE80840DB
:105D580022F0E4B92DE9F04F2DED028B93B0834684
:105D68001BF07CFAB54B1D7825B113B0BDEC028B46
:105D7800BDE8F08FB24B1B685C05F6D5B14FB24E4B
:105D88003B68002B56D0B14C3168D4F810218A1AE0
:105D98007C2A4FD994F81421DFF8FC829FEDAC8A55
:105DA800C4F81011013284F814214FF0240A5E203F
:105DB800984750463B689847A64BF8EC016A9B8A7F
:105DC80007EE103AF8EEE66AB8EEC77A0AF1010A69
:105DD800C6EE877A5FFA8AFA67EE887AFDEEE77A86
:105DE800CDED027ABDF908905FFA89F01CF060FDEC
:105DF800C9F307201CF05CFDBAF1270F3B68D6D128
:105E08005E2098473B683020984700201CF050FDE2
:105E180000201CF04DFD3B685E20984794F8143133
:105E280013F0030800F08481580701F03682282B0C
:105E380001F03283884B1B78002B72D0834C874A41
:105E4800D4F81831ABEB0303934200F27B8794F844
:105E58002091B9F1000F35D1DFF84082D8F8000061
:105E6800FBF792F9C0B201280FD902287C4F41F004
:105E7800A5833B78002B41F02A86D4F82431ABEB7C
:105E88000303B3F57A6F81F09D87D4F82831002B8E
:105E980047D094F82031C3B9724B1B689B78012115
:105EA8001E3B00228B4284F8201184F8342141F2F1
:105EB8002E87D8F80000022104301CF06FFC94F8FB
:105EC8002C3111E0D4F828315BB3D4F8303140F6E6
:105ED800B732ABEB0303934223D994F82C31002B50
:105EE80001F0C382DFF8B481013BDBB284F82C31C6
:105EF800002B00F08287D4F8287194F8342117F821
:105F0800011B94F83531D8F80000C4F828710A4408
:105F1800013384F8342184F83531FBF739F9C4F8B2
:105F280030B1514BD6F800801B7843B14F4F3868D9
:105F380028B14F4B1B78013B012B40F26E874D4B2C
:105F48001B7863B14C4F3B684BB1404CD6F800907E
:105F5800D4F84C31A9EB0303632B00F21C81DFF862
:105F6800408198F80030022B01F05E823C4F97F890
:105F78007430032B00F02B87404B1B7873B1404DD6
:105F88002B685BB1314CFAF7ABFED4F8583102906C
:105F980044F61F62C31A934200F25881394B1B78AA
:105FA800002B7FD1384B1B7843B1284CD4F8A8324A
:105FB80003F5C333A0339B4580F07286334B1B78BF
:105FC800002B3FF4D2AE214E314C324D06F2C92798
:105FD8002068FBF7D9F800283FF4C7AE2068FBF724
:105FE800CBF82B7880465A1E33B120682A70FBF70D
:105FF800CBF80028F2D1B8E603223946781E2CF0F7
:106008003AFB96F8C83296F8C92286F8CB8283F410
:106018007F4383F0FF039B1A1FFA88F89BB2B8EB03
:10602800132FD5D196F8CA22DBB29A42D0D1781E66
:106038001CF032F92B7818442870C9E72C3B002053
:10604800784E0020E847002028710020F41B00202B
:1060580000007A44D4770020364400203F0D030026
:1060680018000020E447002038440020884500201C
:106078004044002048440020186C00205044002070
:106088005444002094440020A54400205A44002091
:1060980060440020644400200C780020E047002081
:1060A800F23100205B4C2278A2B15B4B9B7A53B152
:1060B800FAF716FE594B1B68C31AA3F57A73B3F5A2
:1060C800FA6F07D82278564B56491868FBF72CF810
:1060D80000232370544CD4F8A03203F5C333A03303
:1060E8009B45FFF45FAF514DC4F8A0B22B78002B4D
:1060F80041F030834E4D2B78002B41F01D824D49E5
:1061080094F8A4228D5CE90701F1E784AA0701F15C
:10611800A1846B0701F19983474A94F8A432117856
:10612800013393FBF1F201FB123384F8A43239E70F
:10613800D4F8102141F288339A4201F216823B6862
:106148005E2098473B68142098473C4B3C4AB3F97B
:10615800043082FB03124FEAE378C8EBA2080FFA77
:1061680088F85FFA88F01CF0A3FBC8F307201CF03E
:106178009FFB3B685E2098473B681C20984700209F
:106188001CF096FB00201CF093FB3B685E209847B0
:1061980094F8143148E6DFF8A4A0DFF8A480412081
:1061A8001CF0ACFABAF9023088FB0320DB17C3EB0A
:1061B800A00080B21CF088FABAF9003088FB0320EE
:1061C800DB17C3EBA00080B21CF07EFABAF90430EA
:1061D80088FB0320DB17C3EBA00080B21CF074FA25
:1061E800184B38681978FAF7D3FF94F8503113F040
:1061F800010801F0F481144AC4F84C910133DBB270
:10620800A2FB0312D20802EB8202A3EB420384F83A
:106218005031A4E6284400200C50002060310020B2
:1062280098440020E8430020F41B00209C440020F0
:106238009D440020A0440020A44400205041002098
:106248006766666668700020CDCCCCCC94F85E3169
:10625800002B41F06C81DB4B1A6802F00803002B1D
:1062680048F603414AF60B404BF60F4349F60747F9
:1062780004BF03460F4612F0040F4FF0190118BF70
:106288001F46920684F85E1103D547F4804747F00D
:106298002007CD4B5A79C7F30909002A41F0BF8579
:1062A8009B79002B41F0AA86984664204FF0FF3A6C
:1062B8004FF0000C0A970B97ADF834C0CDF83AC0F0
:1062C800CDF83EC0CDF842C0CDF83090ADF836805C
:1062D800ADF838A08DF846000AAF0FCFDFF800E31D
:1062E80084F805C0AEE80F0097E80F00AEE8070095
:1062F8002EF8023B71464FF0010C1B0CFE271F20A5
:10630800C82201F81E39A770A27184F807C0E0708E
:1063180094F86E01207180F0F10383EA0313DAB276
:10632800130983F0E70343EA022383EAC2031BB29B
:1063380083EA0312D2B2C3F3072383EA121343EAB0
:10634800022383EAC2031BB283F0C80282EA021264
:10635800D2B2C3F3072383EA121343EA022383EA80
:10636800C2031BB283EA0C0787EA0717FFB2C3F31D
:10637800072282EA171242EA072200EB0C0382EA9C
:10638800C7070EEB0C0084F86E31278011F8013B2B
:106398007B4083EA0313DBB21A0982EA172242EA36
:1063A800032282EAC3031BB29FB281422780EDD148
:1063B80083F07C0383EA0313DBB24FEA131E8EEAF1
:1063C800172E8EEA032E8EEAC30E0FFA8EFE1FFAE0
:1063D8008EFADFF810C2A4F800A05FFA8EFE4FEA2A
:1063E8001A2A84F828A084F827E00CF5CB7804F161
:1063F8002209DCF80000DCF80410DCF80820DCF8DE
:106408000C3047460FC70CF1100CCC45B846F0D1FC
:10641800DCF8000038606D4F9CF8043088F80430D0
:1064280007F1270884F8BDE184F8BEA117F8011F19
:106438002868FAF7ADFEB845F8D194F85F31002B1B
:1064480041F070806249326809780A2084F85F0157
:10645800002901F0F0815F4F01293888069041F248
:10646800C1850229B7F802E001F0F484B8880590E4
:10647800032901F0CE85F8880490042901F0DC8511
:106488000529388901F0D3850629B7F80A9001F063
:10649800CA850729B7F80C8001F0C285FB890393E8
:1064A80094F86E110A920B4683F0300282EA0212C7
:1064B800D2B217094849079387F07A0747EA0227B3
:1064C8000988237187EAC202444FC1EB012187FB87
:1064D800013A069B4FF0000C63F30F0C059B6EF31B
:1064E8001F4C4FF0000E63F30F0E049BCDF82CC029
:1064F80012B28A440027C91763F31F4EC1EB6A2AF8
:10650800039BCDF830E082EA021160F30F07002008
:10651800C9B268F30F00C2F3072269F31F4782EA82
:10652800111263F31F404FF000090D978DF83DA03D
:106538000E908DF83C9042EA01220DF1280C82EA77
:10654800C107BCE80F003FB287F0C80888EA0818FE
:10655800DFF88CE084F805905FFA88F8C7F307271E
:10656800AEE80F0087EA181747EA08239CE80300FB
:1065780083EAC8031BB283F023024EF8040B82EAB5
:106588000212D2B2C3F30723079F83EA121370469D
:1065980043EA022383EAC20207F1010C20F8141926
:1065A8004FF023081621FE27C82384F86EC12280E5
:1065B80084F807800EF1020EA770E170A3711146EE
:1065C80012E000BFA0430020304300208B1D0020B4
:1065D80054300020684300206043002003082080D6
:1065E800FC1B0020F61B002010F8013B4B4083EAFF
:1065F8000313DBB21A0982EA112242EA032282EA71
:10660800C3031BB299B270452180EDD183F0F40326
:1066180083EA0313DBB24FEA131E8EEA112E8EEAC9
:10662800032E8EEAC30E0FFA8EFE1FFA8EF8E64F7F
:10663800A4F800804FEA182C5FFA8EFE84F81EE05A
:1066480084F81FC07968BA683868FB6807F5CB78A2
:10665800A8E80F0038697969BA6904F29717A8E8B9
:10666800070004F2B51884F8B5C184F8B4E117F846
:10667800011F2868FAF78CFDB845F8D194F866C16F
:10668800BCF1000F40F04887D04B94F86E71B3F915
:106698000010B3F90220B3F904309FEDCD6ADFF89A
:1066A80040E384F805C007EE103A33680A9387F090
:1066B8006A0383EA031306EE901AD9B20B0983F032
:1066C800D50343EA012383EAC1031BB283EA03111A
:1066D8005242C9B207EE902AC3F3072383EA111383
:1066E80043EA0123F8EEE77AF8EEE66AB8EEC77AED
:1066F80083EAC1031BB267EE867A66EE866A27EEE6
:10670800067A002083F0C808CDED0C7ACDED0B6A2F
:106718008DED0D7A0E900F90109088EA08160DF105
:106728002809F6B2C3F30728B9E80F0088EA161853
:1067380048EA062888EAC6080FFA88F8AEE80F0083
:1067480088F01E0699E8070086EA0616F6B2C8F32E
:10675800072383EA161343EA06238EE8070083EA31
:10676800C6061C20C8214FF005084FF01E0CFE235A
:106778007A1CE070A17184F8668184F807C0A37060
:10678800AEF1100127710EF10C00268084F86E21FD
:1067980011F8013B734083EA0313DBB21A0982EA5A
:1067A800162242EA032282EAC3031BB29EB2814246
:1067B8002680EDD183F0270383EA0313DBB24FEA87
:1067C800131E8EEA162E8EEA032E8EEAC30E0FFAD9
:1067D8008EFE1FFA8EFC7C4FA4F800C05FFA8EFE76
:1067E8004FEA1C2C84F825C084F824E007F5CB7800
:1067F80004F1220938687968BA68FB6846460FC60A
:1068080010374F45B046F5D1724E3B88A8F8003096
:1068180006F1240784F8BAE184F8BBC116F8011F11
:106828002868FAF7B5FCB742F8D194F867A1BAF12D
:10683800000F40F06B8694F86E81644B664AB3F99A
:106848000410B2F90620654EDFF898E1644F84F829
:1068580005A088F0220080EA0010C0B2030983F086
:10686800590343EA002383EAC0031BB2B2F5FA6F67
:1068780083EA0310C0B2A8BF4FF4FA62C3F3072338
:10688800B2F57A7F83EA101343EA0023B8BF4FF4C6
:106898007A7283EAC000A2F57A72642303FB02F2DB
:1068A8008EFB023ED31786FB0162C9174FF0000C1E
:1068B800C3EBAE13C1EBA201CDF828C006B2CDF8E8
:1068C8002CC0CDF830C0CDF834C0ADF83A30ADF8B2
:1068D80038100DF1280CBCE80F0086F0C80E8EEABF
:1068E8000E1E5FFA8EFEC6F3072686EA1E1646EAD5
:1068F8000E260FC786EACE0636B286F04A0383EA2A
:106908000313DBB2C6F3072181EA13113A46DCF818
:1069180000E042F810E941EA032108F1010681EAA2
:10692800C30305204A214FF0FE0C84F86E614FF036
:10693800C80E142684F8670184F80480238004377D
:10694800E17184F802C0E67084F806E0184612F88F
:10695800011B414081EA0111C9B20B0983EA1023E6
:1069680043EA012383EAC10109B288B2BA4220800E
:10697800EDD181F0140181EA0111C9B24FEA111E6B
:106988008EEA102E8EEA012E8EEAC10E0FFA8EFEC6
:106998001FFA8EF60C4F26804FEA16295FFA8EFEF4
:1069A80084F81D9084F81CE079683868BA68FB6838
:1069B800B7F8188007F5CB7CACE80F00386979691F
:1069C800ACE8030010E000BFF61B00205041002097
:1069D80088C3E43A8B1D002068430020676666661A
:1069E800FC1B0020D34D621004F29716ACF800800F
:1069F80084F8B391B04684F8B2E104F2B31918F8F8
:106A0800011F2868FAF7C4FBC145F8D1C44BC54A31
:106A18001B781278013B12F00100DBB214BFC021D1
:106A28004021172B03D8C04A134493F830A0BF4B1A
:106A38001A8893071ABF002341F01001012312F4AA
:106A4800027F18BF022312F0100F18BF062312F09E
:106A5800200F18BF1023002841F08C814FF0030C41
:106A680094F86E910A9389F0460383EA0313DAB225
:106A7800130983F0920343EA022383EAC2031BB299
:106A880083EA0310C0B2C3F3072282EA101242EA73
:106A9800002282EAC00212B282F0C80E8EEA0E1EEE
:106AA8005FFA8EFEC2F30722002382EA1E12032039
:106AB8008DF82CA08DF82FC08DF82D3042EA0E2CC1
:106AC8008DF82E108DF830000AAA07CA8CEACE0E6F
:106AD8000FFA8EFEDFF868A2E3718EEA0E1CAAE8B0
:106AE80003005FFA8CFCCEF3072E8EEA1C1E4EEADA
:106AF8000C2181EACC0C94F808E08AF800200FFAFF
:106B08008CFC8EEA0C0E8EEA0E1E5FFA8EFECCF31B
:106B1800072282EA1E1242EA0E22607AA17A94F8CB
:106B28000BC0637182EACE0212B2504080EA001EA6
:106B38005FFA8EFEC2F3072080EA1E1040EA0E209C
:106B480080EACE0000B2414081EA0111C9B2C0F327
:106B5800072282EA111242EA012282EAC10212B233
:106B68008CEA020C8CEA0C1C5FFA8CFCC2F307223C
:106B780082EA1C1242EA0C2294F80CE0607BA17BAA
:106B880094F8108084F8049082EACC0212B28EEA5B
:106B9800020E8EEA0E1E5FFA8EFEC2F3072282EA0A
:106BA8001E1242EA0E2282EACE0212B2504080EA57
:106BB8000010C0B2C2F3072282EA101242EA002291
:106BC80082EAC00212B2514081EA0111C9B2C2F38D
:106BD800072282EA111242EA012282EAC102E17B1B
:106BE80013B281EA030282EA0212D2B2C3F3072384
:106BF80083EA121343EA022383EAC2031BB288EA38
:106C0800030282EA0212D2B2C3F3072383EA121301
:106C180043EA022383EAC2031BB283F0320282EA08
:106C28000212D2B2C3F3072383EA121343EA022300
:106C380083EAC2031BB29AB24FF0FE0C4FF0090E62
:106C4800C82009F10101DBB284F802C084F803E02E
:106C58004FEA122CA07184F86E11228084F812C0B9
:106C6800637438687968BA68B7F80C900AF5C47E16
:106C7800AEE807000AF5CC7A8EF80280AEF80090EC
:106C880084F8A8C184F8A73116F8011F2868FAF714
:106C98007FFAB245F8D1029BC4F85831FFF77EB9A4
:106CA80094F8AC32204AC4F8A8B202EB8302926C82
:106CB80042B312AD04F2B3231D4E45F8203D002126
:106CC80004F2C52331800B9380211523A52784F86E
:106CD800B232284684F8B11284F8B0729047284638
:106CE8003188FCF7CFF90A9D124804F52C716D1A0A
:106CF800152DA8BF15252A4629F0C0F90E4A94F883
:106D0800AC3215700D4A013382FB0312A2EBE37219
:106D180002EB42029B1A84F8AC32FFF74FB900BF6E
:106D2800A83400209C4500205C2903084C41002021
:106D3800A64300203C2F0020512F002056555555C2
:106D4800FC1B0020D34AD44B92F80BE03168D4F8EE
:106D58001C211B88D148891A4FF47A72DFB202FBD2
:106D68000EF21B0A8777077591424FF00007C37729
:106D780043758770077180F01284C94BC9491A6836
:106D88009B68C4F818B181FB02E7D21781FB03E1C5
:106D9800C2EBA702DB17C3EBA10311124FEA232CA6
:106DA8004FF0F40E02770127417780F82030302128
:106DB8007522782380F821C080F81AE0C77680F819
:106DC800221080F8232080F82430FFF740B8DFF83D
:106DD800F492D9F80000FAF7CBF900283FF4CCA8D0
:106DE800D9F800000121FAF7BFF90222002387F839
:106DF800742088F80030FFF7BFB894F8341194F87D
:106E08003531D8F800004A1C013384F8342184F85D
:106E18003531FAF7BDF9FFF782B8A34CDFF8A8922D
:106E28004FF0000A0AE01B2B00F014830D2B00F032
:106E380012824FF0010389F801303868FAF7A4F993
:106E4800002838D03868FAF797F983B27E2B326871
:106E58002AD099F801100029EFD194F83621002A98
:106E6800E1D07D2B00F00C8294F844E1BEF1000FD4
:106E780004D080F02003DBB284F84411511CC9B25D
:106E88002244092984F8361182F8383100F0EC815F
:106E98000829D2D8B4F84221134403EB132303F092
:106EA800FF03A4F84231C8E784F836A184F837A173
:106EB80089F801A0C1E794F8453133B194F8393124
:106EC80084F84501302B00F0498794F83721774B37
:106ED800DFF8F8C1DFF8F8E1DFF8F8A1012710467C
:106EE80000283FF42CA83268A2EB0802012A00F21D
:106EF800AD8194F84691B9F1000F40F0C28294F840
:106F0800471133F8112012B984F84771E8E70131C5
:106F1800B2F5826F84F8471100F002811FD9B2F5EB
:106F2800E26F00F09A8034D9B2F5046F00F0A480C3
:106F3800B2F5116F00F04781B2F5E46FD0D1104679
:106F48005B4A176C918A642303FB07F393FBF1F107
:106F58001BF00AFC002384F83731FEF7F0BFB2F5C6
:106F6800007F00F0B9802CD8B2F5807F00F0458111
:106F7800B2F5887FB4D1DCF800205207B0D50021E3
:106F88004FF488701BF0F0FB002384F83731FEF7CC
:106F9800D6BFB2F5C06F00F0B380B2F5E06F9FD1F5
:106FA800434A906B918A642303FB00F34FF4E0603B
:106FB80093FBF1F11BF0D8FB002384F83731FEF77F
:106FC800BEBFB2F5047F00F02781B2F5806F87D18C
:106FD80094F848310133DBB2032B00F2588142F2B6
:106FE800107184F8483101FB03F1324B1B88002BE8
:106FF80040F04B810131304B1B78DF072F4B1B884A
:1070080048BF0431D80748BF0A319A0748BF14312E
:107018001F0648BF2831D80548BF28315A0748BF3E
:1070280064311F0748BFC831980548BF01F5C871CA
:107038009A0648BF01F57A71DF0648BF01F5FA6183
:10704800580648BF01F57A614FF480601BF08CFB4D
:10705800002384F83731FEF772BF1046144AD76B05
:10706800918A642303FB07F393FBF1F11BF07CFB8C
:1070780084F83791FEF763BF114BB3F9041001EBA5
:107088008101104649001BF06FFB84F83791FEF729
:1070980056BF00BF144600200C460020684400205C
:1070A8009045002067666666F41B00205C2903088B
:1070B800D4770020A44300209C4500204C410020A8
:1070C800504100205432002018000020A043002026
:1070D80030430020224600209EF8061000293FF485
:1070E800FFAEC44BC4491B68104681FB0321DB1764
:1070F800C3EBA1011BF038FB84F83791FEF71FBFE3
:107108009EF80620002A3FF4EBAEBA4B4FF4C0605D
:1071180099681BF029FB002384F83731FEF70FBF6D
:10712800DCF8002012F020097FF4DAAEB34A1168C7
:10713800090600F1F585B24A127B002A3FF4D0AE69
:1071480094F84911032900F29486DFE801F0322807
:107158001902AC4B1B6859799A79DB7901F14071B6
:1071680001EB022101EB0341002384F849314FF47C
:1071780082601BF0F9FA002384F83731FEF7DFBE8E
:10718800A14B1A68137A507992781B0403EB0023F9
:1071980013444A1C84F8492103EB0161E7E79A4B41
:1071A8001A68D379107952781B0403EB002313442F
:1071B800EFE7954B1A689379D07812781B0403EBA4
:1071C80000231344E5E79EF80520002A3FF488AE23
:1071D8009AF8001000293FF483AE8C4B1B8803EB10
:1071E80083035B004FF4116093FBF1F11BF0BCFAD1
:1071F800002384F83731FEF7A2BEDCF800205107DF
:107208007FF56EAE00214FF480701BF0ADFA0023BD
:1072180084F83731FEF793BE9EF80520002A3FF424
:107228005FAE9AF8001000293FF45AAE744B5B7BAE
:10723800002B00F09B85754B1B8893FBF1F101EB4C
:10724800810149004FF404701BF08EFA002384F882
:107258003731FEF774BE4FF0010184F8361184F817
:107268003831A4F84221E8E5B4F84221C2F1FF021E
:1072780093427FF4DEAD4FF0010384F84531D8E541
:107288004FF0010384F84431D7E50231B3E6012316
:1072980084F8483142F21071A7E63B685E209847AF
:1072A8003B68022098475A4B534AB3F9503082FB47
:1072B80003124FEAE378C8EBA2080FFA88F85FFADE
:1072C80088F01BF0F5FAC8F307201BF0F1FA3B68C9
:1072D8005E2098473B68032098474E4B1B78D90798
:1072E80040F1318114F05CFE4B4B9FED4C7AD3EDAD
:1072F800037A67EE877AFCEEE77ACDED027ABDF87D
:107308000830002800F02285D8B24FEA13281BF075
:10731800CFFA40461BF0CCFADFF8088198F8053020
:10732800002B40F0C4820AA93D481BF085FA3B684F
:107338005E2098473B6813209847BDF928805FFA7C
:1073480088F01BF0B5FAC8F307201BF0B1FA3B68C8
:107358005E2098473B681B209847BDF92A805FFA52
:1073680088F01BF0A5FAC8F307201BF0A1FA3B68C8
:107378005E2098473B68232098474E201BF098FAD8
:1073880000201BF095FA0AA925481BF055FA3B681E
:107398005E2098473B6812209847BDF928805FFA1D
:1073A80088F01BF085FAC8F307201BF081FA3B68C8
:1073B8005E2098473B681A209847BDF92A805FFAF3
:1073C80088F01BF075FAC8F307201BF071FA3B68C8
:1073D8005E2098473B682220984745201BF068FAB2
:1073E80000201BF065FA3B685E20984794F814313A
:1073F800FEF71DBD9045002067666666784E002042
:1074080014460020FC380020704100200C46002063
:10741800047E00209C45002024460020CDCC4C3E14
:107428008096980030430020F9F75AFCB54B1B684A
:10743800C01A40F6B833984200F2C680DFF804A3B9
:107448009AF804303A2B00F09283002388F8003031
:10745800FEF792BD3868F9F797FE00287FF4E9AC8B
:107468004FF0010384F83731E7E4C4F8283184F891
:107478002031DFF8D4821BF0C5F994F82C31FEF7DF
:1074880033BDA14906201AF091FF002384F8460174
:1074980084F83731FEF753BD4FF000093B6884F894
:1074A80014915E203468DFF8A48298473B6817205F
:1074B800984748461BF0FCF9944BA3FB04239B0B0D
:1074C800A8FB03125209C2EB0212A3EB8203D8B243
:1074D8001BF0EEF93B685E2098473B6818209847F8
:1074E8008B4BA3FB04239B09A8FB03125209C2EB95
:1074F8000212A3EB8203D8B21BF0DAF948461BF05C
:10750800D7F93B685E209847FEF794BC0AF1FF3A2A
:1075180084F867A1FFF7BFBB0CF1FF3C84F866C194
:10752800FFF783B9013B84F85F31FFF7A7B8013B48
:1075380084F85E31FEF781BF76493A201AF036FFAB
:107548002870FEF72FBDDFF80882734BB8F8089053
:10755800A3FB09394FEA99095FFA89F01BF0A8F9EA
:107568004FEA19201BF0A4F9D8E63B685E2098473B
:107578003B681020984740461BF09AF940461BF09C
:1075880097F93B685E2098473B682120984740461A
:107598001BF08EF940461BF08BF9FEF7D0BD5F4B10
:1075A80032681B78C4F81C21013B012B3FF6E5AB80
:1075B8001022022382700371FFF7DFBB1BF012F960
:1075C80001233B70FEF761BC554AB2F852310021E5
:1075D8000133A2F8523188F80010FEF7CDBC514BA8
:1075E8001B88DA0515D4D80600F13084990600F115
:1075F8003C845A0600F14884180700F15284D907E0
:1076080000F1EC8413F0020F0CBF4FF004084FF0A8
:107618000C08454B454A1B78D27803F001030AB1A0
:1076280043F00203532002931BF068F8404A128883
:1076380002EB820202EB8202900080B21BF044F857
:1076480000201BF041F83B4A3B4912883868C2EBDE
:10765800C212520081FB023111444FEAE27ACAEBAE
:10766800612A5FFA8AFA5146F9F792FD334B386876
:107678001A78029B48EA0308304B8AEA020A00217A
:1076880083F800A0F9F784FD41463868F9F780FDD2
:107698002A4B2A4A1B78386888EA0303DBB2194662
:1076A8001370F9F775FD94F85031002B7EF4A3ADF3
:1076B8004F201BF023F81DF0A1FC1DF09FFC1DF0CE
:1076C8009DFC01213868F9F763FD1D4A1B4B92F8B0
:1076D80000801B78194A386808F0010883F0010314
:1076E80041461370F9F754FD144B144A1B78386857
:1076F80088EA030319461370F9F74AFD94F85031E4
:10770800FEF779BDF83100206B27020873B2E74510
:10771800D34D6210E5110208CDCCCCCC94430020A7
:10772800F41B00204C4100209C450020843F002091
:107738000C46002060430020030820806870002069
:107748002C430020E0310020E04700208988888809
:1077580030430020AE4EAF4B00930024A6F13F010A
:10776800AD4BAE4A089106F8404CAD4909960AA8B7
:10777800FBF760FD089E731C08933470089B292250
:10778800591C08911A70089BEA22591C08911A7012
:10779800089BC822591C08910AA81A7027F048FEAD
:1077A800471C0AA93A46089828F068FC089AD31991
:1077B80001330893D455089B5A1C08921C70089BE7
:1077C8005A1C08921C70089B5A1C08921C70089B33
:1077D8005A1C08921C70089B5A1C08921C70089B23
:1077E8005A1C08921C70089B5A1C08921C70089B13
:1077F8005A1C08921C70089B5A1C08921C70089B03
:107808005A1C08921C70089B5A1C08921C70089BF2
:10781800FF22591C08911A70089B0122991812A876
:1078280008911A7050F8283D9B1B337019F0A6FC7C
:107838002C70FEF7B7BB8846894608460491059127
:107848008E4606910391FEF72BBE764A704B12685E
:107858000B93A3F1400500202121D70003F8400C29
:10786800A97040F1D08270490326704B1B885805D7
:1078780000F1C682DA0700F1F58203F002036C4AD0
:10788800002B1CBF032611466A4F3246384628F0A3
:10789800F5FBF31912A80133B91E40F8203D002268
:1078A8005B1AF2556B7019F069FCFEF735BC624B38
:1078B80093F800A0BAF1000F3FF435AD5F4AB4F871
:1078C80016E111883B6802924FEA0E1E64201FFAE7
:1078D8008EFE00FB01A14FEA4A00B1FBF0F14EEA2F
:1078E800012E1FFA8EFEC1F303215E204EEA010924
:1078F80098473B68062098475FFA89F01AF0D8FF46
:107908004FEA19201AF0D4FFB4F81631029A4C49FC
:10791800B2F800904A7A01339BB2012A93FBFAF03D
:107928000AFB1033A4F8163100F049836E2345484A
:107938004A7B03FB09F380FB03014FEAE379C9EBB8
:10794800A1092AB13C4B1FFA89F91B7899FBF3F975
:107958003B68DFF8FCA05E2098471FFA89F93B686E
:107968003A209847AAFB093A4FEA5A1A1FFA8AF3AB
:10797800D8B202931AF09CFF029B180A1AF098FFDB
:107988003B685E2098473B683B209847642303FB8D
:107998001A939BB22C48053380FB0320DB17C3EBFB
:1079A800A000C0B21AF084FF00201AF081FF3B68E3
:1079B800DFF898A0DFF890905E2098473B68282071
:1079C8009847DAF8003089FB0329DB17C3EBA909CC
:1079D8005FFA89F01AF06CFFC9F307201AF068FF04
:1079E8003B685E2098473B6804209847B8F8083001
:1079F800002B40F04D82DAF8083083F310085FFA64
:107A080088F01AF055FFC8F307201AF051FF8AE4EE
:107A1800E843002079410020045003080C50030873
:107A28001850030898430020E84F03084C410020F1
:107A380000500308AB430020224600200C460020DB
:107A480014460020310CC3306766666690450020F6
:107A58001F85EB51CC4ACD4B0B9212AEA2F13D00E3
:107A680046F8200D1988CA4FA2F1400300204FF0B4
:107A78000A0E02F8400C082283F801E030469A709A
:107A8800FBF7DAFA3B68C349DA1781FB0313C2EB49
:107A9800A30399B23046FBF7CFFA0BF007FABF6899
:107AA8000A9B3A0C591C0A911A700A9B3A0A591CEB
:107AB8000A911A700A9B5A1C0A921F700A9B5A1C38
:107AC8000A921870304619F059FBFEF722BBC4F829
:107AD80024B187F80090FEF7D8B9AF4F9FEDAF8A71
:107AE800B7F90220A8480B9007EE902AF8EEE77A3B
:107AF80012AE67EE887AA0F13D01FDEEE77A46F80E
:107B0800201D00F8403C0823CDED027A00F83F3CE8
:107B18001E23BDF8081000F83E3C3046FBF78CFAEF
:107B2800B7F9003007EE903AF8EEE77A304667EE9C
:107B3800887AFDEEE77ACDED027ABDF80810FBF7FA
:107B48007BFAB7F9043007EE903AF8EEE77A304658
:107B580067EE887AFDEEE77ACDED027ABDF8081077
:107B6800FBF76AFA304619F009FBFEF7CFBA9AF824
:107B78000240C4B1013CE4B20134544451460022ED
:107B880011F8013B534083EA0313DBB2120ADF000A
:107B980042EA03228C4287EA131382EA0302EFD1F6
:107BA800002A7FF452AC794A7D4F794B12887D4C7C
:107BB800FA61DFF808921A68FA629B68B4F85221F1
:107BC800F8660021FB64D9F80000F963FA65F8F754
:107BD80093FB029000287EF4CAA90221D9F800007C
:107BE800F9F7C2FA94F854319AF803200392642BF7
:107BF8004FF0040287F8742040F0578194F855310B
:107C0800072B04BF9DF8083084F8553194F8553196
:107C1800069307EB031ADAF804100291084627F0D6
:107C280007FCDAF8081005915FFA80FA084627F091
:107C3800FFFBC0B204900AEB0002069B5A48029967
:107C480002900832C27123F00F02864682720498AD
:107C580003F00F0300EBCA008EF80D3052468EF881
:107C68000E000EF10F0028F009FA504B049A0599FE
:107C78000AF10900184428F001FA0298C37903F1BF
:107C8800010ACBB1013B5FFA83FC0CF1080CDFF869
:107C980030E184440023073010F8011B59408B0061
:107CA800CA0883EA410302F018024B404EFA02F276
:107CB80053408445DBB2EFD13C4A03980AF80230BE
:107CC8001DF06AF994F855310022013384F85531D2
:107CD80084F85421029BDDF808A09B785BB11AF860
:107CE8000510D9F80000F9F753FA01359AF802306F
:107CF800EDB2AB42F3D894F854310322013384F83F
:107D0800543187F8742088F80020FFF762B8022100
:107D1800D8F80000F9F728FA94F82C31FEF7E4B8FF
:107D28001023042218460AA98DF82A908DF82B9062
:107D38008DF82C908DF82D908DF828308DF829200D
:107D48001AF0F4FC84F83791FEF7F9B8184A12686B
:107D5800D2067FF5D9AA8046FFF7D9BA1549881FF8
:107D68001AF0C8FB84F84601FFF7AFB8074B19882B
:107D7800FFF765BA104AD278002A0CBF4FF0040CFE
:107D88004FF0050CFEF76CBEE84300200C460020BF
:107D980090450020676666665041002058A08B41D8
:107DA80018000020F41B0020F06B0020F66B002068
:107DB800784E0020341D0020843F002054320020DB
:107DC8000007090E0123D8F800003B70F9F7D4F931
:107DD8000746D8F80000F9F7CFF97F067EF455A8D2
:107DE8008E287EF452A894F82031002B7EF46AA8DD
:107DF800944BC4F828312D2384F82C31FEF74CB865
:107E08000326914940E5914B914A1B68914903F437
:107E1800800383420ABF11460326042625E58E49BE
:107E28009A790B8803EB830303EB83034FEA8308F8
:107E38001FFA88F8002A00F0DE80884B1B680FFACA
:107E480083FA0BF033F840B2FEF732BA4FF0340839
:107E5800FFF7DFBB984699461846049305930393AA
:107E6800FEF71EBB7E4904260EE54FF02408FFF7F7
:107E7800D0BB4B1CDBB2042B84F849314FEA0161BB
:107E88007FF475A9FFF770B94FF01008FFF7C1BB71
:107E98000BF00CF81AF00CFD00201AF009FDFFF7A2
:107EA80042BA4FF02008FFF7B4BB97F875A06D49A8
:107EB80004951AF00F0F04BF0AF1010A5FFA8AFA53
:107EC800BAF1070F28BF4FF0010A4FEA0A1C07EB67
:107ED8000C03187C644B02930A18002392F82410B0
:107EE800614A93725FFA8CF31A46604B964607EB29
:107EF8000C024EEA000001291870D26803F1010053
:107F08000CD90239C9B28D1C1D44034603F8012B54
:107F1800AB424FEA1222F9D101310844BC4422F0A5
:107F280060030AF1010A9CF811205FFA8AFA1343E8
:107F3800BAF1080F037000F1010366D04FEA0A1C7A
:107F480007EB0C01494A087C464901449A1A91F802
:107F5800241055180EF1100E132D5FFA8EFEC6DD93
:107F6800049D0298DFF80CE1D1B28B1DDBB243F01F
:107F78004002C27103F1010CCBB14B1DDBB20833D7
:107F8800C31804930EF10100002310F8011B594097
:107F98008B0083EA4103CA084B40354902F01802B6
:107FA80041FA02F25340049A8242DBB2EDD10398BF
:107FB8000CF80E3087F875A01CF0EEFF8AE63B68D7
:107FC8005E2098473B68392098475FFA89F01AF095
:107FD8006FFC4FEA19201AF06BFCE8E44FF0080830
:107FE800FFF717BB984699461846049305939E4693
:107FF8000393FEF755BA4FF0FF3320E7174B90462F
:10800800B3F900A06420FEF753B9184A049D9A1AE0
:10801800A7E798469946184604930393FEF740BA93
:108028000393FEF73DBA98460393FEF739BA98468C
:1080380099460393FEF734BA98469946184603932F
:10804800FEF72EBA68440020F44F0308784E00204B
:10805800EC4F0308E84F03080C4600209045002029
:10806800F84F03085C290308F06B0020FD6B002023
:108078000007090EF66B00202DE9F047B0F908500B
:108088000D81EDB2442D92B00C46174600F0878260
:1080980006462FD9812D00F0D18100F28280542D1F
:1080A80000F0AF8040F2B7816E2D00F04682802D3F
:1080B80040F0F880A94B1D780B3D15F0FF0512D054
:1080C800A74F00220A2621683B88481C20600E70B2
:1080D8002168FF2B02F10102A8BFFF23481CAA4216
:1080E80020600B70EFDB01252B462846638112B018
:1080F800BDE8F087052D00F040821ED8022D78D00B
:1081080040F27681032D00F00E82042D40F0CA80E3
:108118002A4694492046FAF785FF00212046FAF7B7
:10812800B1FF22680221531C0125236028462B46F3
:108138001170638112B0BDE8F087242D57D040F24A
:10814800EE80282D00F0B481382D40F0AB800A680D
:10815800854B0125511C2160157022680521501995
:108168002060117022680A2150192060117022685D
:108178000021501920601170226819785019206068
:108188001170226859785019206011702268997806
:10819800531923602B4611702846638112B0BDE83D
:1081A800F087A02D11D040F2F980B82D00F0B981E8
:1081B800FE2D77D16D4D05F1080635F8021B2046D6
:1081C800FAF760FFAE42F8D18DE7694B08461968A7
:1081D800FAF740FF674B20461968FAF73BFF664BF2
:1081E800196820460125FAF735FF2B467DE7634BD2
:1081F800F6E70422624920460125FAF713FF2B46C9
:10820800CAE70B685F4A604F581C1121206019703B
:1082180023681278591C21601A70236897F85B202C
:10822800591C21601A70236897F85A20591C21603C
:108238001A70B7F856102046FAF724FF0021204696
:10824800FAF720FFB7F858102046FAF71BFFBD1EB3
:1082580007F1480635F8021F2046FAF713FFB54222
:10826800F8D12268494B0C21501C20605D18117010
:10827800226813F8011F501CAB4220601170F7D11F
:1082880023680222591C21601A70B7F85C10204636
:10829800FAF7F8FE0125B7F85E102046FAF7F2FE65
:1082A8002B4679E721462846FBF790FD00287FF406
:1082B8001AAF742D00F0B580772D0CD13368726831
:1082C8009A421BBF5A1C326001461978304A204630
:1082D80022F0B4FD07E7F52D00F06981392D3768E4
:1082E80000F0568200F2EE81212D01F0CD81292D7A
:1082F80040F08E827B1C33603B780A2B01F00C82A5
:10830800502B40F0FA873046FAF77AFE214F388032
:108318003046FAF775FE012578802B463CE7202D7C
:10832800C0D10B681C4D591C6A7821601A702368EB
:108338002A78591C21601A702368AA78591C216070
:108348001A7029892046FAF79DFE23686A79591C14
:1083580021601A702268A979E5E600BFAA450020C5
:108368001422002079410020EF80002000460020E0
:10837800ACF7FF1FB0F7FF1FB4F7FF1F48820020BC
:10838800805003081C480020C44200200D430020F0
:108398001DA102080422002030430020822D81D133
:1083A8000B68B14AB14D1178B14A581C2060197058
:1083B80011892046FAF766FEAE4B22681B88FF2B10
:1083C80002F10101A8BFFF2321601370A96881F39E
:1083D800100189B22046FAF755FE296801F30F010A
:1083E80089B22046FAF74EFEA34B226819789AE61E
:1083F800012D7FF457AF0B680022591C21601A70B9
:1084080023685A1C22601D7022682421531C236093
:108418002B461170C0E6522D7FF444AF226800212C
:1084280081E6336872689A421BBF5A1C3260014663
:108438001978924A204622F001FD54E6904B1E78A6
:108448000A3E16F0FF063FF44EAE8E4B8E4F1E448A
:1084580003F101080A2314E0502B00F002810025E3
:1084680029462268501C206020461370FAF70AFE3D
:1084780029462046FAF706FEB0453FF434AE18F810
:10848800013B0A2BE8D1814A9568116805EB8505FF
:108498004FF6FF726D009542A8BF15469142A8BFDE
:1084A800114625EAE57521EAE171ADB289B2D8E74E
:1084B8000B68DFF80882764E591C022221601A7078
:1084C800236806275A1C22601F7023680A22591C39
:1084D80021601A70236801255A1922601D70B8F8A6
:1084E80000102046FAF7CEFDB8F802102046FAF739
:1084F800C9FD23685A1922601F7023685022591930
:1085080021601A7023680022591921601A70318875
:108518002046FAF7B7FD71882046FAF7B3FD2B46D7
:108528003AE65C4B5CE60B685A1C0A601D700B68E7
:108538000222591C21601A7070E74E4B0A681B888A
:108548004A4DFF2BA8BFFF23511C21601370A96857
:1085580081F3100189B22046FAF794FD4E4B20466C
:108568001988FAF78FFD296801F30F0189B22046AF
:108578000125FAF787FD2B460EE60B2247492046D0
:10858800FAF750FD082246492046FAF74BFD012527
:10859800072244492046FAF745FD2B46FCE5002A08
:1085A8003FF4A1AD404B136001252B46F4E5336839
:1085B80072689A4241F088803C4BFF221A704FF053
:1085C80000093B4D09F06EFB49462022394885F8E1
:1085D80000902AF06AF88DF808909DF80830072B6B
:1085E80001F21681DFF8D880324E4A469DF80830ED
:1085F80003EB430308EBC3035B7CE3B19DF808304E
:1086080003EB430308EBC30320215B699BB19DF88F
:10861800083003EB430308EBC303586946F822000C
:10862800F9F7EAFB2B7856F82300F9F7A7FD2A7823
:108638000132D2B22A709DF808300133DBB28DF8CE
:1086480008309DF80830072BD0D92368591C2160C1
:108658001A70002F3FF447AD174B3B6001252B469E
:108668009AE5BD68396811E7224600209045002048
:10867800304300200C46002094430020FDAC020843
:10868800AA450020B029030808220020D021002094
:1086980004220020FC2A00206043002088500308A0
:1086A80094500308A0500308FD3C0008C01E002099
:1086B800FF860020D0860020A5EA02082478002042
:1086C800644A0020552D73D0572D40F0A1807B1CA3
:1086D8003846336010F8377B0DF1070201333360F9
:1086E80013F8011C02F8011F8342F7D1434A13789B
:1086F800002BFCD1DFF8109199F80050002DFDD126
:10870800DFF808A10126DAF8000089F80060F9F717
:108718002FFD3B4B28461E7025F000F8284624F014
:10872800FDFF092024F0FAFF384624F0F7FF02AFD6
:108738003D460DF13E08EE1BF6B20A2024F0EEFF8E
:10874800304624F0EBFF15F8016B0B2024F0E6FF10
:10875800304624F0E3FF0020F8F724FD4545EAD130
:10876800082024F0DBFFA02024F0D8FFA02024F06C
:10877800D5FF002024F0D2FF10F02006F6D1DAF859
:1087880000000125F9F7FAFC89F800602B4603E59B
:108798007B1C33603B780A2B00F0C4873046FAF71D
:1087A8003BFC3046FAF738FC3046FAF735FC9AE4D9
:1087B8007B1C336097F80080B8F1FF0F01F006804A
:1087C800B8F1FE0F00F0BF873046FAF719FC96E8BB
:1087D8000C009B1A002B07DD531C336013781BB960
:1087E800B8F10B0F40F2E787B8F1240F00F25F826F
:1087F800044B012523F818002B46CDE4213900202D
:10880800363B0020C44200202D3B002014480020A5
:1088180072680B3DD31BEF2D00F2498201A151F87C
:1088280025F000BFE5910008B78C0008B78C000858
:10883800B78C0008B78C0008B78C0008B78C000804
:10884800B78C0008B78C0008B78C0008B78C0008F4
:10885800B78C0008B78C0008B78C0008B78C0008E4
:10886800B78C0008B78C0008B78C0008B78C0008D4
:10887800B78C0008B78C0008B78C0008B78C0008C4
:10888800B78C000895910008B78C0008779200080B
:10889800B78C000855920008B78C0008B78C000800
:1088A800B78C000891920008B78C00083B9100082B
:1088B800B78C00084D960008B78C0008279600086A
:1088C800B78C00087F960008B78C000895930008BD
:1088D800B78C000849930008B78C0008B78C0008CB
:1088E800B78C0008B78C0008EF800008B78C000828
:1088F8002D930008B78C0008B78C00081393000864
:10890800B78C0008B9920008B78C0008B78C00082B
:10891800B78C0008B78C0008B78C0008B78C000823
:10892800B78C0008B78C0008E7950008B78C0008DA
:1089380059950008B78C0008B78C0008A79500085F
:10894800B78C0008B78C0008B78C0008B78C0008F3
:10895800B78C0008B78C0008B78C0008E9930008AA
:10896800B78C0008B5940008B78C0008D1900008AF
:10897800B78C000841900008B78C000819900008CF
:10898800FB8F0008B78C0008B78C0008B78C00086C
:10899800B78C0008B78C0008B78C0008B78C0008A3
:1089A800B78C0008B78C0008B78C0008B78C000893
:1089B800B78C0008B78C0008B78C0008B78C000883
:1089C800B78C0008B78C0008B78C0008B78C000873
:1089D800B78C0008B78C0008B78C0008B78C000863
:1089E800B78C0008B78C0008B78C0008B78C000853
:1089F800B78C0008B78C0008B78C0008B78C000843
:108A0800B78C0008B78C0008B78C0008B78C000832
:108A1800B78C0008B78C0008B78C0008B78C000822
:108A2800B78C0008B78C0008B78C0008B78C000812
:108A3800B78C0008B78C0008B78C0008B78C000802
:108A4800B78C0008B78C0008B78C0008B78C0008F2
:108A5800B78C0008B78C0008B78C0008B78C0008E2
:108A6800B78C0008B78C0008B78C0008B78C0008D2
:108A7800B78C0008B78C0008B78C0008B78C0008C2
:108A8800B78C0008B78C0008B78C0008B78C0008B2
:108A9800B78C0008B78C0008B78C0008B78C0008A2
:108AA800B78C0008B78C0008B78C0008B78C000892
:108AB800B78C0008B78C0008B78C0008B78C000882
:108AC800B78C0008B78C0008B78C0008B78C000872
:108AD800B78C0008D18F0008B78C0008BB8F00083E
:108AE800B78C0008B78C0008B78C0008B78C000852
:108AF800B78C0008B78C0008B78C0008B78C000842
:108B0800B78C0008B78C0008B78C0008B78C000831
:108B1800B78C0008B78C0008618F0008B78C000874
:108B2800298F0008B78C00084D8E0008338E000886
:108B3800178E0008B78C0008FD8D0008B78C000858
:108B4800D58D0008B78C00087B8D0008B78C00080D
:108B58004D8D0008B78C0008B78C00082B8D0008D5
:108B6800FD8C0008E98C0008C18C0008998C00086D
:108B7800778C0008B78C0008B78C0008B78C000801
:108B8800B78C0008B78C0008B78C0008B78C0008B1
:108B9800B78C0008B78C0008B78C0008B78C0008A1
:108BA800B78C0008B78C0008B78C0008B78C000891
:108BB800B78C00085D8C0008B78C0008B78C0008DB
:108BC800058C0008B78C0008B78C0008B78C000823
:108BD800B78C0008B78C0008B78C0008B78C000861
:108BE800ED8B0008BE4B1B78DB0760D40125FCF732
:108BF800EFF8FCF7EFFE2B46FFF7CEBA7B1C33608D
:108C08003B780F2B53D8BA1C3260C3EBC303B54A69
:108C18007978D154F91C31601344BA785A703A1DE6
:108C28003260FA789A707A1D32603A79DA70BA1D31
:108C380032607A791A71FA1D3260BA795A7107F17D
:108C480008023260FA799A71012523F02BFD2B4630
:108C5800FFF7A2BA3046FAF7D3F9A34FF8813046A6
:108C6800FAF7CEF90125B8812B46FFF795BA3046B9
:108C7800FAF7C6F99D4F38823046FAF7C1F978827B
:108C88003046FAF7BDF90125B8822B46FFF784BABA
:108C98003B467A1C326013F8020B3360FB1C797870
:108CA8003360BA7816F0D2FA00287FF41CAA4FF085
:108CB800FF352B46FFF770BA3B467A1C32608C4A68
:108CC80013F8021B11703360874A7B789370FB1C82
:108CD8003360884BBA789A7001252B46FFF75CBA47
:108CE800854B864918684E22012527F0C7F92B467F
:108CF800FFF752BA3A467B1C3360814B12F8021BCD
:108D0800197032607A785A70FA1C3260BA789A70A0
:108D18003046FAF775F97B4B0125D8802B46FFF7CB
:108D28003BBA3046FAF76CF9764F38803046FAF796
:108D380067F978803046FAF763F90125B8802B4641
:108D4800FFF72ABADFF8CC8198F80030002B3FF4FF
:108D5800CAA96D4F00253046FAF752F90CF056F9BA
:108D680098F80030A7EC010A01359D42F3DBFFF7C4
:108D7800BAB90D2B9BD17B1C33603D78072D96D853
:108D8800DFF8948130460C27FAF73AF907FB05F724
:108D980008EB0705A8803046FAF732F9E880304634
:108DA800FAF72EF9336828811A46591C316012F8EF
:108DB800021BA97232605B78EB723046FAF708F949
:108DC800012548F807002B46FFF7E6B97B1C3360FE
:108DD8003878060600F1DB85414B1B78DD073FF547
:108DE80082A9032828BF00200125FBF7D5FF2B46C1
:108DF800FFF7D2B93A4B1B78D8073FF574A901257C
:108E0800FCF7B6F8FCF7E6FD2B46FFF7C5B9344B7F
:108E18001B78DA073FF567A93C4A1378012543F028
:108E2800040313702B46FFF7B7B92D4B1B78D907EE
:108E38003FF559A9364B4FF4C87201251A802B46C5
:108E4800FFF7AAB9092B7FF732AFDFF8D0803B468E
:108E58007A1CD8F80050326013F8022B2A7033605D
:108E68007B78AB70FB1C3360BB78642BA8BF642392
:108E78003A1D6B713260FB78642BA8BF64237A1D9E
:108E8800AB7132603B79EB71BB1D33607B79642B2E
:108E9800A8BF6423FA1D2B723260BB79EB7007F10F
:108EA80008033360FB792B713046FAF7A9F872682A
:108EB80033686881D11A00290CDD591CD8F80000E4
:108EC8003160521A002A1978417203DD9A1C326007
:108ED8005B784370012513F0AFF82B46FFF75CB9B8
:108EE8009C450020247B002034780020244B00205F
:108EF800544E00204478002070410020E02A0308E6
:108F08002C780020DC2C0020342C00202C4300205E
:108F180006870020AA450020307A0020FC3800206F
:108F2800BC4B1868FB1C02462137991E316013F8A8
:108F3800031C1170591E316013F8021C5170336004
:108F480013F8011C91700333BB4202F10302ECD108
:108F580023F05AFFFFF7C7B8C3F34705122D3FF6B2
:108F6800A6AEB5B112AB0DF1060903EB4507C8462D
:108F7800423F3046FAF744F828F8020F4745F8D13F
:108F8800A54B39F8022F23F8022FC845F9D1112D26
:108F980009D8A24A6B00023B13440021223223F86D
:108FA800021F9A42FBD19E4A01231D461370FFF708
:108FB800F3B89C4F002330463B60FAF709F80125C7
:108FC80038602B46FFF7E8B83B467A1C326013F846
:108FD800025B3360FB1C78783360B978002D00F0B1
:108FE800E184012D7FF47FA809F030FF2B46FFF7BD
:108FF800D3B88D4B1B7813F001017FF458AE7B1C5E
:1090080033603878012509F063FE2B46FFF7C4B8B2
:109018003B467A1C3260854A13F8021BD1703360D4
:10902800834A7B785371FB1C3360824BBA78DA70C1
:1090380001252B46FFF7B0B83046F9F7E1FF304677
:10904800F9F7DEFF3046F9F7DBFF3046F9F7E4FFC2
:109058003368704D1946581C2A68306011F8020BA5
:1090680082F82C003160597882F83610D91C3160AA
:109078009B7882F837303046F9F7CEFF3046F9F75B
:10908800CBFF3046F9F7C8FF30462F68F9F7B8FF2D
:10909800788730462F68F9F7B3FF336872683887E6
:1090A800D11A01290ADD591C2A6831601B7882F817
:1090B8002E303046F9F7B0FF33687268D31A032BA5
:1090C80000F35984286843E77B1C3360514DDFF86F
:1090D80078813B7888F8053030462F68F9F790FF9B
:1090E800388430462F68F9F78BFF72683368F88345
:1090F800D11A072900F31084D11A032900F3FE833B
:10910800D21A002A05DD591C2A6831601B7882F8BA
:109118002630FBF767FE1AF023FA474B28681B68CE
:10912800002B00F07883012523F04EFB2B46FFF738
:1091380033B87B1C414D33603B782B723046F9F7CE
:109148005FFFA8833046F9F75BFF28833046F9F7BD
:1091580057FF32686883531C33601278EA74726868
:10916800D31A032B00F396833368D11A052900F329
:109178005D83D21A002A7EF7B6AF5A1C32601B787C
:1091880085F8213001252B46FFF706B87B1C336094
:109198003D78132D3FF68BADBB1C3360787821F0FA
:1091A80087FE00283FF483AD254B027803F825207D
:1091B800FA1C326003EB8503BA785A703A1D3260A4
:1091C800FA789A707A1D326012493A79DA7008682A
:1091D800012512F0BFFE2B46FEF7DEBF194A102B01
:1091E8004FF0000128BF1023116051609160D160D9
:1091F8001174002B3EF477AF3168013A0B4401310A
:10920800316011F8010C02F8010F8B42F7D1FEF71B
:109218006ABF00BF70410020623000206430002027
:1092280088300020FC2A00209C450020347800204B
:109238004C45002044780020903400200C50002039
:10924800AC34002058410020544E00203046F9F735
:10925800D7FEB34F38603046F9F7D2FE7860304613
:10926800F9F7CEFE0125B8602B46FEF795BFAD4F46
:1092780000233B603046F9F7ABFE3B68012503430A
:109288003B602B46FEF788BF7B1C3360A6493878C5
:109298000870D21A002A7EF726AFBB1C33607B7891
:1092A800003318BF012301254B702B46FEF774BF0E
:1092B8007B1C33609C4B3A78DFF868821A70002375
:1092C800C8F800303046F9F783FE3268D8F8003025
:1092D8009649934D0343501CC8F80030306013780A
:1092E8000B723046F9F78CFE28603046F9F788FE95
:1092F80068603046F9F784FEA8603046F9F780FECA
:109308003046F9F77DFEFEF7EEBE894B07F10802FD
:109318000137376017F8011C03F8011FBA42F7D16B
:10932800FEF7E1BE3B467A1C3260824A13F8021B04
:10933800917033607B78537001252B46FEF72CBF64
:109348000722B3FBF2F2C2EBC2055B1B7FF4AFACA2
:10935800D2B202F1FF385FFA88F8002A3EF4C3AEB1
:10936800DFF8D49108F101081D467B1C3360724B6D
:1093780097F90010002793F902208A4203F10803A5
:1093880000F0F4810137062FF5D190E47B1C33609F
:109398003B780E2B3FF68BACBA1C326078780328EA
:1093A8003FF685AC6549062202FB03F28B18FD1CCB
:1093B80058713560B87888543A1D3260FA785A7016
:1093C8007A1D32603A799A70BA1D32607A79DA7009
:1093D800FA1D3260BA791A7101252B46FEF7DCBEF8
:1093E8003046F9F70DFE054613F062FFFF283EF4FC
:1093F8007AAE3F2D00F2A8820DF14808002308F844
:10940800403DEF0841460DF107008DF80730013760
:1094180013F04EFE9DF80730FFB205F00705BB427A
:1094280005F1010503D19DF80830AB4203D0294668
:10943800384613F029FF33687268D21A012A7EF77A
:1094480052AE5A1C12A8326000221D7800F8412D35
:1094580013F022FE9DF80730AB420AD0384B1B6848
:109468003BB19A79AA4204D31B681B690BB1284601
:10947800984733685A1C3260404600221D788DF8A0
:10948800082013F0FDFD9DF80830AB423EF42BAEEA
:109498002B4B1B68002B3EF426AE1B685B69002B28
:1094A8003EF421AE28469847FEF71DBE3B467A1C7F
:1094B8003260DFF8988013F8022B88F802203360B6
:1094C800204A7B781370FB1C33601F4DBB782B71CF
:1094D8003B1D3360FB78092BA8BF09233046AB70CE
:1094E800F9F78EFD336872682880D11A012905DDE5
:1094F8003046F9F785FD33687268E8819A4240F092
:10950800E881FBF76FFC336872689A423EF4EBAD72
:109518005A1C32601B78EB7001252B46FEF73CBEC7
:10952800282A002048820020A83400200C5000205F
:109538000B5000205078002028480020082B0020DD
:109548006C41002028780020244B0020544E002035
:109558007B1C336097F80080B8F1110F3FF6A7AB7A
:10956800BB1C3360B94D7B7805F818303046F9F7E5
:1095780047FD40F6CA039842A8BF184640F2EE23BA
:10958800984205EB4801B8BF18460125A0F2EE2223
:109598002B46192092FBF0F24A70FEF7FDBDAC4B4A
:1095A8001B78012B3EF69FAD39467B1C3360DFF8F4
:1095B800E08211F8023B88F802303160FB1C7878B1
:1095C8003360D31A012BB97840F38C813046F9F710
:1095D80017FD0125A8F800002B46FEF7DDBD3B4628
:1095E8007A1C9C4D326013F8022B2A7133607B7809
:1095F8006B713046F9F704FD336828805A1C3260D5
:109608001B78AB713046F9F7FBFC336868805A1C4D
:1096180032601B78EB7101252B46FEF7BDBD7A1C25
:1096280032603D781F2D3FF642AB052B7FF43FABF0
:109638003046F9F7CDFC884B43F8250013F07CFC45
:10964800FEF751BD844D05F140073046F9F7D8FCC7
:109658003368A5F88000591C1A46316012F8021BBD
:1096680085F8821032605B7885F883300435BD4216
:10967800EBD1FEF738BD7B1C3360784B3A785A75CE
:1096880001252B46FEF788BD3B467A1C3260744D97
:1096980013F8022B6A7033607B782B70FB1C3360E5
:1096A800BB78AB703046F9F7ABFC33682881591C9E
:1096B8001A46316012F8021B697132605B78AB712F
:1096C80001252B46FEF768BD5A1C194632606548CD
:1096D80011F8022B027031605B784370042A04D9B8
:1096E800FF2A7EF49BAEFEF76ABF5F49097899426C
:1096F80005D8022A7EF492AEFF2B7EF48FAE236843
:1097080001255A1922601D70002F3EF4ECAC574B0E
:109718003B602B46FEF740BD3046F9F771FC544FCD
:10972800FEF7F5BDBB1C3360524B7A781A70FA1CF1
:109738003260BA785A703A1D3260FA789A70012508
:109748002B46FEF729BDBB1C33607D78022D3FF602
:10975800AEAA3046F9F754FC474B03EB45034FF0EC
:10976800FF35A3F85C002B46FEF716BD09EBC70AC8
:1097780030468AF80210F9F743FC336829F83700B5
:109788001A46591C316012F8021B8AF8031032601D
:109798005A788AF80420DA1C32609A788AF8062007
:1097A8001F1D37600135DB788AF80530A8457FF43E
:1097B800DCADFEF798BC304B0030984418BF012050
:1097C800012588F84A002B46FEF7E6BCBB1C33602F
:1097D8002A4B7A781A70FB1C3360DFF89C80BB78C0
:1097E80088F85B303B1D3360FB7888F85A30304688
:1097F800F9F706FCA8F856003046F9F701FC3046A0
:10980800F9F7FEFB0125A8F858002B46FEF7C4BC63
:109818004A46FEF71ABF1A481A491B4A1B4B0360EF
:1098280001250B6013602B46FEF7B6BC5A1C32604C
:109838001B78EB723046F9F7CBFB3368E8605A1CAB
:1098480032601B782B743368726892E4AC32002063
:1098580041820020F42C0020244000200C500020DD
:1098680030430020C01E0020AA450020153D0008F6
:1098780024780020EF800020C44200201C480020EB
:109888009C7B0020F07B0020587C002039060008D3
:10989800404300203046F9F7B3FBA8843046F9F777
:1098A800AFFB33687268E884D11A03297FF75DAC8F
:1098B8001A46591C316012F8021BA97732605B788E
:1098C80085F820303046F9F79BFB33687268688466
:1098D8004BE45A1C32601B78003318BF012388F808
:1098E80007300EE6324B1A88012512FB00F22B4690
:1098F80092FBF1F2A8F80020FEF74EBC3046F9F7CB
:109908007FFBA8F80E003046F9F77AFB33687268D7
:10991800A8F81000FFF7F4BB3046F9F771FBA8F878
:109928000A003046F9F76CFBA8F80C0030462F689F
:10993800F9F766FB788430462F68F9F761FB3368DE
:109948007268B884FFF7D8BB0DF10808404613F0D9
:109958008BFBBDF80830AB423FF46DAD154B1B686F
:10996800002B3FF468AD1B689B69002B3FF463AD87
:10997800284698475FE530462F68F9F741FB788617
:1099880030462E68F9F73CFBB086FFF79BBB00F02A
:109998007F00032828BF0020012509F073FA2B4611
:1099A800FEF7FABB012523F0A5F82B46FEF7F4BB1A
:1099B800BC7700206C4100202DE9F04F2DED0C8B79
:1099C8003C4B1B7891B0012B059001F072863A4C04
:1099D80094F80021002A41F0BF80072B374D01F091
:1099E8006386002302936B6834489847002800F088
:1099F8006981B5F8B470002285F85520002F40F031
:109A08004187B5F93E00AA6AB5F93C60696AB5F9BB
:109A18004030DFF8B4B0821AE86A6A63711A1B1A18
:109A28002963274895F85610AB6310F07FFEDBF8E2
:109A38000030990040F1F080D5ED0D5AD5ED0C7A43
:109A4800204A94ED636AD4ED646A94ED657AD4F89B
:109A580098311268B8EEE58AD5ED0E5AF8EEE77A35
:109A6800F8EEE58A013377EE867A38EE268A78EEC4
:109A7800878A9342C4ED637A84ED648AC4ED658A6B
:109A8800C4F8983101F0D0830A4B1F78142F02F0E4
:109A980048870023D4F8A0610393062E00F2AF8014
:109AA800DFE816F07A16D6159C14EA151400671527
:109AB800001500BFFC450020C41E0020047E0020C5
:109AC800347E002000350020784E0020D64B1A78CE
:109AD800D4F8A4E1DFF8C4C39FEDD47A4FEACE00EE
:109AE8000CEB000383ED007A002A7DD0D049B0EE5C
:109AF800476AF0EE476A0023F1EC017A013367EE1A
:109B0800A77A05EE903AB4EEE77AF1EE10FAF8EE9D
:109B1800E55AB8BFB0EE677A934276EEA76AA7EE29
:109B2800A56AE9D1F5EEC06A0CEB0003F1EE10FA74
:109B380083ED007A58DDC6EE265ABE4BBE4A12881F
:109B4800F7EE007A75EEE75AD3ED007A65EEA77A5C
:109B5800FDEEE77A17EE903A812B43F3F8849342AF
:109B6800A8BF134607EE903AF8EEE77AB34B00EB3E
:109B78000E0103EB810393ED057AD3ED003A93EDE3
:109B8800066A93ED014AD3ED046AD3ED034A93EDD7
:109B9800025AA3EEA77AA4EE276A66EEC76AA7EE72
:109BA800646ABDEEC77AE5EE276A17EE101A8129B6
:109BB80083ED056AC3ED066A43F3CD848A42A8BFE4
:109BC8000A4607EE902AF8EEE77AFCEEE77ACDED42
:109BD800047ABDF810300CEB00029380BEF1000F40
:109BE80002D1132F04F02481152F42F04C846044D5
:109BF800DFF8AC82838828F81E30D4F8A061904B37
:109C0800013683FB06239A19F317C3EBA203C3EBB0
:109C1800C303F61AC4F8A0618A4B1B78002B01F025
:109C2800A180894EDFF87C92DFF874A206F5BC7833
:109C38000027864BD5ED087A1B78172B01F08E8309
:109C480096ED007AB8EEC78A082B28EE278A07D146
:109C5800B0EE480A039326F01BFC039B2AF8170072
:109C6800DBF8002092000BD5002F04F09B85B0EEA6
:109C7800480AD5F8143208F170009847B0EE408AC7
:109C8800B0EE480AD5F83431A8F170009847D5F8F5
:109C9800A431404698476D4B1B78032BB0EE408AA1
:109CA80001F05683D6F8F800D5F8B830B0EE480A77
:109CB80098470137032F08F12408A9EC010A06F197
:109CC8000406B6D1614B93F80090B9F1070F00F084
:109CD800968694F8B031002B40F09E865C4B5B79F9
:109CE800002B40F0C9850123584A84F8B031127816
:109CF800072A02F0578000230793564B94ED6E9A7B
:109D080093ED007A544BD4ED6DCAD3F800A0534BB1
:109D18000393F7EE007A37EEC9CA514B06932CEE3F
:109D280007CA504B0493B4EEE7CA0025F1EE10FAC7
:109D38004D4BDFF87491DFF874B1DFED4C8A9FED7D
:109D48004CAADFED3ABADFED4B9A9FED4BBADFED47
:109D58004BAADFF85C814A4F029388BFB0EE67CA0E
:109D68002E46484B99ED008A2B44D3ED007AF5EE48
:109D7800407AF1EE10FA17D0434B2B44D3ED006A2A
:109D880038EE667AB0EEC76AF4EEC67AF1EE10FAEB
:109D980008D5B5EEC07AF1EE10FACCBF37EEA68A38
:109DA80036EEE78A83ED008A039B1A88930700F052
:109DB8008180022E7ED09AF82E10344B07EE901A2E
:109DC8002B4493ED007A4B42F8EEE76A07EE903A9F
:109DD80026EE877AF8EEE77AB4EEE77AF1EE10FA33
:109DE8000AD407EE901AF8EE677AF4EEC77AF1EE25
:109DF80010FA88BFF0EE477A254B264903EB460355
:109E080031F91600B3F90C30C01A07EE100AB8EE93
:109E1800C77AD007E7EE687A40F106861E4B93EDC5
:109E2800008A27EE888A45E00635002000000000F9
:109E3800C41E002008350020043500203C370020CF
:109E480093244992FC340020347E0020FC450020F5
:109E5800544E0020AC7C0020704100204C41002072
:109E680090000020684E0020E8320020CDCCCC3D88
:109E7800AE47813F0000C842610BB63B0000344347
:109E8800F4320020A07C0020802000203020002018
:109E98003478002050410020887C0020243700209E
:109EA800004600206C4E0020C81F0020987B002030
:109EB80000330020049B94F8C8212B44D3ED01DA29
:109EC80038EE6DDA002A3DD0D24BD4F8CC21059972
:109ED8001B688A1A9A4235DD9AF84830022B01F03D
:109EE800D687022E04F0C683CB4B1B68990740F136
:109EF8002087CA4BCA49DFF894E331F916C09EEDB2
:109F0800008ADFF88CE3C7ED00BA03EB460028EEC1
:109F1800288AB0F90C00A0EB0C0007EE900AF8EEC6
:109F2800E77ADEF8000027EE888A904238EE6DDA8C
:109F3800C1F22C81F7EE007AB4EEE79AF1EE10FA4E
:109F480001F1FB80B74B2B4493ED000A029B2CEEEA
:109F5800800A022E20EE0D0AA3EC010A029304F0F7
:109F6800A383069B9BED007AD3ED007AAE4BD7ED29
:109F7800006A93ED006AAD4B67EE277A2B4427EE13
:109F88008C7AD3ED007A67EE277AF0EE665AEDEE1A
:109F9800275AB1EE467AB4EEE57AF1EE10FA08DC0B
:109FA800F4EEC65AF1EE10FA8CBFB0EE467AB0EE77
:109FB800657A94ED6E6AF7EE007AB4EEE76AF1EE30
:109FC80010FAACBF0123002343B1F0EEE66AF0EECD
:109FD800C77AF4EEE67AF1EE10FA01D587ED007A49
:109FE800022E04F0FB82924A924B52F826001B681C
:109FF800B0EE6D0A9847904A904B52F826001B68BD
:10A0080098479AF8373023B1039B1B88002B00F040
:10A018006F85B0EE6B8A8A4B9BED007A38EE400A6A
:10A028002B4493ED008A83ED000A9AF8483030EE0D
:10A03800480AC0EE077A2BB3824B1B78DB0721D581
:10A04800B7EE007AB4EEC79AF1EE10FA04DB94F892
:10A05800C831002B00F05B87D4F8CC31059AD31AAD
:10A068006C4A12689A420DDD774B93ED007AB0EE98
:10A07800CDDAB4EEC7DAF1EE10FA41F1A38000238D
:10A0880084F8C831714B94F8D8212B4493ED007AA9
:10A098002CEE877A67EE277AC8ED007A32B9029BF0
:10A0A800C7ED00BA43ED01BAC8ED00BA0136032E78
:10A0B80009F1040908F1040807F1040705F104058A
:10A0C8007FF44FAE624B1B78072B01F03D83012BC9
:10A0D80001F05586002594F8E031002B40F0F38517
:10A0E8005C4A5D4B10681B6810F4805E93F82C3056
:10A0F80040F06286594A5A4992ED006A498B594A9A
:10A1080084ED7C6A92ED007A574A84ED7D7A07EEF9
:10A11800901AF8EEE76AD2ED037A544A84ED7A6A27
:10A1280037EE467A77EEE67AD2ED006A84ED797AF0
:10A13800012284F8F821C7EEA65A4D494D4A91EDFF
:10A14800005A4D499FED4D6A91ED004A4C49DFEDAB
:10A158004D6AD1ED004A92ED007A35EE045AF7EED9
:10A16800007AF4EEE75A35EE245AF1EE10FA88BF79
:10A17800F0EE675A25EE065AF4EEE65AB1EE476A53
:10A18800F1EE10FAB4EEC65AB8BFF0EE665AF1EE28
:10A1980010FAC4ED7F5A01F1D480B4EEC75AF1EE3B
:10A1A80010FA88BFB0EE475A314ADFED346AD2ED73
:10A1B800017A314A92ED014A314A77EE847AD2ED3A
:10A1C800014A77EEA47A67EEA67AB4EEE76AF1EE72
:10A1D80010FA08DCB4EEE77AF1EE10FA8CBFB0EEB4
:10A1E800676AB0EE476A224ADFED246AD2ED027A46
:10A1F800214AD2ED024A244A77EEA47A92ED007AF7
:10A2080067EEA67AB1EE473AF4EEC37AF1EE10FAA9
:10A2180049D43FE0B47C0020A043002034780020DB
:10A22800504100205C7C0020D07C0020687C00200D
:10A23800A07B00209C7B0020F47B0020F07B00208A
:10A24800942000209C450020C07C0020747C0020C5
:10A25800FC450020784E002070410020CC7700207B
:10A268000C500020D077002024460020E42C002049
:10A27800E8320020D47C0020F43200206F12833AA8
:10A288000033002000000000D87C0020887C0020DB
:10A29800B07C0020F4EEC77AF1EE10FA8CBFB0EE75
:10A2A800473AB0EE673AF04A52780AB9B1EE433A03
:10A2B800002B41F09283F7EE003AEC4E3278002AF8
:10A2C80002F01085EA4BDFEDEB7AD3ED024AD3EDCD
:10A2D800016A93ED037A66EE244AE5EE264AE3EE38
:10A2E800074A63EEA44AF4EEE74AF1EE10FAB4BF67
:10A2F800B0EE674AB0EE644A98BFF0EE647A012A7D
:10A30800CDED084A02F0568693ED067AD3ED052A7C
:10A31800D3ED076A26EE077AA5EE227AA3EE267A0F
:10A3280023EE877AB4EEE77AF1EE10FAB4EEC47A47
:10A338008CBFF0EE676AF0EE476AF1EE10FA88BF5C
:10A34800F0EE676AB4BFF0EE447AF0EE477A022A7C
:10A358008DED097A00F0DE8093ED0A7AD3ED092AB3
:10A3680093ED0B4A26EE077AA5EE227AA3EE047A3D
:10A3780023EE877AB4EEE67AF1EE10FAB4EEE77AD5
:10A388008CBFB0EE664AB0EE474AF1EE10FA98BFBD
:10A39800F0EE446AA8BFF0EE477A032A8DED0A7AF8
:10A3A80000F0B88093ED0E7AD3ED0D2A93ED0F4AA5
:10A3B80026EE077AA5EE227AA3EE047A23EE877AB0
:10A3C800B4EEE67AF1EE10FAB4EEE77A8CBFB0EEAE
:10A3D800664AB0EE474AF1EE10FA98BFF0EE446ACA
:10A3E800A8BFF0EE477A042A8DED0B7A00F0928030
:10A3F80093ED124AD3ED112A93ED137A26EE044A0F
:10A40800A5EE224AA3EE074A23EE844AB4EEE64AB2
:10A41800F1EE10FAB4EEE74A8CBFB0EE667AB0EE11
:10A42800447AF1EE10FA98BFF0EE476AA8BFF0EE52
:10A43800447A052A8DED0C4A6CD093ED164AD3ED7B
:10A44800152A93ED177A26EE044AA5EE224AA3EEC2
:10A45800074A23EE844AB4EEE64AF1EE10FAB4EE67
:10A46800E74A8CBFB0EE667AB0EE447AF1EE10FAA5
:10A4780098BFF0EE476AA8BFF0EE447A062A8DED41
:10A488000D4A47D093ED1A4AD3ED192A93ED1B7A5A
:10A4980026EE044AA5EE224AA3EE074A23EE844A92
:10A4A800B4EEE64AF1EE10FAB4EEE74A8CBFB0EE2D
:10A4B800667AB0EE447AF1EE10FA98BFF0EE476A89
:10A4C800A8BFF0EE447A072A8DED0E4A22D093ED0C
:10A4D8001E7AD3ED1D2A93ED1F4A26EE077AA5EEC4
:10A4E800227AA4EE037A27EE237AB4EEE67AF1EE26
:10A4F80010FAB4EEE77A8CBFB0EE666AB0EE476A3F
:10A50800F1EE10FA8DED0F7A98BFF0EE466AA8BF0B
:10A51800F0EE477A77EEE67AF7EE006AF4EEE67A3E
:10A52800F1EE10FAC4ED6E7A43F3678486EEA77AEB
:10A53800022ADDED097A67EE244A67EE877ACDEDC7
:10A54800084ACDED097A2DD0DDED0A7A67EE877AD3
:10A55800032ACDED0A7A25D0DDED0B7A67EE877AEE
:10A56800042ACDED0B7A1DD0DDED0C7A67EE877AE3
:10A57800052ACDED0C7A15D0DDED0D7A67EE877AD8
:10A58800062ACDED0D7A0DD0DDED0E7A67EE877ACD
:10A59800072ACDED0E7A05D0DDED0F7A27EE877A02
:10A5A8008DED0F7A344B1F6817F0805701F09A80B1
:10A5B800F6EE005AC4ED7F5A002A02F088832F4B2A
:10A5C800D4ED7D4A93F8039094F9F8312C49D4EDF1
:10A5D8007C6A91F800C0DFF8B4802A49DFF8B0A09F
:10A5E800B1F9061098ED007A029106EE103AFDEEE8
:10A5F800E44A254B9AF800A0B3F81AB094ED795ABA
:10A60800D4ED7A7A14EE903AFDEEE64A00F010089E
:10A6180000F480000CF0010CB8EEC66A14EE901A33
:10A628000390B9F1000F41F02182B8F1000F41F019
:10A63800A080DFF83C80DDED086A98ED007ADFF84D
:10A6480054E025EE877AA6EE267AF0EE676AE5EE04
:10A65800076ABDEEE67A17EE107A17EE100A9F42E7
:10A66800A8BF184618E000BFA8340020AA4500205B
:10A67800542C00200000000098430020843F002054
:10A688009C450020684300200C500020302C0020FE
:10A69800484B00201C330020B942C8BF084607EECB
:10A6A800100AB8EEC77A012A8EED007A00F0DC8035
:10A6B80098ED047ADDED096A25EE877AA6EE267A0A
:10A6C800F0EE676AE5EE076ABDEEE67A17EE107AF5
:10A6D80017EE100A9F42A8BF1846B942C8BF0846DD
:10A6E80007EE100AB8EEC77A022A8EED017A00F05A
:10A6F800BB8098ED087ADDED0A6A25EE877AA6EE2A
:10A70800267AF0EE676AE5EE076ABDEEE67A17EE9E
:10A71800107A17EE100A9F42A8BF1846B942C8BF60
:10A72800084607EE100AB8EEC77A032A8EED027AB9
:10A7380000F09A8098ED0C7ADDED0B6A25EE877AA9
:10A74800A6EE867AF0EE676AE7EE056ABDEEE67A6F
:10A7580017EE107A17EE100A9F42A8BF1846B942A2
:10A76800C8BF084607EE100AB8EEC77A042A8EED6D
:10A77800037A79D098ED107ADDED0C6A25EE877AA8
:10A78800A6EE867AF0EE676AE7EE056ABDEEE67A2F
:10A7980017EE107A17EE100A9F42A8BF1846B94262
:10A7A800C8BF084607EE100AB8EEC77A052A8EED2C
:10A7B800047A59D098ED147ADDED0D6A25EE877A82
:10A7C800A6EE867AF0EE676AE7EE056ABDEEE67AEF
:10A7D80017EE107A17EE100A9F42A8BF1846B94222
:10A7E800C8BF084607EE100AB8EEC77A062A8EEDEB
:10A7F800057A39D098ED187ADDED0E6A25EE877A5C
:10A80800A6EE867AF0EE676AE7EE056ABDEEE67AAE
:10A8180017EE107A17EE100A9F42A8BF1846B942E1
:10A82800C8BF084607EE100AB8EEC77A072A8EEDA9
:10A83800067A19D098ED1C7ADDED0F6A65EE875A15
:10A84800E6EE265AE5EE257AFDEEE77A17EE900A4F
:10A858008342A8BF03468142C8BF0B4607EE903A21
:10A86800F8EEE77ACEED077ABCF1000F40F03882B7
:10A87800002A40F0308233E2AB4B1B78013BDBB25D
:10A88800FFF732BAA94B04934FF47A761B68B6FBEC
:10A89800F3F3C3EB4316A649DFF8B88291F801A099
:10A8A800A449B8F9060091F8009003EB8603DE008E
:10A8B800B6B2B74202F01881D5F88810B5F93CE075
:10A8C800EB6E4A1C07EE90EA7344012AC5F888200B
:10A8D800EB66F8EEE77A02F01281D5ED1E5AD5ED57
:10A8E800206A07EE102A37EEE56AB8EEC75A012F3C
:10A8F80086EE057A37EE257A77EEC77A85ED1F7AE8
:10A90800E7EE866A85ED1E7AF0EE667AC5ED216A75
:10A91800C5ED206A02F06E84D5F89C10B5F93EE0CA
:10A928002B6F4A1C07EE90EA7344012AC5F89C2055
:10A938002B67F8EEE77A02F0FB80D5ED235AD5EDC8
:10A94800256A07EE102A37EEE56AB8EEC75A012FD6
:10A9580086EE057A37EE257A77EEC77A85ED247A82
:10A96800E7EE866A85ED237AF0EE667AC5ED266A0B
:10A97800C5ED256A02F06684D5F8B010B5F940E057
:10A988006B6F4A1C07EE90EA7344012AC5F8B020A1
:10A998006B67F8EEE77A02F0E480D5ED285AD5ED3A
:10A9A8002A6A07EE102A37EEE56AB8EEC75A012F71
:10A9B80086EE057A37EE257A77EEC77A85ED297A1D
:10A9C800E6EE276A85ED287AF0EE667AC5ED2B6A01
:10A9D800C5ED2A6A02F05E84A8F80600B5F8B4301E
:10A9E800544A013B92F80090A5F8B430049900232A
:10A9F800B9F1070F4B608B60CB607FF46AA9F6F75B
:10AA08006FF9029BDFF84C81C01A94F8B031A8F8AE
:10AA18000000002B3FF462A9013B84F8B03111B06B
:10AA2800BDEC0C8BBDE8F08F94ED5E7AB1F90000B7
:10AA3800D4ED5F6AB1F902E03F4AF4EEC76A80EAF2
:10AA4800E0738EEAEE71A3EBE073F1EE10FAA1EB7E
:10AA5800EE71B8BFF0EE476A8B42B8BF0B4607EEFF
:10AA6800103A1378B8EEC77A27EE287A002B40F010
:10AA78001F82324B93ED006AB4EECA6AF1EE10FA07
:10AA880041F11081F7EE005A75EEC65A3AEEC77AD0
:10AA980065EE8B5A2A4BA5EE876A93ED007A26EE6F
:10AAA800076AB5EEC06AF1EE10FA40F21786C9EEF1
:10AAB800865AB7EE007AB0EE476AA6EEE56AF0EE7F
:10AAC800466AF4EEC76AF1EE10FA88BFF0EE476AFC
:10AAD800F5EEC06AF1EE10FAB8BFF0EE6B6A194BEA
:10AAE80093ED007A67EE877AA7EEA68AFFF7E2B9B8
:10AAF800154B164A2B4493ED007AD2ED007A144B8D
:10AB080067EE277AF7EE006AF4EEE67AF1EE10FACD
:10AB180093ED007A88BFF0EE667A67EE877A27EEC3
:10AB2800888AFFF778BA00BF28780020684E00208E
:10AB3800544E0020FC450020947C00209C7C002082
:10AB4800907C00208C7C00203C200020847C00200D
:10AB5800807C002000460020072B02F0E3800027BD
:10AB6800DFF840B3B64DDBF80030590501F19F809E
:10AB7800B44B1B78002B40F0F581B34E94F812319A
:10AB880023B1B24A1288920742F0628094F81821E1
:10AB9800002A41F09680B37F002B00F0F583022B4A
:10ABA80002F04A80032B01F0F482A94B5B88F17F05
:10ABB8000231C9B2002A02F03080002B02F02D8049
:10ABC800A4480068B3FBF0F30FFA83F9A4F848919E
:10ABD800002903F01A8107EE909AF8EEE77AF7EE6B
:10ABE800006A86EEA77A9C4B0129D4ED576AD3ED0B
:10ABF800007A77EEE67A67EE877AC4ED537A21D049
:10AC0800D3ED017AD4ED586A77EEE67A022967EE39
:10AC1800877AC4ED547A15D0D3ED027AD4ED596A07
:10AC280077EEE67A032967EE877AC4ED557A09D07C
:10AC3800D3ED037AD4ED5A6A77EEE67A67EE877A2F
:10AC4800C4ED567A85480078092803F0AE81B9F139
:10AC5800000F40F3A08391B394ED577AD4ED537A63
:10AC680077EE877A0129C4ED577AC3ED007A21D0AF
:10AC780094ED587AD4ED547A77EE877A0229C4EDA8
:10AC8800587AC3ED017A15D094ED597AD4ED557AF6
:10AC980077EE877A0329C4ED597AC3ED027A09D091
:10ACA800D4ED5A7A94ED567A77EE877AC4ED5A7ACB
:10ACB800C3ED037A01390229B8BF0221C9B2002ABB
:10ACC80018BF022168E3664B664E1B78DF0700F168
:10ACD8006581327822B192006349644825F0CEF943
:10ACE800634B1B68002B40F03083624B1B789BB191
:10ACF800307870B1DFF87481DFF8AC910027F8B2D2
:10AD0800D9F80030B8EC010A984730780137874203
:10AD1800F5DB594B1B689847504B1B78072B00F005
:10AD2800E684012384F8003111B0BDEC0C8BBDE83A
:10AD3800F08F524BC7ED00BA1B689342BFF6FAA8D2
:10AD48004F4B1A88002384F8C831002A41F0A486A2
:10AD58004C4A4D4B1178186881F00101F7F764FAF5
:10AD6800FFF7F0B8494EDFF8449106F5F47806F598
:10AD78001577F6EC017A95ED080AD5F81432F8EE55
:10AD8800E77A404627EE800A9847A8F1E000D5F810
:10AD980034319847A8F17000D5F8A4319847D6F80F
:10ADA800F400D5F8B830984708F124084745A9ECCD
:10ADB800010ADED1FEF786BF294A1278D60703D4E6
:10ADC800214A128BA4F8EC21314A2349128891EDCB
:10ADD800037A07EE902AF8EEE77AB4EEE77AF1EE16
:10ADE80010FA41F2B8802B49098807EE901AF8EE5C
:10ADF800E77AB4EEE77AF1EE10FAC1F21D8026493F
:10AE0800264AD1ED006A92ED006A2549C4ED7C6AB4
:10AE1800BCEEC75A76EE665A15EE102AC4ED7A6A69
:10AE2800C4ED795A84ED7D6AA4F8EC210122D1EDB4
:10AE3800006A84F8F82177EE677AFFF77CB900BFDB
:10AE4800047E0020050200200C5000204C41002008
:10AE5800543000209034002024460020FC45002077
:10AE68009C450020AA450020342C00201C330020DB
:10AE7800947B0020504E0020444B0020B07C0020E2
:10AE8800007100200271002004710020347E00202F
:10AE9800E82C0020EA2C0020D42C0020D0770020B9
:10AEA800F02C0020784E00203C4B00206C4E0020F7
:10AEB800CC4B93ED005AB5EEC05AF1EE10FA40F3C0
:10AEC8000D84C94BD3ED004AF5EEC04AF1EE10FAF5
:10AED80040F3048434EEC77A66EEE95A87EE246AB2
:10AEE800C5EE856AB7EE007AB4EEC76AF1EE10FADD
:10AEF80088BFB0EE476AB5EEC06AF1EE10FA76EE9A
:10AF0800876AB8BFB0EE6B6A66EE266AD9E5B74ABB
:10AF180092ED007AF0EEE76AF4EEC76AF1EE10FA05
:10AF28007FF79AA8B24A92ED007AF0EECD6AF4EE75
:10AF3800C76AF1EE10FA7FF78FA8AE4A99ED007A4A
:10AF4800D2ED006AB0EEC77AB4EEE67AF1EE10FA06
:10AF58007FF582A801220599C4F8CC1184F8C8218C
:10AF6800FFF77EB8A44BA54EB3F90620738B9A421F
:10AF78003FF704AEA24B1B78012B01F03986192B41
:10AF880001F036860E2B3FF4F9AD082B3FF4F6ADF1
:10AF98009C4B00229A60C4F80C21EFE53378002B13
:10AFA8003FF49EAED4ED5F3A94ED5E6AD4ED7A7AC2
:10AFB800954A94ED797AD2ED005A94ED5C4AD4ED35
:10AFC8005B4ADFF85C82DFF85CE2F4EEC63AF3EE47
:10AFD800046AF1EE10FA37EEA65A01F12B8098EDCB
:10AFE800026A26EE446AF0EE674AE6EE074AF4EE95
:10AFF800C54A34EEE66AF1EE10FA48BFB0EE656A6B
:10B00800012B8EED006A3FF46BAE98ED066A26EED2
:10B01800446AF0EE674AE6EE074AB4EEE45A34EEC4
:10B02800E66AF1EE10FAC8BFB0EE656A022B8EED43
:10B03800016A3FF455AE98ED0A6A26EE446AF0EECE
:10B04800674AE6EE074AF4EEC54A34EEE66AF1EEE0
:10B0580010FA48BFB0EE656A032B8EED026A3FF422
:10B068003FAE98ED0E6A26EE446AF0EE674AE6EEC9
:10B07800074AB4EEE45A34EEE66AF1EE10FAC8BFB5
:10B08800B0EE656A042B8EED036A3FF429AE98EDA5
:10B09800126A26EE446AF0EE674AE6EE074AB4EE14
:10B0A800E45A34EEE66AF1EE10FA88BFB0EE656A4B
:10B0B800052B8EED046A3FF413AE98ED166A26EE62
:10B0C800446AF0EE674AE6EE074AF4EEC54A74EEC3
:10B0D800E66AF1EE10FA48BFF0EE656A062BCEED8F
:10B0E800056A3FF4FDADD8ED1A6A66EEC46AF0EE63
:10B0F800674AE6EE874AB3EE046AB4EEE45A74EEA1
:10B10800C66AF1EE10FAC8BFF0EE656A072BCEEDFD
:10B11800066A3FF4E5ADD8ED1E6A26EEC44AE4EEB1
:10B12800077AB4EEE75A77EEC67AF1EE10FAC8BF9E
:10B13800F0EE657ACEED077AD2E50499334BD1ED7E
:10B14800017A93ED007AF0EEE77AF4EEC77AF1EE41
:10B1580010FA7EF5F7AED1ED027AF0EEE77AB4EEAA
:10B16800E77AF1EE10FA7EF7EDAED1ED037AF0EE64
:10B17800E77AB4EEE77AF1EE10FA7EF7E3AE244B05
:10B188001B689A077FF5DCAD2249234BB3F90C20E5
:10B19800B1F900E02148AEEB020E00688EEAEE72CB
:10B1A800A2EBEE728242BEF6CDAEB3F90E30B1F923
:10B1B8000220D21A82EAE273A3EBE27398427EF786
:10B1C800C1AEBDE50B4B99ED007AD3ED006AB0EE48
:10B1D800C77AB4EEE67AF1EE10FA7EF753AFFEF7CF
:10B1E8004EBF00BF907C0020987C0020C47C0020CB
:10B1F800C07C0020C87C0020684300200C50002040
:10B20800A834002024460020302C0020BC7C0020DC
:10B21800A04300205041002034780020B87C002052
:10B22800542C00201C33002007EE103A524BDFF854
:10B2380054811B78C4F89871B8EEC77AF7EE006AA3
:10B24800132B86EE879AB8F90400B4F89C7195ED33
:10B25800080A01F0AC83494B494A93ED001A93ED73
:10B26800053A93ED122A93ED176AD3ED091A93ED77
:10B278000E4AD3ED015AD3ED063A93ED0A7A93EDCF
:10B288000F5AD3ED132AD3ED186AD3ED044AD3ED40
:10B29800030A67EE897A69EE288A29EE088AA1EE00
:10B2A800273A02EB87060021A2EE286AC4F88C111F
:10B2B800C4F89011A1EE884AE5EEA73AA7EE085A1D
:10B2C80093ED167AD3ED0D5A93ED021AD3ED0C1ABD
:10B2D80086ED003AE2EEA86A64EEC34A27EE467AA3
:10B2E80093ED0B2AD3ED152A86ED204AE0EEC33AFA
:10B2F80065EEC45A93ED143AC3ED053AE1EE274AD8
:10B30800F0EE477AA1EEC45AE2EE085AE2EEC66AB7
:10B31800E3EE287AC3ED064A83ED0E5AC3ED0F5AC1
:10B3280086ED406AC3ED176AC3ED187AC4F8941124
:10B338007B1C03F01F03A4F89C31A8F80400FEF757
:10B34800A3BBB0EE465AFEF72FBF20F0FFFDCCE4BA
:10B3580025F09EF82AF81700FEF7A4BC96ED007AAF
:10B3680005EB4702B8EEC78A928F2AF8172028EE15
:10B37800278AFEF775BC00BFFC450020A8370020CF
:10B388002435002000460020A4F848319946002AB8
:10B3980000F07281D94B0221D94ADFEDDA6A1068D0
:10B3A800D94A90F802C092F800E0027807EE902A95
:10B3B800F8EEE77AB0EE007A67EEA67AF4EEC77A8E
:10B3C800F1EE10FA40F33A8337EEC77ADFEDCF6A31
:10B3D800B0EE676AA7EE266AB0EE467A9FEDCC6AB1
:10B3E800D3ED006A66EE866AB0EEE66AC4ED5B6A83
:10B3F80084ED5E6ABCF1000F13D005EE90CAB8EE7A
:10B40800E55ADFEDC05A66EEA64A25EE255AF7EE54
:10B41800005A75EEC55A64EE864AE4EE855A66EE21
:10B42800A56ADFEDBC5A427927EE257A27EE267AFF
:10B43800CAB1DFEDB46ADFEDB85A26EE266A06EE29
:10B44800902AF8EEE66A26EE266AB4EEE56AF1EE90
:10B4580010FA00F3A785F7EE005A35EEC66AC5EE76
:10B46800866A27EE267ABEF10C0F9FEDAC8ADFEDD7
:10B47800AC6A00F04885B4EEC87AF1EE10FA98BFCD
:10B48800B0EE478AB4EEE68AF1EE10FAB8BFB0EE35
:10B49800668A84ED418A002900F0E280B0EE007AE5
:10B4A800F4EEC77AF1EE10FA05DD37EEC77ADFED74
:10B4B800976AE7EE267A93ED017ADFED956A27EE33
:10B4C800267AB0EEC76A84ED5C7A84ED5F6ABCF1D7
:10B4D800000F13D006EE90CADFED8A5AF8EEE66A3E
:10B4E80027EE075A66EEA56AF7EE005A75EEE65A99
:10B4F80025EE065AE5EE265A27EE257ADFED856A0F
:10B50800827967EEA67A67EE877AAAB107EE102AE3
:10B51800B8EEC77ADFED7B5ADFED7F6A27EE067A51
:10B5280027EE257AB4EEE67AF1EE10FA40F33E857E
:10B53800DFED7C6A67EEA67ABEF10C0F00F0C284DC
:10B54800DFED766A9FED767AF4EEE67AF1EE10FAA0
:10B5580088BFF0EE667AF4EEC77AF1EE10FAB8BF5B
:10B56800F0EE477A0129C4ED427A79DD4278DFEDC1
:10B57800656A07EE902AF8EEE77AB0EE007A67EE91
:10B58800A67A427AF4EEC77AF1EE10FA05DD37EEC4
:10B59800C77ADFED5E6AE7EE267A93ED027ADFED91
:10B5A8005C6A27EE267AB0EEC76A84ED5D7A84ED90
:10B5B800606A9AB106EE902ADFED525AF8EEE66A12
:10B5C80027EE075A66EEA56AF7EE005A75EEE65AB8
:10B5D80025EE065AE6EE855A27EE257ADFED4D6A06
:10B5E800C37967EEA67A67EE877A0BB307EE103A4F
:10B5F800B8EEC77ADFED435ADFED476A27EE067AE1
:10B6080027EE257AB4EEE67AF1EE10FA0CDCB5EE08
:10B61800C07AF1EE10FA01F1F282B7EE006A36EE66
:10B62800477AC6EE076A01E0DFED3E6A67EEA67A62
:10B63800BEF10C0F00F03C84DFED386A9FED387ADC
:10B64800F4EEE67AF1EE10FA88BFF0EE667AF4EEE0
:10B65800C77AF1EE10FAB8BFF0EE477AC4ED437A34
:10B66800BEF1090F00F0078496F82160002E40F023
:10B678009E83002384F8183114F0F2F9002840F072
:10B688008681294B1B7823B9284B9B78002B41F0E6
:10B69800DA821D4B1B78072B00F052840022072BFF
:10B6A80084F800217EF49DA9F5F71AFB0290FEF7B5
:10B6B8009AB91F4B1F4C1A681F4BDFF8888094F803
:10B6C8000001D2691B88A8F80020A8F802300028D9
:10B6D8007FF445AA0290194DFEF785B9DFED186A87
:10B6E800FFF7FDB941023EF563AFFEF765BFF5F719
:10B6F800F7FA144B401BD880FFF713BB24460020F1
:10B70800FC3800200AD7233CFC450020D7A3684119
:10B718006F12033B00004843A4707D3F00C0F9440A
:10B7280000C0F9C40000C8422C3B00204043002060
:10B7380060450020C41E0020722E0020047E0020D8
:10B748000000000000460020F5F7CAFABD4B079A32
:10B758001B78DFF80C83801A012BA8F8020000F090
:10B768001083072B7EF4B6ACF5F7BAFA0546FEF758
:10B77800B2BCDFF8F082BCF1000F41F02D8498EDE7
:10B78800007ADDED086ADFF8E0E225EE877AA6EEBA
:10B79800867AF0EE676AE7EE056ABDEEE67A17EE9E
:10B7A800107A17EE100A9F42A8BF1846B942C8BFC0
:10B7B800084607EE100AB8EEC77A012A8EED007A1D
:10B7C8003FF489AA98ED047ADDED096A25EE877AB7
:10B7D800A6EE867AF0EE676AE7EE056ABDEEE67ACF
:10B7E80017EE107A17EE100A9F42A8BF1846B94202
:10B7F800C8BF084607EE100AB8EEC77A022A8EEDCF
:10B80800017A3FF468AA98ED087ADDED0A6A25EE18
:10B81800877AA6EE867AF0EE676AE7EE056ABDEEED
:10B82800E67A17EE107A17EE100A9F42A8BF18465C
:10B83800B942C8BF084607EE100AB8EEC77A032A0D
:10B848008EED027A3FF447AA98ED0C7ADDED0B6A8B
:10B8580025EE877AA6EE867AF0EE676AE7EE056A45
:10B86800BDEEE67A17EE107A17EE100A9F42A8BFCF
:10B878001846B942C8BF084607EE100AB8EEC77A9C
:10B88800042A8EED037A3FF426AA98ED107ADDEDAE
:10B898000C6A25EE877AA6EE867AF0EE676AE7EEFE
:10B8A800056ABDEEE67A17EE107A17EE100A9F4287
:10B8B800A8BF1846B942C8BF084607EE100AB8EE36
:10B8C800C77A052A8EED047A3FF405AA98ED147A12
:10B8D800DDED0D6A25EE877AA6EE867AF0EE676AC8
:10B8E800E7EE056ABDEEE67A17EE107A17EE100A53
:10B8F8009F42A8BF1846B942C8BF084607EE100ABB
:10B90800B8EEC77A062A8EED057A3FF4E4A998EDD9
:10B91800187ADDED0E6A25EE877AA6EE867AF0EEC5
:10B92800676AE7EE056ABDEEE67A17EE107A17EE5B
:10B93800100A9F42A8BF1846B942C8BF084607EE7A
:10B94800100AB8EEC77A072A8EED067A3FF4C3A923
:10B9580098ED1C7ADDED0F6A65EE875AE6EE265AF9
:10B96800E5EE257AFDEEE77A17EE900A8342A8BF46
:10B9780003468142C8BF0B4607EE903AF8EEE77AD5
:10B98800CEED077A002A7FF4A6A9FFF7A9B92E4EB3
:10B9980014F0A8FC7378022B01F0C981032B7FF403
:10B9A80070AE41F2B813F35C002B42F0F18041F223
:10B9B800A403F35C002B42F0E68041F2E803F35C59
:10B9C800002B42F0EA8041F22C13F35C002B3FF489
:10B9D80058AE1E481AF034F853E61D4B5A79002A1F
:10B9E8003EF469AC1B4A1278002A3EF464AC1B781A
:10B9F800DFED194A07EE903A184BB8EE677A1B88C4
:10BA080007EE902A06EE903AF8EEE77AF8EE666AC4
:10BA180067EE277AB7EE007AC7EEA63AF4EEE43A74
:10BA2800F1EE10FA88BFF0EE643AF4EEC73AF1EEA0
:10BA380010FAB8BFF0EE473AFEF73FBCB0EE677AAF
:10BA4800CCE400BFFC450020CC590020F86A002057
:10BA58003043002022460020713DAA3F0C460020BA
:10BA680000460020542C00201C330020B8F1000FA1
:10BA780000F09983DFF8B085BCF1000F41F03487FE
:10BA8800BAF1000F41F08F85D8ED006ADDED084A64
:10BA9800DFF898E565EEA66ABDEEC77A17EE101ACC
:10BAA800B0EE667AA4EE867AF0EE676AE7EE056A8B
:10BAB800BDEEE67A17EE107A17EE100A9F42A8BF7D
:10BAC8001846B942C8BF084607EE100AB8EEC77A4A
:10BAD800012A8EED007A3FF4FEA898ED047ADDED98
:10BAE800096A25EE877AA6EE867AF0EE676AE7EEAF
:10BAF800056ABDEEE67A17EE107A17EE100A9F4235
:10BB0800A8BF18468F42B8BF084607EE100AB8EE1D
:10BB1800C77A022A8EED017A3FF4DDA898ED087AFB
:10BB2800DDED0A6A25EE877AA6EE867AF0EE676A78
:10BB3800E7EE056ABDEEE67A17EE107A17EE100A00
:10BB48009F42A8BF18468F42B8BF084607EE100AA2
:10BB5800B8EEC77A032A8EED027A3FF4BCA898EDB6
:10BB68000C7ADDED0B6A25EE877AA6EE867AF0EE82
:10BB7800676AE7EE056ABDEEE67A17EE107A17EE09
:10BB8800100A9F42A8BF18468F42B8BF084607EE62
:10BB9800100AB8EEC77A042A8EED037A3FF49BA800
:10BBA80098ED107ADDED0C6A25EE877AA6EE867A96
:10BBB800F0EE676AE7EE056ABDEEE67A17EE107AF0
:10BBC80017EE100A9F42A8BF18468F42B8BF084612
:10BBD80007EE100AB8EEC77A052A8EED047A3FF40C
:10BBE8007AA898ED147ADDED0D6A25EE877AA6EE2F
:10BBF800867AF0EE676AE7EE056ABDEEE67A17EE3A
:10BC0800107A17EE100A9F42A8BF18468F42B8BF95
:10BC1800084607EE100AB8EEC77A062A8EED057AAE
:10BC28003FF459A898ED187ADDED0E6A25EE877A6B
:10BC3800A6EE867AF0EE676AE7EE056ABDEEE67A6A
:10BC480017EE107A17EE100A9F42A8BF18468F42C7
:10BC5800B8BF084607EE100AB8EEC77A072A8EED75
:10BC6800067A3FF438A898ED1C7ADDED0F6A65EE88
:10BC7800875AE6EE265AE5EE257AFDEEE77A17EEC4
:10BC8800900A8342A8BF03468142D8BF194607EEEF
:10BC9800901AF8EEE77ACEED077A002A7FF41BA80F
:10BCA800FFF71EB8C84B93ED006AFEF7FABEAB6803
:10BCB800002B3EF45DAF05F1500128469847FEF78A
:10BCC80057BFC24BC249D3F8EC30086844F620612C
:10BCD8008B42A8BF0B46B3F57A7FB8BF4FF47A738F
:10BCE80099B2C006A4F81A11DBF8003041F17D8240
:10BCF800DB0440F16D83B74BD3F800C0BCF832E0E9
:10BD08004FEA5E0EB44BB548D3ED037AD4F81C3134
:10BD1800A0FB01018809642191FBF0F11429BDEE13
:10BD2800E77A04EB4308A8BF142101338B42C4F817
:10BD38001C3117EE109AA4BF0023C4F81C3104EB81
:10BD48004303A8F82091B3F9203107EE103AB8EE72
:10BD5800C77A77EEC77AFDEEE77ACDED027ABDF9BC
:10BD6800081081EAE173A3EBE173734502F33680AF
:10BD78009B4B19464FF07E530B60FEF70CBFDFF864
:10BD8800B082F4F7ADFF974AD4F8DC311268C4F8F2
:10BD9800DC01C31A9A1A0546A8F80430A8F8062048
:10BDA800FEF799B9F4F79CFF0790FDF7A6BF1E218F
:10BDB8008748F7F74DFB00283FF45BAC8A4B1B889C
:10BDC80058063FF556AC94F88431B34242F03E80B1
:10BDD800834BD4ED627A93ED010AD4ED435A9FED7B
:10BDE800836ADFED836A27EEE57A68EE277AA8EEA4
:10BDF800007AE5EE807AB4EEC67AF1EE10FA88BFE2
:10BE0800B0EE467AB4EEE67AF1EE10FAF4EEC67ABF
:10BE1800B8BFB0EE667AF1EE10FA88BFF0EE467A57
:10BE2800F4EEE67AF1EE10FAB8BFF0EE667A84ED39
:10BE3800417AC4ED437A1CE4B4F8EC11914240F223
:10BE480085856C496C4AD1ED007A92ED007A6B4990
:10BE5800C4ED7C7A77EE676AC4ED7A7A0122C4ED84
:10BE6800796A84ED7D7AD1ED006ADFED657A84F830
:10BE7800F821FEF760B9FDEEC87ADFF8B48117EE55
:10BE8800903AA8F80490A8F80630FFF7EDBB5D4B90
:10BE98001B88002B40F079855B4A5C4B1178186849
:10BEA800F6F7C2F9D4F8CC21059B9A1AFEF719B80F
:10BEB800BDEEE77ADFF8788117EE103AA8F804307B
:10BEC800FFF7BABB9FED497ADFED496ADFF8608179
:10BED800F4EEC77AF1EE10FA98BFB0EE677AFDEE8D
:10BEE800E77AB4EEE67AF1EE10FA17EE902AB8BFC8
:10BEF800B0EE667A012984ED427AA8F802203FF76D
:10BF080035ABFFF7B1BBB4EEC87AF1EE10FA98BFC3
:10BF1800B0EE478ABDEEC77AB4EEE68ADFF8108144
:10BF2800F1EE10FA17EE102AB8BFB0EE668A84ED6B
:10BF3800418AA8F8002000297FF4B0AAFFF794BB33
:10BF4800F4F7CEFEDFF8E880314BC01B1B78A8F869
:10BF58000400FFF7A3BB2F4A2F49D2ED006A2F4AEE
:10BF680091ED006A1278C4ED7C6A84ED7D6A002A3E
:10BF780040F0E88476EEC65AF0EE466ABCEEC76A30
:10BF88002749C4ED795A16EE102AC4ED7A6AA4F846
:10BF9800EC21FF22D1ED006A84F8F82177EEC77A08
:10BFA800FEF7C9B8DFED1F6AFFF75BBAB5EEC07AD6
:10BFB800F1EE10FA00F12786B7EE006A36EE477AFE
:10BFC800C6EE076AFFF7B6BA907C00201802002078
:10BFD800984300207041002024460020D34D621071
:10BFE80090000020903400204C41002000C0F9440B
:10BFF80000C0F9C4D42C0020D0770020F02C0020F9
:10C00800000000000071002002710020047100206F
:10C01800FC450020CC770020D82C0020484B00207D
:10C02800EC2C00200000C842542C00201C330020B7
:10C038000046002098ED016A26EE646AB0EE674A71
:10C04800A6EE074AB4EEC45A34EE666AF1EE10FA68
:10C05800C8BFB0EE656A012B8EED006A3EF440AEB3
:10C0680098ED056A26EE646AB0EE674AA6EE074ABE
:10C07800B4EEC45A34EE666AF1EE10FAC8BFB0EEF8
:10C08800656A022B8EED016A3EF42AAE98ED096AC4
:10C0980026EE646AB0EE674AA6EE074AB4EEC45AC2
:10C0A80034EE666AF1EE10FAC8BFB0EE656A032B8B
:10C0B8008EED026A3EF414AE98ED0D6A26EE646ABF
:10C0C800B0EE674AA6EE074AB4EEC45A34EE666A82
:10C0D800F1EE10FAC8BFB0EE656A042B8EED036A64
:10C0E8003EF4FEAD98ED116A26EE646AB0EE674A3A
:10C0F800A6EE074AB4EEC45A34EE666AF1EE10FAB8
:10C10800C8BFB0EE656A052B8EED046A3EF4E8AD53
:10C1180098ED156A26EE646AB0EE674AA6EE074AFD
:10C12800B4EEC45A74EE666AF1EE10FAC8BFF0EEC7
:10C13800656A062BCEED056A3EF4D2ADD8ED196AD4
:10C1480066EEE46AB0EE674AA6EE874AB3EE046A82
:10C15800B4EEC45A74EE466AF1EE10FAC8BFF0EEB7
:10C16800656A072BCEED066A3EF4BAADD8ED1D6AB6
:10C1780066EEE44AE4EE877AF4EEC57A77EEC67A9C
:10C18800F1EE10FAB8BFF0EE657ACEED077AFEF759
:10C19800A7BD96F82030C3EB431103EB8103DB0006
:10C1A8009BB2FEF704BDDFF8D885BAF1000F41F065
:10C1B8008F80D8ED006ADDED084ADFF8C8E565EE46
:10C1C800A66ABDEEC77A17EE101AB0EE667AA4EE2C
:10C1D800867AF0EE676AE7EE056ABDEEE67A17EE54
:10C1E800107A17EE100A9F42A8BF1846B942C8BF76
:10C1F800084607EE100AB8EEC77A012A8EED007AD3
:10C208003EF432AB98ED047ADDED096A25EE877AC3
:10C21800A6EE867AF0EE676AE7EE056ABDEEE67A84
:10C2280017EE107A17EE100A9F42A8BF18468F42E1
:10C23800B8BF084607EE100AB8EEC77A022A8EED94
:10C24800017A3EF411AB98ED087ADDED0A6A25EE25
:10C25800877AA6EE867AF0EE676AE7EE056ABDEEA3
:10C26800E67A17EE107A17EE100A9F42A8BF184612
:10C278008F42B8BF084607EE100AB8EEC77A032AFD
:10C288008EED027A3EF4F0AA98ED0C7ADDED0B6A99
:10C2980025EE877AA6EE867AF0EE676AE7EE056AFB
:10C2A800BDEEE67A17EE107A17EE100A9F42A8BF85
:10C2B80018468F42B8BF084607EE100AB8EEC77A8C
:10C2C800042A8EED037A3EF4CFAA98ED107ADDEDBC
:10C2D8000C6A25EE877AA6EE867AF0EE676AE7EEB4
:10C2E800056ABDEEE67A17EE107A17EE100A9F423D
:10C2F800A8BF18468F42B8BF084607EE100AB8EE26
:10C30800C77A052A8EED047A3EF4AEAA98ED147A1F
:10C31800DDED0D6A25EE877AA6EE867AF0EE676A7D
:10C32800E7EE056ABDEEE67A17EE107A17EE100A08
:10C338009F42A8BF18468F42B8BF084607EE100AAA
:10C34800B8EEC77A062A8EED057A3EF48DAA98EDE6
:10C35800187ADDED0E6A25EE877AA6EE867AF0EE7B
:10C36800676AE7EE056ABDEEE67A17EE107A17EE11
:10C37800100A9F42A8BF18468F42B8BF084607EE6A
:10C38800100AB8EEC77A072A8EED067A3EF46CAA30
:10C3980098ED1C7ADDED0F6A65EE875AE6EE265AAF
:10C3A800E5EE257AFDEEE77A17EE900A8342A8BFFC
:10C3B80003468142D8BF194607EE901AF8EEE77A8D
:10C3C800CEED077ABCF1000F7EF48AACFEF750BAC6
:10C3D800DF4BD3F800C0BCF932E093E4DFF8A89350
:10C3E800D4ED017A94ED006AB9F80000D9F8143058
:10C3F80077EEA77AF0EE006AB0EE677AA6EE267AB4
:10C40800013804EBC002D6EE267A083A1033F6EE6D
:10C41800003A27EE237A67EEA37A84ED207AC4EDFA
:10C42800217ACC4CA64604F1800192ED027A92ED75
:10C43800036ADEED036ADEED027A53ED014A13ED7D
:10C44800025A37EE674A76EEC65A77EE277AE4EE56
:10C45800845A0138A2F10802E5EE047A0EF1080EBA
:10C4680003F1080336EE267A01F10801E4EE877A33
:10C47800E5EE475A67EEA37A25EEA37AC1ED007A76
:10C4880081ED017AD1D1142F7DF4B9ABF4F728FCF2
:10C49800039BDFF8F882C01AA8F80200D4F8A0615C
:10C4A800FDF7ADBBD4F8A481B4F89CA1AA4BCAF19E
:10C4B80020095FFA89F90AEB481E03EB8E0E5FEA42
:10C4C800990301F0988501331801A449A44A0EEB99
:10C4D800000C0EF1100313ED024A13ED035A13ED8D
:10C4E800016A13ED047A51ED024A51ED035A51EDF8
:10C4F800016A51ED047A64EE244A65EE255A66EE27
:10C50800266A67EE277A10339C4542ED024A42EDCF
:10C51800035A42ED016A42ED047A01F1100102F179
:10C528001002D8D18F49A0F11002964401EB020CF9
:10C53800224419F0030309D0BEEC017AFCEC017A1D
:10C5480067EE277A013BE2EC017AF5D1BAF1000FE8
:10C5580041F06881142F7DF452ABF4F7C1FB039BC3
:10C56800DFF82882D4F8A061C01AA8F80200FDF705
:10C5780046BBD4F8A4917C4B7C4ADFED7D7AD2EDA2
:10C58800008A7C4A4FEAC9010B44F8EE688A9B8806
:10C5980009EE103A643BC82BA8BFC82368EEA78AE7
:10C5A800F8EE497A782BB8BF782368EEA78A07EEA9
:10C5B800903A4944B0EE680A02EB8108B8EEE78A7F
:10C5C80023F0B2FFB8EEC99AF0EE409AB0EE680ACE
:10C5D80023F00CFF38EE097A79EE487A28EE098ABA
:10C5E80067EE877AB7EE006A88EE277A142FF8EE9E
:10C5F800007A77EE076A60EE277A89EEA67A77EEF8
:10C60800065A36EE477AC6EE256A67EEA67A27EE10
:10C61800267AC8ED006A88ED047AC8ED026AC8ED8A
:10C62800017AC8ED037A01F04586534B534A09F164
:10C63800010983FB0938A8EBE97808EB48080136BB
:10C64800A9EB08081778C4F8A061C4F8A4812BE7FF
:10C65800DFF834913F48D9F80820B9F80C1022F0D7
:10C668007DFE464B1F78142F01F00886D4F8A06190
:10C678000136C4F8A061B3E6DFF8149199F80020F8
:10C68800900801F0CC86DFF80CC100F101084FEAF0
:10C6980048180CEB080E0CF12003ACF1700113EDF7
:10C6A800076A53ED056A13ED037A53ED017A53EDEA
:10C6B800025A13ED084A53ED064A13ED045A26EEC2
:10C6C800066A66EEA66A27EE077A67EEA77AA4EEF0
:10C6D800046A20339E45E4EEA46A01F11001A5EE38
:10C6E800057AE5EEA57AF1EEC65AB1EEE66AF1EE04
:10C6F800C76AB1EEE77A41ED085A01ED076A41EDE4
:10C70800066A01ED057ACAD1A8F12008C44404EBF1
:10C71800001012F0030318BF0CF1080C0FD05CEDE9
:10C72800017A1CED027A67EEA77A013BE7EE077AF9
:10C738000CF1080CB1EEE77AA0EC017AEFD1142FD6
:10C7480001F0A8850136C4F8A061FDF7C1B900BFA2
:10C7580070410020C41E002024350020B43600207B
:10C76800D41E0020A436002024370020684E002064
:10C7780027D4D2361C80002056555555FC4500203C
:10C78800542C00201C3300200C35002000460020CB
:10C7980006350020441F0020DFF83C93B9F800E07C
:10C7A800D9F804C04FEA5E084FEA880204EB8E0607
:10C7B8005FEADE0E04EB020300F0A08010320EF1F7
:10C7C800010EBA4803EB0E1E324410330CF1100769
:10C7D80006F1100151ED032A51ED043A10ED043A27
:10C7E80010ED032A51ED026A11ED016A10ED020AFB
:10C7F80010ED018A12ED044A12ED035A53ED044A72
:10C8080053ED035A13ED027A53ED017A52ED020A01
:10C8180012ED011A73EE238A72EE221A40ED048A91
:10C8280040ED031A70EE268A78EE061A40ED028A69
:10C8380040ED011A74EE848A75EE851A43ED048A78
:10C8480043ED031A77EE208A77EE811A43ED028AC8
:10C8580043ED011A73EE633A75EE655A17ED035A04
:10C8680032EE623A74EE644A65EE631A17ED044AD2
:10C8780023EE052A64EE652AE3EE041A10339E457A
:10C8880024EE843AA3EE842A00F1100007F1100781
:10C89800A5EE853A01F1100102F11002E4EE852AB5
:10C8A80041ED071A01ED082A02ED073A42ED082A80
:10C8B80057ED055A17ED065A70EE666A38EE466A65
:10C8C80030EEC77A71EE677A26EE253A65EEE63ADB
:10C8D80025EE674A67EE054AE6EE053AA6EE853A82
:10C8E800A7EE254AE7EEA54A01ED063A41ED053ADD
:10C8F80002ED064A42ED054A7FF46CAF1FFA88F84C
:10C90800624641466A481AF0F7F84146D9F80420C9
:10C9180030461AF0F1F8674B1B78142B7FF4BEAD44
:10C92800B4E5F4F7DDF9634B03901F78142F05BFC6
:10C93800DFF8A881D4F8A061D4F8A061A8F8006055
:10C94800FDF7ABB876EE665AFFF718BB5A4A5B4953
:10C95800D2ED007A5A4A91ED007A1278C4ED7C7AC9
:10C9680084ED7D7A002A01F0338277EE676A5549B3
:10C97800C4ED7A7AC4ED796AFF22D1ED006ADFED61
:10C98800597A84F8F821FDF7D6BB4F494B69002B3B
:10C998003DF4A7AA4D484E4B008893FBF0F00B6876
:10C9A8004FF0010E186081F811E0FDF79ABA494E70
:10C9B800DFF82C9196ED004A96ED057AD6ED014AFE
:10C9C80096ED066AD6ED046A96ED035AD6ED025A3C
:10C9D80067EE897A09EB8703A4EE277AA4EEA76AA3
:10C9E80066EEC76AA5EE476AE5EEA76A20EE070A73
:10C9F80086ED056AC6ED066A83ED007A29EE088A97
:10CA080023F046FD69EE288AD6ED0E5AD6ED176A50
:10CA180096ED091AD6ED121A96ED0F5A96ED187A78
:10CA280096ED0A2AD6ED132A96ED0D6AD6ED167AFA
:10CA380096ED0C3AD6ED0B3A96ED154AD6ED144A1A
:10CA4800E1EE085A002209EB8703E8EEA16A00B27A
:10CA5800C4F88C21A2EE085AC4F89021C4F8942195
:10CA6800A8EEA27A26EE656A67EEE67AA3EE655A24
:10CA7800A3EE886AA6EEC47AE8EEA47A86ED0E5A8A
:10CA8800C3ED205A86ED0F6AC3ED406A86ED177A2A
:10CA9800C6ED187AFEF74CBC0B494A69002A3DF4EA
:10CAA80051AA0A6813604B74FDF74CBAD41E0020D3
:10CAB800C41E0020FC450020CC770020D82C002084
:10CAC800484B0020EC2C0020087100202071002029
:10CAD80020A10700A83700200C35002000460020C0
:10CAE8002435002000000000B5F93C306A6207EEEA
:10CAF800903A0122F8EEE77AEB66C5F88820002321
:10CB0800012FC5ED1F7AC5ED1E7AC5F8803001F0FA
:10CB18008781B7427DF400AFB5F93E302B6707EE49
:10CB2800903A00220123F8EEE77AAA62C5F89C3011
:10CB38000023012FC5ED247AC5ED237AC5F894307A
:10CB480001F07281B7427DF417AFB5F940306B67D9
:10CB580007EE903A00220123F8EEE77AEA62C5F878
:10CB6800B0300023012FC5ED297AC5ED287AC5F824
:10CB7800A8307DF431AF1FED258AB9F1030F46D0F7
:10CB8800BAF1000F09D007EE90AAF8EEE77AF4EEB2
:10CB9800C87AF1EE10FA01F14784C34A6B6F126844
:10CBA80094F8A811A8F8060003EB560393FBF6F6D1
:10CBB8000023EE6293621363D36231B1BB4B1B88CF
:10CBC80023F40063002B7DF409AFB94B1B6813F401
:10CBD800003341F01D81B7491A46C85C012803F1AA
:10CBE8000C0300F0BB840132152AF6D1FDF7F6BE1E
:10CBF800B14B9B7B002B3EF4CBA9FDF7BFBFF7EEF3
:10CC0800006AFEF713BDF7EE006AFEF793BCB0EEBC
:10CC1800480A23F03DFC00B2B2E7B4F8489109F1A4
:10CC2800FF390FFA89F9B9F1000FA4F848917EF796
:10CC3800AEABA24BFEF70FB8B4F81A3103F57A730E
:10CC48009BB2FDF7B4BF05981CF006FBFEF721BDAB
:10CC58009B4ADFED9C7A92ED080A0293B4EEE70A4C
:10CC6800F1EE10FA40F2348623F0A8FCD4ED457AB0
:10CC780020EE270A23F00CFCB0F5617F029B00F33D
:10CC8800688707EE900AF8EEE76ADFED8F7A66EEBE
:10CC9800A76A07EE903AB8EEE77AFDEEE67A17EE65
:10CCA800903A2033402B41F213839FED880A23F0FA
:10CCB800EFFB00B207EE900AB8EEE77A7F4BD3EDB0
:10CCC800037A77EE877AC3ED037AFDF75FBF804B6F
:10CCD80093F800C00CF0010CBCF1000F7EF400A822
:10CCE800FDF7C6BD7B4BDFED7C7A1F68C4ED6E7A1D
:10CCF80017F0805740F04A8410F4800700F0D6827D
:10CD08000027B6EE007A67EE877AF4EEE57AF1EE60
:10CD180010FAC8BFF0EE675A40F33884C4ED7F5A62
:10CD2800FDF74ABCF3F7DCFF0746FDF719BFB378F8
:10CD3800072B3EF6A6ACDFE813F0580017010B01ED
:10CD480071007C0042004C00080003237370FEF75A
:10CD580098BC33690622652BB2703AD93278032A17
:10CD680014BF6FF0FF026FF07F02A3F1650303EABF
:10CD7800020303F1010314BF4FF4807280229A4228
:10CD8800336126D2D8F80020D6F80C80023203EBA3
:10CD98000809914502D31EF0DDF833694F4AC6F8F9
:10CDA8000480D16FC6F80890490203FB01F30521FE
:10CDB800C2F8008042F81C3C42F8183CB170B268D6
:10CDC800474901201EF058FE012841F045850623F9
:10CDD800B370002143481EF0F3F9012841F03C8567
:10CDE800B3780133DBB2B370A2E700230DF1200959
:10CDF80049461846092212F00FFC01287EF441AC7E
:10CE0800089B93F8FE21552A01F0C68241F2B4121C
:10CE180002210123B1547370FEF733BC41F2701341
:10CE2800F35C002B3EF42DAC2E4818F009FEFEF7FB
:10CE380028BC3278337DDFF8B880DFF8A4A0032A55
:10CE480014BF4FF480794FF08009002B6BD0012B71
:10CE5800FBD1254B72681968D8F8000000234FEA07
:10CE6800412E4FF0FF31B1FBFEF112EB010B43F104
:10CE7800000C0021614500F1020008BF58455A46E0
:10CE88001A4938BF0246022012F006FD032801F2B3
:10CE9800638201A353F820F08BB60008FDCE00088A
:10CEA8008BB60008FDCE000860450020A443002092
:10CEB800FC2A0020A02E03085C48002024460020FD
:10CEC800882A00208FC2753CD06D393A00000000D6
:10CED8009C4500209843002000000080606B0020E3
:10CEE800D05900203C6B0020DC6B0020D459002076
:10CEF800D46B00207268D6F808E03369AEEB020103
:10CF0800994284BFF260316103283FF422AF0EF1E9
:10CF18000103B3FBF9F209FB12320AB14B449B1A25
:10CF2800002273603275D8F8002051460232002082
:10CF380012F0B2FC032801F20F8201A353F820F08B
:10CF48008BB60008AFCF00088BB600085BCD000891
:10CF5800DB4B00930320B07030230522D949DA480F
:10CF68001EF0F8FCFEF78DBB0DF1200941F2FC180C
:10CF7800494656F808000023092212F04DFB012803
:10CF88007EF47FAB0023089A3370B2F80B30B3F508
:10CF9800007F01F0B78241F2B41203210123B1549A
:10CFA8007370FEF76EBB73684FF001020133327580
:10CFB800B3604EE774EE677AB7EE007AF4EEC77A9C
:10CFC800F1EE10FAC4ED6E7A40F3178784EEA77A73
:10CFD8008DED087AFDF7E6BABEF1000F00F0E285A4
:10CFE80098ED007ADDED086ADFF8E0E225EE877A51
:10CFF800A6EE867AF0EE676AE7EE056ABDEEE67A97
:10D0080017EE107A17EE100A9F42A8BF1846B942C9
:10D01800C8BF084607EE100AB8EEC77A012A8EED97
:10D02800007A3DF45DAE98ED047ADDED096A25EEEF
:10D03800877AA6EE867AF0EE676AE7EE056ABDEEB5
:10D04800E67A17EE107A17EE100A9F42A8BF184624
:10D05800B942C8BF084607EE100AB8EEC77A022AD6
:10D068008EED017A3DF43CAE98ED087ADDED0A6A62
:10D0780025EE877AA6EE867AF0EE676AE7EE056A0D
:10D08800BDEEE67A17EE107A17EE100A9F42A8BF97
:10D098001846B942C8BF084607EE100AB8EEC77A64
:10D0A800032A8EED027A3DF41BAE98ED0C7ADDED85
:10D0B8000B6A25EE877AA6EE867AF0EE676AE7EEC7
:10D0C800056ABDEEE67A17EE107A17EE100A9F424F
:10D0D800A8BF1846B942C8BF084607EE100AB8EEFE
:10D0E800C77A042A8EED037A3DF4FAAD98ED107AEA
:10D0F800DDED0C6A25EE877AA6EE867AF0EE676A91
:10D10800E7EE056ABDEEE67A17EE107A17EE100A1A
:10D118009F42A8BF1846B942C8BF084607EE100A82
:10D12800B8EEC77A052A8EED047A3DF4D9AD98EDAC
:10D13800147ADDED0D6A25EE877AA6EE867AF0EE92
:10D14800676AE7EE056ABDEEE67A17EE107A17EE23
:10D15800100A9F42A8BF1846B942C8BF084607EE42
:10D16800100AB8EEC77A062A8EED057A3DF4B8ADF6
:10D1780098ED187ADDED0E6A25EE877AA6EE867AA6
:10D18800F0EE676AE7EE056ABDEEE67A17EE107A0A
:10D1980017EE100A9F42A8BF1846B942C8BF0846F2
:10D1A80007EE100AB8EEC77A072A8EED067A3DF424
:10D1B80097AD98ED1C7ADDED0F6A65EE875AE6EEBD
:10D1C800265AE5EE257AFDEEE77A17EE902A934285
:10D1D800A8BF13468A42A8BF194607EE901AF8EE70
:10D1E800E77ACEED077AFDF77BBDD8003EF580AD36
:10D1F800FDF7D1BC012A40F3138607EE101AB8EEEA
:10D20800C77AC7EE876AB1EEE68AB9F1030F13D081
:10D21800BAF1000F09D007EE90AAF8EEE77AF4EE1B
:10D22800C87AF1EE10FA01F1FF80EB6E03EB5603BA
:10D2380093FBF6F36B626CE4B0EE480A23F028F92E
:10D2480000B2E5E7012A40F3EF8507EE101AB8EEC1
:10D25800C77AC7EE876AB1EEE68AB9F1030F13D031
:10D26800BAF1000F09D007EE90AAF8EEE77AF4EECB
:10D27800C87AF1EE10FA01F1D7802B6F03EB560351
:10D2880093FBF6F3AB625DE4B0EE480A23F000F9D5
:10D2980000B2E5E7012A7FF76EAC07EE101AB8EE88
:10D2A800C77AC7EE876AB1EEE68A66E4B6EE007A18
:10D2B800F4EEC75AF1EE10FA3FF723ADFDF77CB94B
:10D2C80021AF0208AC5003083C6B00201C3300203F
:10D2D800D8ED004A9DED084ADFF808E665EEA44A55
:10D2E800FDEEC73AE4EE064AB0EE674AA4EE854A78
:10D2F80013EE901AF4EEC46AF1EE10FAF0EE444A16
:10D3080088BFF0EE474AFDEEE44A14EE900A14EEA8
:10D31800907A9842A8BF1F468142C8BF0F4604EEC4
:10D32800907AF8EEE44A012ACEED004A3DF49CAA30
:10D33800D8ED044A9DED094A65EEA44AE4EE064A92
:10D34800B0EE674AA4EE854AF4EEC46AF1EE10FA2C
:10D35800F0EE444A88BFF0EE474AFDEEE44A14EE88
:10D36800900A14EE907A9842A8BF1F468842B8BF28
:10D378000F4604EE907AF8EEE44A022ACEED014A0E
:10D388003DF472AAD8ED084A9DED0A4A65EEA44A12
:10D39800E4EE064AB0EE674AA4EE854AF4EEC46AA3
:10D3A800F1EE10FAF0EE444A88BFF0EE474AFDEE7F
:10D3B800E44A14EE900A14EE907A9842A8BF1F46E9
:10D3C8008842B8BF0F4604EE907AF8EEE44A032A82
:10D3D800CEED024A3DF448AAD8ED0C4A9DED0B4A21
:10D3E80065EEA44AE4EE064AB0EE674AA4EE854A22
:10D3F800F4EEC46AF1EE10FAF0EE444A88BFF0EE9B
:10D40800474AFDEEE44A14EE900A14EE907A9842E8
:10D41800A8BF1F468842B8BF0F4604EE907AF8EEC0
:10D42800E44A042ACEED034A3DF41EAAD8ED104A78
:10D438009DED0C4A65EEA44AE4EE064AB0EE674A52
:10D44800A4EE854AF4EEC46AF1EE10FAF0EE444A0E
:10D4580088BFF0EE474AFDEEE44A14EE900A14EE57
:10D46800907A9842A8BF1F468842B8BF0F4604EE7C
:10D47800907AF8EEE44A052ACEED044A3DF4F4A980
:10D48800D8ED144A9DED0D4A65EEA44AE4EE064A2D
:10D49800B0EE674AA4EE854AF4EEC46AF1EE10FADB
:10D4A800F0EE444A88BFF0EE474AFDEEE44A14EE37
:10D4B800900A14EE907A9842A8BF1F468842B8BFD7
:10D4C8000F4604EE907AF8EEE44A062ACEED054AB5
:10D4D8003DF4CAA9D8ED184A9DED0E4A65EEA44A56
:10D4E800E4EE064AB0EE674AA4EE854AF4EEC46A52
:10D4F800F1EE10FAF0EE444A88BFF0EE474AFDEE2E
:10D50800E44A14EE900A14EE907A9842A8BF1F4697
:10D518008842B8BF0F4604EE907AF8EEE44A072A2C
:10D52800CEED064A3DF4A0A9D8ED1C4A9DED0F4A60
:10D5380065EEA45AE6EE045AE5EE257AF4EEE76ABB
:10D54800F1EE10FAC8BFF0EE477AFEF72BBFDFED19
:10D55800E27AFCF70BBB8223FCF73DBBD4F8AC6145
:10D5680053003EB1981801EB800076784078B042BD
:10D57800BDF434AA134401EB83010023C4F8AC11B1
:10D58800A4F80032C4F80432FDF728BAB7EE007ADE
:10D5980077EE677AF4EEE75AF1EE10FA88BFF0EE0C
:10D5A800675AFFF7BBBBD8ED004A9DED084ADFF884
:10D5B80034E365EEA44AFDEEC73AE4EE064AB0EE5F
:10D5C800674AA4EE854A13EE901AF4EEC46AF1EEA7
:10D5D80010FAF0EE444A88BFF0EE474AFDEEE44AFE
:10D5E80014EE900A14EE907A9842A8BF1F46814222
:10D5F800C8BF0F4604EE907AF8EEE44A012ACEED51
:10D60800004A3DF468ABD8ED044A9DED094A65EE41
:10D61800A44AE4EE064AB0EE674AA4EE854AF4EE60
:10D62800C46AF1EE10FAF0EE444A88BFF0EE474AB9
:10D63800FDEEE44A14EE900A14EE907A9842A8BFE0
:10D648001F468842B8BF0F4604EE907AF8EEE44AC7
:10D65800022ACEED014A3DF43EABD8ED084A9DEDD5
:10D668000A4A65EEA44AE4EE064AB0EE674AA4EE1A
:10D67800854AF4EEC46AF1EE10FAF0EE444A88BF27
:10D68800F0EE474AFDEEE44A14EE900A14EE907A62
:10D698009842A8BF1F468842B8BF0F4604EE907A4A
:10D6A800F8EEE44A032ACEED024A3DF414ABD8ED75
:10D6B8000C4A9DED0B4A65EEA44AE4EE064AB0EE2C
:10D6C800674AA4EE854AF4EEC46AF1EE10FAF0EE69
:10D6D800444A88BFF0EE474AFDEEE44A14EE900A49
:10D6E80014EE907A9842A8BF1F468842B8BF0F46EA
:10D6F80004EE907AF8EEE44A042ACEED034A3DF4AB
:10D70800EAAAD8ED104A9DED0C4A65EEA44AE4EE6B
:10D71800064AB0EE674AA4EE854AF4EEC46AF1EE12
:10D7280010FAF0EE444A88BFF0EE474AFDEEE44AAC
:10D7380014EE900A14EE907A9842A8BF1F468842C9
:10D74800B8BF0F4604EE907AF8EEE44A052ACEED0B
:10D75800044A3DF4C0AAD8ED144A9DED0D4A65EE81
:10D76800A44AE4EE064AB0EE674AA4EE854AF4EE0F
:10D77800C46AF1EE10FAF0EE444A88BFF0EE474A68
:10D78800FDEEE44A14EE900A14EE907A9842A8BF8F
:10D798001F468842B8BF0F4604EE907AF8EEE44A76
:10D7A800062ACEED054A3DF496AAD8ED184A9DED15
:10D7B8000E4A65EEA44AE4EE064AB0EE674AA4EEC5
:10D7C800854AF4EEC46AF1EE10FAF0EE444A88BFD6
:10D7D800F0EE474AFDEEE44A14EE900A14EE907A11
:10D7E8009842A8BF1F468842B8BF0F4604EE907AF9
:10D7F800F8EEE44A072ACEED064A3DF46CAAD8EDC5
:10D808001C4A9DED0F4A65EEA45AE6EE045AE5EE71
:10D81800257AF4EEE76AF1EE10FAC8BFF0EE477A1F
:10D82800FEF72BBA2D4B4FEA890E5FEA9A0901EBF6
:10D838000E0C03EBC818A64400F0618609F1010933
:10D848004FEA091908EB090008F110030CF110015F
:10D858000EF1100213ED024A13ED035A13ED016A9B
:10D8680013ED047A51ED024A51ED035A51ED016A64
:10D8780051ED047A64EE244A65EE255A66EE266A6E
:10D8880067EE277A1033984242ED024A42ED035A76
:10D8980042ED016A42ED047A01F1100102F1100231
:10D8A800D8D1A9F11009C8440CEB0901CE441AF0EB
:10D8B800030A3EF44FAEB8EC017AF1EC017A67EE58
:10D8C800277ABAF1010AEEEC017AF4D1FEF742BEEA
:10D8D8009FED037AFFF7F2B90000024324350020D8
:10D8E800000000001C330020D8ED004A9DED084AD6
:10D8F80065EEA44AE4EE064AB0EE674AA4EE854A0D
:10D90800F0EE444ABEF1000F00F08383BAF1000F35
:10D9180006D0F4EE446AF1EE10FAC8BFF0EE474ABA
:10D92800BDEEC77A17EE10CABDEEE47A04EE90CACF
:10D9380017EE101A8C4500F3CE859942A8BF1946F8
:10D9480007EE101AB8EEC77ADFF8D8E5012A8EED8F
:10D95800007A3DF4C5A998ED047A9DED094A25EEB3
:10D96800877AA4EE067AB0EE674AA7EE054AB0EECB
:10D97800447ABAF1000F00F09D85F4EEC46AF1EE26
:10D9880010FA40F3978561469942A8BF194607EEF9
:10D99800101AB8EEC77A022A8EED017A3DF4A0A9D2
:10D9A80098ED087A9DED0A4A25EE877AA4EE067A64
:10D9B800B0EE674AA7EE054AB0EE447ABAF1000F16
:10D9C80000F06D85F4EEC46AF1EE10FA40F3678555
:10D9D80061469942A8BF194607EE101AB8EEC77AF1
:10D9E800032A8EED027A3DF47BA998ED0C7A9DED21
:10D9F8000B4A25EE877AA4EE067AB0EE674AA7EEC0
:10DA0800054AB0EE447ABAF1000F00F03D85F4EE15
:10DA1800C46AF1EE10FA40F3378561469942A8BF0F
:10DA2800194607EE101AB8EEC77A042A8EED037A63
:10DA38003DF456A998ED107A9DED0C4A25EE877AAB
:10DA4800A4EE067AB0EE674AA7EE054AB0EE447A2D
:10DA5800BAF1000F00F00D85F4EEC46AF1EE10FA89
:10DA680040F3078561469942A8BF194607EE101A88
:10DA7800B8EEC77A052A8EED047A3DF431A998EDFF
:10DA8800147A9DED0D4A25EE877AA4EE067AB0EE5B
:10DA9800674AA7EE054AB0EE447ABAF1000F00F0E3
:10DAA800DD84F4EEC46AF1EE10FA40F3D7846146DF
:10DAB8009942A8BF194607EE101AB8EEC77A062A87
:10DAC8008EED057A3DF40CA998ED187A9DED0E4A75
:10DAD80025EE877AA4EE067AB0EE674AA7EE054AE5
:10DAE800B0EE447ABAF1000F00F0AD84F4EEC46AE7
:10DAF800F1EE10FA40F3A78461469942A8BF19468F
:10DB080007EE101AB8EEC77A072A8EED067A3DF4AA
:10DB1800E7A898ED1C7A9DED0F4A65EE875AE4EE6A
:10DB2800065AE5EE857ABAF1000F00F08384F4EE28
:10DB3800E67AF1EE10FA40F17D8462469A42A8BF77
:10DB48001A4604EE902AF8EEE44ACEED074AFDF7AD
:10DB5800C7B807EE903ADFEDE06AB8EEE77A66EE0E
:10DB6800A65A9FEDDE5A9FEDDE6ADFEDDE7AA5EE5E
:10DB7800856A26EEA55AE5EE867AE5EE276A26EE50
:10DB8800870AFFF794B8D84817F05AFFFDF715BF72
:10DB9800D64817F055FFFDF70ABFD54817F050FFD4
:10DBA800FDF711BFD8ED006ADDED084A65EEA66AFB
:10DBB800E4EE866AF0EE674AE6EE854AFDEEE46A30
:10DBC80016EE90EA714500F31B829E45A8BF9E465B
:10DBD80006EE90EAF8EEE66A002F00F0B785DFF867
:10DBE80044E3012ACEED006A3DF47AA8D8ED046A30
:10DBF800DDED094A65EEA66AE4EE866AF0EE674A4C
:10DC0800E6EE854AFDEEE46A16EE90CA614500F339
:10DC1800FD819C45A8BF9C4606EE90CAF8EEE66AD0
:10DC2800002F00F06086022ACEED016A3DF458A864
:10DC3800D8ED086ADDED0A4A65EEA66AE4EE866A62
:10DC4800F0EE674AE6EE854AFDEEE46A16EE90CA03
:10DC5800614500F3D8819C45A8BF9C4606EE90CA52
:10DC6800F8EEE66A002F00F0CE85032ACEED026AB0
:10DC78003DF436A8D8ED0C6ADDED0B4A65EEA66AD0
:10DC8800E4EE866AF0EE674AE6EE854AFDEEE46A5F
:10DC980016EE90CA614500F382819C45A8BF9C4658
:10DCA80006EE90CAF8EEE66A002F00F0A185042A75
:10DCB800CEED036A3DF414A8D8ED106ADDED0C4AE8
:10DCC80065EEA66AE4EE866AF0EE674AE6EE854AF5
:10DCD800FDEEE46A16EE90CA614500F35D819C454D
:10DCE800A8BF9C4606EE90CAF8EEE66A002F00F040
:10DCF8009585052ACEED046A3CF4F2AFD8ED146A96
:10DD0800DDED0D4A65EEA66AE4EE866AF0EE674A36
:10DD1800E6EE854AFDEEE46A16EE90CA614500F328
:10DD280041819C45A8BF9C4606EE90CAF8EEE66A7B
:10DD3800002F00F08685062ACEED056A3CF4D0AFA8
:10DD4800D8ED186ADDED0E4A65EEA66AE4EE866A3D
:10DD5800F0EE674AE6EE854AFDEEE46A16EE90CAF2
:10DD6800614500F316819C45A8BF9C4606EE90CA03
:10DD7800F8EEE66A002F00F03085072ACEED066A35
:10DD88003CF4AEAFD8ED1C6ADDED0F4A65EEA65A3D
:10DD9800E4EE865AE5EE257AFDEEE77A17EE902A4C
:10DDA800914203DC9A42A8BF1A46114607EE901A20
:10DDB800F8EEE77A002F7FF414AA039B002B7FF478
:10DDC80010AA029B5B45B8BFF0EE477AFFF709BA85
:10DDD80077EEC76AF0EE477AFEF7C9BDBCF8343073
:10DDE8009FED447A07EE903AF8EEE77A424B67EEF9
:10DDF800877AC3ED007AFCF7CEBE404B1F6817F058
:10DE080080577EF47EAFFEF777BF3D4BFCF71ABF15
:10DE18003C4B1B78032B00F06E830023FEF7DBBE20
:10DE28009FED398AFFF7F1B99FED378AFFF715BAE9
:10DE38009FED360ADFF8F08025EE800A22F028FBF5
:10DE4800D4F8A061A8F80600FBF7D9BE07EE906ADF
:10DE5800F8EEE78ADFED2E7A9FED340A84F88461C4
:10DE680068EEA78A38EE800AFDEEC07A17EE903A7F
:10DE78002033402B40F229839FED230A1E4BFDEEF1
:10DE8800E87A83ED010A17EE903A2033402B00F22E
:10DE98001F83DFED277AF4EEE78AF1EE10FA40F3FC
:10DEA8004884DFED1C6ADFED1C7A01E0F0EE478A5A
:10DEB800F4EEE78AF1EE10FA38EEE67AF6DCDFEDFA
:10DEC800177AB4EEE77AF1EE10FA40F136849FED56
:10DED800116ADFED136A35E084F9223F92E741B910
:10DEE8009730083C15A82ABE706A0020846B002071
:10DEF800B46A00206F12833A9000002098430020F3
:10DF08002446002094430020000000000000C8427E
:10DF180035FA8E3CDB0FC940E4CB1641DB0F49C014
:10DF2800E4CB16C11C33002000460020DB0FC93F9C
:10DF3800DB0F494092E741B99730083C15A82ABE43
:10DF4800B0EE677AB4EEE67AF1EE10FA77EE067A7A
:10DF5800F6D41FED0A7AF4EEC77AF1EE10FA40F320
:10DF6800BE821FED0D7A77EE677A27EEA76A5FED1E
:10DF78000F5A5FED0F6A1FED0F7AE6EE256A67EE1E
:10DF8800865AA6EE267AE5EE877AC4ED627AFDF720
:10DF980024BF06EE901AEBE606EE901AA4E606EE0B
:10DFA800901A7FE606EE901AC0E693ED000A0293F7
:10DFB8000491039222F06CFADFF8CCE3DFF8CC830B
:10DFC800DEF8ECE0DFF8C8C3A8F800008CFB0E3CD4
:10DFD8004FEAEE70C0EBAC1007EE900AF8EEE77A65
:10DFE800029B039A0499FDEEE77A17EE900AA8F8C7
:10DFF8000200FCF72CBEDA49DA4A8C46FEF799BAD9
:10E0080006EE901AE6E506EE901A29E606EE901A54
:10E0180004E6BAF1000F06D0F4EE446AF1EE10FA05
:10E02800C8BFF0EE474ABDEEC74AFDEEE44A14EE1B
:10E0380010CA14EE901A8C4514EE109A00F3178348
:10E048009942A8BF194604EE901AF8EEE44A002F48
:10E0580000F01684DFF83CE3012ACEED004A3CF4D8
:10E068003FAED8ED044A9DED094A65EEA44AE4EEB8
:10E07800064AB0EE674AA4EE854AF0EE444ABAF181
:10E08800000F00F0EB82F4EEC46AF1EE10FA40F3F0
:10E09800E58261469942A8BF194604EE901AF8EE47
:10E0A800E44A002F00F0E283022ACEED014A3CF454
:10E0B80017AED8ED084A9DED0A4A65EEA44AE4EE8B
:10E0C800064AB0EE674AA4EE854AF0EE444ABAF131
:10E0D800000F00F0BA82F4EEC46AF1EE10FA40F3D1
:10E0E800B48261469942A8BF194604EE901AF8EE28
:10E0F800E44A002F00F0D983032ACEED024A3CF40B
:10E10800EFADD8ED0C4A9DED0B4A65EEA44AE4EE5E
:10E11800064AB0EE674AA4EE854AF0EE444ABAF1E0
:10E12800000F00F08982F4EEC46AF1EE10FA40F3B1
:10E13800838261469942A8BF194604EE901AF8EE08
:10E14800E44A002F00F0A783042ACEED034A3CF4EA
:10E15800C7ADD8ED104A9DED0C4A65EEA44AE4EE31
:10E16800064AB0EE674AA4EE854AF0EE444ABAF190
:10E17800000F00F05882F4EEC46AF1EE10FA40F392
:10E18800528261469942A8BF194604EE901AF8EEE9
:10E19800E44A002F00F09D83052ACEED044A3CF4A2
:10E1A8009FADD8ED144A9DED0D4A65EEA44AE4EE04
:10E1B800064AB0EE674AA4EE854AF0EE444ABAF140
:10E1C800000F00F02782F4EEC46AF1EE10FA40F373
:10E1D800218261469942A8BF194604EE901AF8EECA
:10E1E800E44A002F00F06B83062ACEED054A3CF482
:10E1F80077ADD8ED184A9DED0E4A65EEA44AE4EED7
:10E20800064AB0EE674AA4EE854AF0EE444ABAF1EF
:10E21800000F00F0F681F4EEC46AF1EE10FA40F354
:10E22800F08161469942A8BF194604EE901AF8EEAB
:10E23800E44A002F00F06283072ACEED064A3CF438
:10E248004FADD8ED1C4A9DED0F4A65EEA45AE6EE97
:10E25800045AE5EE257ABAF1000F40F0C681FDEECA
:10E26800E77A17EE902A944540F3C68107EE909A14
:10E27800F8EEE77A002F7EF4B4AF9EE5F2F730FDB2
:10E28800394BDFF808811F78039BC01AA8F80200F1
:10E29800FEF7ECB9F2F724FD334BDFF8F0801F7876
:10E2A800039B99F80020D4F8A061C01AA8F80400CC
:10E2B800FEF748BAF2F714FD039BDFF8D080D4F8D4
:10E2C800A491D4F8A061C01AA8F80200FEF7ADB96D
:10E2D800DFED267AF4EEE76AF1EE10FA40F33382C6
:10E2E800DFED235A9FED236A01E0F0EE676AF4EE52
:10E2F800C66AF1EE10FA76EEE57AF6DCDFED1E6A14
:10E30800F4EEE67AF1EE10FA40F11A82DFED185ACF
:10E318009FED1A6A01E0F0EE667AF4EEC67AF1EE45
:10E3280010FA77EEA56AF6D4DFED157AF4EEE76A0F
:10E33800F1EE10FA04DDDFED0D7A77EEE66A0EE411
:10E34800DFED107AF4EEE76AF1EE10FA44BFDFED84
:10E358000A7A77EEE66A02E4337DFEF776BD00BFFF
:10E36800A4360020C41E0020FC450020DB0F4940D5
:10E37800DB0FC940E4CB1641DB0F49C0E4CB16C123
:10E38800DB0FC93FDB0FC9BF180200200046002081
:10E39800D34D62101C33002093F8FF21AA2A7EF483
:10E3A80035ADD3F8C6214AB193F8C211A1F10B00DB
:10E3B80001282DD901F0F701062929D0D3F8D62153
:10E3C8004AB193F8D211A1F10B00012820D901F02C
:10E3D800F70106291CD0D3F8E6214AB193F8E211D7
:10E3E800A1F10B00012813D901F0F70106290FD07C
:10E3F800D3F8F621002A3EF409AD93F8F231A3F1DF
:10E408000B01012904D903F0F703062B7EF4FEACB7
:10E4180041F2FC1101237250B370FEF7A7BDD14839
:10E4280000F1800CFEF775B9A8F80600A5F8B460ED
:10E43800FCF7DCBAFDEEE77A17EE902A6245FFF6A4
:10E4480082ABFFF77BBBBDEEC77A17EE101A6145AA
:10E45800BFF653AB07EE10CAFFF754BBBDEEC77A41
:10E4680017EE101A6145BFF623AB07EE10CAFFF787
:10E4780024BBBDEEC77A17EE101A6145BFF6F3AAA2
:10E4880007EE10CAFFF7F4BABDEEC77A17EE101AF6
:10E498006145BFF6C3AA07EE10CAFFF7C4BABDEEBE
:10E4A800C77A17EE101A6145BFF693AA07EE10CA8D
:10E4B800FFF794BABDEEC77A17EE101A6145BFF69A
:10E4C80063AA07EE10CAFFF764BAF4F7E9FED5E4C9
:10E4D800DFEDA57A59E507EE10CAFFF733BA9FEDCD
:10E4E800A37AF4EEC77AF1EE10FA44BF9FEDA07A52
:10E4F80077EE677A39E519F015FDFCF76FBA6146D2
:10E50800FFF7D5B9137C022B7EF445AD92F8FE31A6
:10E51800552B7EF440AD92F8FF31AA2B7EF43BAD2B
:10E5280056F80810B2F80E80924B08EB010CC3F8AD
:10E5380000C092F80DE041F210210EF1FF337F2B5D
:10E5480046F801E03EF627ADCEF100033EEA0303AC
:10E558007EF421AD4FEA4E2341F21821013B73505E
:10E56800D08A00B9506A844941F20423F050B2F8C5
:10E5780011305B0103F2FF135B120B60B2F813104A
:10E5880001B9116A08EB030940008144A1EB0901B4
:10E5980041F2082840F6F479B1FBFEF1494546F806
:10E5A800081040F24A814FF6F47E714540F24181ED
:10E5B80003213170D26A71496344184441F20C2E28
:10E5C80041F21C23097846F80E00F25009B921F0EF
:10E5D800FFFCB3780133B370FDF753B894F8D83122
:10E5E800002B7BF46FADFBF75ABDF4EEE76AF1EE52
:10E5F80010FA7FF734AE62469A42A8BF1A4691468F
:10E6080034E6FDEEE44A14EE901A6145BFF60AAE10
:10E6180061460AE6FDEEE44A14EE901A6145BFF63B
:10E62800D9AD6146D9E5FDEEE44A14EE901A61458C
:10E63800BFF6A8AD6146A8E5FDEEE44A14EE901ACF
:10E648006145BFF677AD614677E5FDEEE44A14EE25
:10E65800901A6145BFF646AD614646E5FDEEE44ACF
:10E6680014EE901A6145BFF615AD614615E514EE36
:10E67800101AE8E4424BD3ED007AB1EE677AB4EEB3
:10E68800C7DAF1EE10FA51D4B4EEE7DAF1EE10FA87
:10E6980088BFB0EE67DA3B4BC7ED00BA1B68934200
:10E6A800BBF648ACFCF76BBD374A384B10681B68A3
:10E6B8009847069BDBED007A93ED007A344BD7ED53
:10E6C800006A83ED020A334B67EE277A2B4427EE64
:10E6D8008C7AD3ED007A304B67EE277AF0EE665AE3
:10E6E800EDEE275A93ED006AB1EE467AB4EEE57A7C
:10E6F800F1EE10FA08DCB4EEE56AF1EE10FA8CBF20
:10E70800B0EE657AB0EE467A244B1B78012B02D026
:10E71800192B7BF44EACDFED227AB4EEE7DAF1EE9A
:10E7280010FACCBF01230023FBF74EBCB0EE47DA4A
:10E73800B1E7B0EE687AFFF7C2BBF0EE477A08E4BB
:10E74800F0EE676AF0E5F0EE667AD7E50398002800
:10E758007FF445AA02985845B8BFF0EE476AFFF71C
:10E768003EBA00BFC41E002000000000DB0FC9BF76
:10E77800DB0F49C0CC6B0020EC6B0020AC6B002099
:10E78800CC7C0020B07C0020447C0020587C0020F9
:10E79800E8320020687C0020D07C00202C7A002001
:10E7A80000009642132B05D1B0EE480A21F070FE06
:10E7B800AAF80000B0EE480AD5F814325448984731
:10E7C800544B1B78132BB0EE408A7BF459AA21F0E6
:10E7D8005FFEAAF80200FBF753BA039800287FF4FB
:10E7E800CCAA02985845B8BFF0EE476AFFF7C5BAF9
:10E7F800039800287FF45BAA02985845B8BFF0EE4A
:10E80800476AFFF754BA039800287FF42EAA0298A3
:10E818005845B8BFF0EE476AFFF727BA03980028B3
:10E828007FF467AA02985845B8BFF0EE476AFFF729
:10E8380060BA022232700022BDE601233370FEF76F
:10E84800AABB039800287FF476AA02985845B8BF57
:10E85800F0EE476AFFF76FBA02287CF412AF41F274
:10E86800B4120123B3547370FCF70BBF039900294A
:10E878007FF41AAC02995945B8BFF0EE474A13E441
:10E88800039900297FF4E6AB02995945B8BFF0EE29
:10E89800474AFFF7DFBB039900297FF455AC02997B
:10E8A8005945B8BFF0EE474A4EE4039900297FF472
:10E8B80023AC02995945B8BFF0EE474A1CE40399C6
:10E8C80000297FF491AC02995945B8BFF0EE474A48
:10E8D8008AE4039900297FF45FAC02995945B8BFCF
:10E8E800F0EE474A58E4039800287FF49CA9029860
:10E8F8005845B8BFF0EE476AFFF795B90399002964
:10E908007FF49AAC02995945B8BFF0EE474A93E4B0
:10E918001C800020FC4500202DE9F04F2DED028BD6
:10E92800984B994A1C7893B000F59C412031814658
:10E9380006911160002C00F08886944A1268904273
:10E9480040F28A80924A93491768934DDFF888B25B
:10E958000492013C02911C7007F48057002F40F08C
:10E968008880029B5B7D002B40F03986049B1B68E6
:10E978001E0401F1FB80894B99459BF8023000F297
:10E988000785002B40F00885854B0593049B1F687D
:10E9980017F4805940F0C785029BB5F906605B8B78
:10E9A8009E42B4BF002601267E4B1B6813F080539D
:10E9B80069D0059A127812F001026AD002987A4951
:10E9C800408C91ED037A039107EE900AF8EEE77A0E
:10E9D800B4EEE77AF1EE10FA81F26681002E60D18A
:10E9E800724C94F8A01000295BD1714871490068F5
:10E9F80090F82D0000240C604C608C606E49002853
:10EA080050D10870002A51D0F8064FD56B4A1278B9
:10EA1800D1064BD4B9F1000F48D1002B46D17A0268
:10EA280044D4674B1B78002B01F0BA86654B9B7862
:10EA3800002E41F035873BB1634A644B12681B686E
:10EA48009B1A002BC1F237871020584C19F086FA10
:10EA5800012384F8A13029E04D4B4E4A1F680493E6
:10EA680007F4805702924C4DDFF86CB1002F3FF449
:10EA780078AF00214B48F4F7EBFC00287FF471AF26
:10EA880003F0A2FA6DE77C0293D4059A127802F09B
:10EA98000102464C002184F8A01043490391002E3E
:10EAA800A3D0454901200870002AADD1484B1A78F7
:10EAB800002A50D10299B5F900E0488B898BB5F945
:10EAC80002407045B4BF8027002747F040037145D6
:10EAD800D8BF3B469B0843F08007A042B8BF3B46DF
:10EAE80043F04007A142C8BF3B469B08B5F9044024
:10EAF800B5F9067043F0800EA042B8BF734643F0E4
:10EB0800400EA142C8BF73469B0843F0800E274CB5
:10EB18008742C8BF734643F0400E94F8A2C08F42A4
:10EB2800B8BF73469C4501F09D82A4F8A42084F8E0
:10EB3800A620234984F8A2300F78002F01F02F82F5
:10EB48005F2B01F069826F2B01F00A81059B1B780E
:10EB5800DE0741F1CE80049B1B6803F00403002B01
:10EB680040F073860DF140081A4C0022C8F80420C2
:10EB780004F15009109240F6330A192740F28336FF
:10EB88002FE000BF04320020603000200032002057
:10EB9800784E00200C50002068430020404B4C0069
:10EBA8009C4500209843002024460020D0200020C7
:10EBB80070410020F43200209C2000202C430020CB
:10EBC800050200205078002028710020BC21002078
:10EBD80035770020AC340020843F002004344C45B5
:10EBE80020D0A278E3789A4217FB0260F6D26178C7
:10EBF800043117FB036235F911305345A8BF53465A
:10EC0800B3F5617FB8BF4FF461739842E6DA9A4270
:10EC1800E4DB21782429E1D840460434F4F708FCE1
:10EC28004C45DED1634A644B177898E8030083E8C3
:10EC38000300002F00F09285604B06935E48012187
:10EC4800F4F706FC002840F010839BF80330002BF3
:10EC580040F00B835A4B07935A4C23881EB226F078
:10EC680001061FFA86F84345A4F8008000F0DD8706
:10EC7800554E4FF002090E2014274FF0FF0A86F870
:10EC88000090777086F802A019F068F949464A485A
:10EC9800B4F80080F4F7DCFB002800F0038328F0C8
:10ECA800010292B24245228009D00E2086F80090D7
:10ECB800777086F802A019F051F9B4F8008018F0BE
:10ECC800020F01F06680414B414A19785068089359
:10ECD80018F0030F08BF81F00201C1F34001099247
:10ECE800F3F7A2FA24213448F4F7B2FB30B9059AB5
:10ECF80013785E0744BF23F004031370079B1B6857
:10ED080013F00A0F1AD006212B48F4F7A1FB0028AC
:10ED180000F098872388580641F1CD8007212648BE
:10ED2800F4F796FB50B12B4B2B4AB3F904302B491F
:10ED380082FB0302DB17C3EBA2030B800C211E48E6
:10ED4800F4F786FB2288002800F0E08242F4807302
:10ED58009A42238009D01C4B02201421FF221870EC
:10ED68000E2059709A7019F0F9F81D4B1B78082B72
:10ED780000F0D8820E2B00F0D582049B1B68590541
:10ED880061D5184B1B79002B00F0268114210A4805
:10ED9800F4F75EFB002840F0248112F05FFA0120AE
:10EDA80019F01EF800284ED0DFF83C9000264FF0EE
:10EDB800CC0A1EE02C3B002098430020FC380020A1
:10EDC800A04300204C410020FC2C0020F3700020C0
:10EDD800F47000205041002067666666BA21002062
:10EDE800A8340020144600201C6C0020DEB2022E3D
:10EDF80029D80AFB06F8731C59F80870002FF5D1BA
:10EE0800C378BA4A90F9020052F8233001970322D6
:10EE1800009201213A4618F0C9FB034606EB46006A
:10EE280000EB0010079353B1394609EB8000CC2260
:10EE380023F03BFC079B49F808300136F6B213F083
:10EE4800CFFD0028D3D1059B1E7816F0010600F0EF
:10EE5800DB80A74B01221A70069BB5F906101B68C8
:10EE6800A4485A8901279142077080F23582A24B43
:10EE78004FF07E521A60A14A029BB5F900E01F8B41
:10EE880092F90430107892F801C0002BAEEB07031A
:10EE980014BF01224FF0FF32002BB8BF5B42B3F51D
:10EEA800FA7FA8BF4FF4FA73984280F212821B1AB5
:10EEB80007EE903AF8EEE77A039BBE45C3ED007A79
:10EEC80003DAF1EE677AC3ED007AB5F902E0AEEB4A
:10EED8000703002BB8BF5B42B3F5FA7FA8BF4FF416
:10EEE800FA73984280F2F2811B1A07EE903AF8EE14
:10EEF800E77A039B7745C3ED017A03DDF1EE677A84
:10EF0800C3ED017AB5F90400C31B002BB8BF5B42FF
:10EF1800B3F5FA7FA8BF4FF4FA736345CCBFA3EBF0
:10EF28000C03002302FB03F307EE903A039A049BB9
:10EF3800F8EEE77AB842C2ED027ABCBFF1EE677A22
:10EF4800C2ED027A1A6812F4805200F0FE81B1F51F
:10EF5800FA6F6B4BA8BF4FF4FA61B1F57A7F187856
:10EF6800B8BF4FF47A71A1F57A71002840F0068293
:10EF7800644D654885FB013ECB17C3EB6E1303F167
:10EF8800010E6FF0630C30F91EE030F913000CFB32
:10EF98000313AEEB000103FB01F385FB0315DB173D
:10EFA800C3EB651303441BB207EE903A039BB8EE1C
:10EFB800E78A83ED038A002A40F0898323885B0669
:10EFC80000F1B880002E40F0438120F0A7F813B07C
:10EFD800BDEC028BBDE8F08F059B1B78DA077FF547
:10EFE800DCAE3C2015F00AFE00283FF42CAF04F0FC
:10EFF80051FA3C2015F0A4FD0028F8D1059B1E7895
:10F0080016F001067FF425AF394B1B780793002BC8
:10F018007FF422AFDFF814A1DFF814911AF8030C7B
:10F0280099F800805146AAF103070CF063FF002805
:10F0380000F04285079BB8F1000F53D107F1080192
:10F0480078790CF057FF002841F03C832F49B87AB3
:10F058000CF050FF002800F04385B8F1020F41F092
:10F0680034832B49F87B0CF045FF002841F03083AE
:10F078002849387D0CF03EFF002800F04385B8F1A0
:10F08800040F41F028832449787E0CF033FF0028D0
:10F0980041F024832149B87F0CF02CFF002800F0B0
:10F0A8004385B8F1060F41F01C831D4997F82300EA
:10F0B8000CF020FF002841F09A801A4997F82800A0
:10F0C8000CF018FF002800F04385B8F1080F41F054
:10F0D8009F80154997F82D000CF00CFF00283FF48D
:10F0E800BBAE09231A4601F084B800BFA442030846
:10F0F8009D450020DC1F0020782000202C7800206F
:10F10800442200201F85EB5100390020FC2B0020F1
:10F11800012C0020062C00200B2C0020102C002095
:10F12800152C00201A2C00201F2C0020F22B002068
:10F1380098000020BD4BBE4AB3F90430BD49DFED4D
:10F14800BE6A09889FEDBD7A82FB0302DB17C3EB19
:10F15800A2035B1A1BB207EE903AF8EEE77A67EE65
:10F16800A67A77EE876ABDEEE66A16EE103A203385
:10F17800402B40F2AC86DFEDB26ABDEEE77A17EEBF
:10F18800103A2033402B00F29E869FEDAE7AF4EEC3
:10F19800C77AF1EE10FA41F31182DFEDAB5A9FED19
:10F1A800AB6A01E0F0EE477AF4EEC67AF1EE10FAB7
:10F1B80037EEE57AF6DCDFEDA67AB4EEE77AF1EE23
:10F1C80010FA41F1FF81DFEDA05A9FEDA26A01E03C
:10F1D800B0EE677AB4EEC67AF1EE10FA77EE257AD9
:10F1E800F6D49FED967AF4EEC77AF1EE10FA00F3B2
:10F1F80073859FED997AF4EEC77AF1EE10FA44BF61
:10F208009FED937A77EE677A67EEA75A9FED935A48
:10F218009FED936A9FED937AA5EE856A27EEA55A2E
:10F22800A5EE867AE5EE077A039A92ED016AD2EDA9
:10F23800005A27EEC67A65EEA77AA5EEA67AE6EE1C
:10F24800267A82ED007AC2ED017A002E3FF4BDAE37
:10F25800089B1978099B01F001011868F2F7E4FF8F
:10F2680013B0BDEC028BBDE8F08F7F4B07931B6892
:10F278009F077FF5F1AC7D4CB4F8008018F0010FC2
:10F2880010D148F00103984523800BD0784B022217
:10F2980014211A700E20FF2259709A7018F05EFE21
:10F2A800B4F8008028F002039BB2434523803FF462
:10F2B8000AAD6F4B1421FF2202260E201E705970D2
:10F2C8009A7018F04BFEB4F80080FCE4DFED5C7A2D
:10F2D8000FE6DFED5B7AEFE5B1F5FA6F80F2E683D2
:10F2E800187A8B1A03FB00F3C2F5FA6293FBF2F368
:10F2F800C3F1640307EE903AF8EEE77A9FED5D7A82
:10F308005D4B67EE877AC3ED007AB4E522F480732B
:10F318009BB29A4223807FF41EAD584B1B78082B72
:10F328007FF428AD228822F040039BB29A422380C2
:10F338003FF423AD4E4B02201421FF2218700E20FB
:10F3480059709A7018F00AFE17E5029B588B814293
:10F35800C0F27F83B1F5FA6FD4BFC0EB0101C0F5ED
:10F36800FA614FF47A7303FB01F1454B1D78C0F540
:10F37800FA60B1FBF0F1002D3FF4FAAD5B7841483B
:10F3880001FB03F380FB0301DB17C3EB6111EFE51E
:10F3980013B901238BF802303B4B05931B201F78D0
:10F3A8009BF821600CF0D0FD012E07F00109824680
:10F3B80000F02E8607F0020303939BF82030DFF855
:10F3C800D480324C052B00F2A180DFE813F09100C5
:10F3D80085000600E2000601C400012E04BF0523D3
:10F3E8008BF82030B9F1000F00F01A81029B284FEA
:10F3F800B3F91810B8F80030002261F30F0263F374
:10F408001F42002361F30F0361F31F436A603968E9
:10F41800DBF814202B608A42C0F02D84012E41F0C5
:10F42800588203229BF820300392CBE750410020FA
:10F4380067666666BA21002035FA8E3CDB0FC93F45
:10F4480000000000DB0F4940DB0FC940E4CB164148
:10F45800DB0F49C0E4CB16C1DB0FC9BF92E741B946
:10F468009730083C15A82ABEA04300204C41002034
:10F47800FC2C00200AD7233C78200020A834002048
:10F48800442200201F85EB519C450020A443002006
:10F4980028710020F42C00200CF082FD012808D1EE
:10F4A800A14FB8F802303A68642101FB0323CBF876
:10F4B8001030BAF1000F03D098F80630002B5FD156
:10F4C800012E23D0984FDBF810203B689A42C0F0F9
:10F4D8001A8601238BF82030012E3CD098F807308B
:10F4E800012B00F0A78006F021FB9BF8203069E78C
:10F4F800B9F1000FD0D14FF48060BAF1000F00F0DD
:10F508009E8318F03BFE0023CBF81030039B002BA2
:10F518003FF43CAA039818F021FD049B1F6817F4D8
:10F5280080593FF439AA1D218048F3F791FF00283C
:10F538007FF432AA7E4A029BD2881B8BB5F90660FB
:10F54800991A8E4240F3D48513449E42B4BF0026D4
:10F558000126FFF729BA744F3A68B8F802306421D7
:10F5680001FB03234FF480600022CBF810308BF8A6
:10F5780020208BF8032018F0E9FD9BF8203021E7C4
:10F5880006F0D4FA03224FF47A738BF82020CBF8D4
:10F598001C30654F238843F00203238002F014FDDA
:10F5A8003A68DBF81C3013440422CBF818308BF887
:10F5B8002020012E40F09F853B68DBF818209A42F6
:10F5C800A4D25C4B187818B90CF0BEFC00289DD169
:10F5D800238823F002032380BEE7534FE9E7029A0A
:10F5E800013BD27D35F91330002A40F03F83A3F563
:10F5F8007A73B3F57A7FA8BF4FF47A7323EAE3737B
:10F6080007EE903A9FED4C7AF8EEE77A67EE877A44
:10F618004A4AFCEEE77A17EE903A1380FFF7ABB947
:10F62800414F3B6847F230520323CBF81C208BF83C
:10F638002030AFE706F07AFA032240F6B8338BF8A9
:10F648002020CBF81C30384FA4E73D4F3B78002BE7
:10F6580000F0DA873B4BDFF8F880DFF8F8B0DFF826
:10F66800F8A0029345465E46039099460EE019F8C5
:10F6780004109847032C28DC88B93B782AF8020F35
:10F6880001349C4205F1040580F20381072CE1B2A4
:10F698003046DBF80430EADD984700B2EDE738F889
:10F6A80024206B88801A4FF47A719B1A01FB00F0B2
:10F6B80040F6CA0290FBF3F00844904240F2EE2371
:10F6C800A8BF10469842B8BF184600B2D5E71D211A
:10F6D8001648F3F7BDFE00283FF470AC9BF80330E2
:10F6E800002B7FF46BACDFED187A184938EE678A87
:10F6F800C7F5FA63FDEEC87A1BB2CDED027ABDF903
:10F708000820120381FB0201D217C2EBA11203FBEE
:10F7180002F343F30F333B4407EE903A039BF8EEB2
:10F72800E77AC3ED037A49E4287100209843002062
:10F73800DC2C002005020020AAF1823F6043002053
:10F74800583200200C50002000007A44D34D62103B
:10F758007832002054300020CE200020DFF83CA36F
:10F76800DFF83C83BC4C0AF15A064FF001095146B8
:10F778001AF8010C0CF0BEFBF8B19AF804009AF8DC
:10F7880002309AF803E000EB400104EB8101013BF1
:10F79800D1F8B42003EB4303434493420DD094F8CB
:10F7A800E02081F8B0E009FA00F022EA0000C1F890
:10F7B800B430C1F8B87084F8E0000AF1060AB2451E
:10F7C800D5D1A64B06931946A54AA64BA64C09685F
:10F7D8001B78D2F8009008910793A4F1B00A00268C
:10F7E80063685BB31F784FB3A268A9EB0202002AD3
:10F7F8000ADB9AF8E0200121B14022EA010209F56A
:10F80800FA718AF8E020A160079ABAB1227859788B
:10F818000432D2B2002940F04D82029935F9122003
:10F82800098B01F1C800824240F334849AF8E01051
:10F838009A7841FA06F3D90740F1D4840136042EA8
:10F8480004F10C04CCD1FFF7F9B9834C94F8AA3031
:10F8580053B1059B1B78D80706D5029BB5F906203E
:10F868005B8B9A4200F3938411218048F3F7F0FDF3
:10F87800002800F0078294F8AE302BB994F8A8302D
:10F8880013B93223A4F8AC30012384F8AE30FFF763
:10F8980069B9DDF80C90764A04921146754A0968F0
:10F8A80042F2010AA2FB092B11EA0A0A4FEA9B1B42
:10F8B80000F0E481704D71486A4C714A95F800E097
:10F8C800007884F800E01070BEF1000F04D06C4A94
:10F8D80092F800E08EF0010E5F4C0F2084F82400AF
:10F8E800002B00F03C83674B0B931B780A931E4652
:10F8F8003B78029F644AB7F824C0DFF8A8810990D2
:10F908003D46FF8C08973746A2FB066252082D8BAE
:10F918000E9502EB420294F825500C95BA1AD2B211
:10F9280001F48051079204F128060BF59672674698
:10F93800564DCDF80CE0A4465446DDF830A00F91A2
:10F9480000200592CDF834909E46039B002B00F0D2
:10F9580057823CF910101FFA81F9B9454FEA400265
:10F9680003D3089B994540F28D8258F820108B45A7
:10F9780080F04F82A95E002C40F063820130704510
:10F98800A95206F10606E0DB0998414ADDF83490F1
:10F998008CF824000F28644651460CBF0121002131
:10F9A800734684F825A0117000F0DF82DFF8F8B004
:10F9B800384E2B4F34883868DBF80810DBF8042001
:10F9C800CBF80C0044F00404401A90422B4F3480CA
:10F9D8002B4C4FF0010188BF00223970217088BF7D
:10F9E8008BF82120002B00F0D582049A0299176821
:10F9F800294EB1F824C0B1F818E0244817F480570C
:10FA0800344640F0E78239460EE0627802EB820223
:10FA180002EB820202F2EE2292B201318B4220F80E
:10FA2800022B04F102040ED016F81120002A00F06F
:10FA38002D82022AE9D00131028820F8022B8B425C
:10FA480004F10204F0D10B9A137801331370FEF716
:10FA580085BF114689E400BFD0200020FC38002073
:10FA68002871002021410020802100209843002097
:10FA7800784E0020D34D621030300020F001002075
:10FA8800F101002005320020ABAAAAAA6843002091
:10FA9800E4320020A4430020AC320020092B0020CF
:10FAA800B429030808320020843F00201B7AC3F1E0
:10FAB800640307EE903A1FE40AF1050178790CF027
:10FAC80019FA00283FF4C2AAB8F1010F40F0FA85EC
:10FAD80007F10D01B87A0CF00DFA002840F0F58511
:10FAE800B649F87B0CF006FA00283FF4C1AAB8F131
:10FAF800030F40F0ED85B249387D0CF0FBF9002882
:10FB080040F0E985AF49787E0CF0F4F900283FF41D
:10FB1800C1AAB8F1050F40F0E185AB49B87F0CF0F8
:10FB2800E9F9002840F0DD85A84997F823000CF092
:10FB3800E1F900283FF4C1AAB8F1070F40F0578354
:10FB4800A34997F828000CF0D5F9002840F0608305
:10FB5800A04997F82D000CF0CDF900283FF47CA9B6
:10FB6800B8F1090F3FF478A9FFF7BBBA9A4CD4F85B
:10FB78008830A9EB0303002BFEF6FDAE974A94F8F4
:10FB88008C30517C069AC4F888200133944A029E2E
:10FB980032F81120B17D03F00F0384F88C30234430
:10FBA80092B292FBF1F283F8902094F8901094F8B6
:10FBB800912094F8923094F89C000A4494F8931099
:10FBC800134494F89420194494F895300A4494F80E
:10FBD8009610134494F89720194494F898300A44DE
:10FBE80094F89910134494F89A20194494F89B3087
:10FBF8000A44134494F89D1094F89F20184494F8EC
:10FC08009E3001440B441A4442F30B12642AF17DDE
:10FC1800A8BF642213B209B1C2F1640307EE903A97
:10FC28009FED707AF8EEE77AF0E402216E48F3F778
:10FC38000FFC00283FF436AB2680FFF740B818F0D9
:10FC480085FA60E4228822F040039BB29A4223801E
:10FC58003FF464A8654B02201421FF2218700E207F
:10FC680059709A7018F07AF9FFF758B8C3F53B63E2
:10FC780008331BB2BBE403230393D3E45C4A92F832
:10FC880000E021E694F8A830002B3EF46BAF059B0A
:10FC98001B7813F001037EF465AF012284F8A830C5
:10FCA80084F8A920FEF75EBF4B4C012184F8A01010
:10FCB800FEF7F7BE012900F044849AF8E0200123FA
:10FCC800B34001361343042E8AF8E03004F10C04E3
:10FCD8007FF486ADFEF7B2BF9FED467A77EE677A7E
:10FCE800FFF792BA059B444A1B781060DB0700F1C6
:10FCF8005C8294F8A60000287EF42DAFB4F9A430F5
:10FD0800322B7EF728AF94F8A2200121572A84F8D5
:10FD1800A61000F0C384049B1B6813F0040302D0F0
:10FD28005A2A00F077855D2A00F015855B2A00F0D5
:10FD380027855E2A00F03085562A00F08285972AAA
:10FD480000F05E85A72A40F0D7842C49049B0A78E6
:10FD58001B6842F004020A7003F00403FEF7FFBEBA
:10FD6800B2F5FA7FFEF6F7AE94F8A620002A7EF4E4
:10FD7800F2AE059B1B780121DF0784F8A61000F17D
:10FD8800B38401F0D5FA049B1B6803F00403FEF763
:10FD9800E6BE48F00203434523803EF494AF134B7C
:10FDA800022214211A700E20FF2259709A7018F03E
:10FDB800D5F8B4F80080FEF786BF00BF012C0020FC
:10FDC800062C00200B2C0020102C0020152C0020C5
:10FDD8001A2C00201F2C0020D0200020E07D0020BD
:10FDE800FC7D002014AE234198430020FC2C002009
:10FDF80021410020DB0F4940C02100202C43002076
:10FE0800002F3DD058F820108B454FEA4002FFF4F0
:10FE1800B1ADC24B995C03EB0209002900F0CC801C
:10FE2800022946D199F8011001EB810101EB81010A
:10FE380001F2EE2189B2032832DD09B2002C3FF429
:10FE48009DAD079B26F81310BAF1000F03D10A9B4A
:10FE5800022B7FF693ADB6F800A07188B6F804902F
:10FE6800AF4B514489440FFA89F983FB0931AD4BF3
:10FE7800A1EBE97123F8029009B24FF0010A7DE580
:10FE880039464200059B48F8203074E5CAB2022A78
:10FE980004D9032A7FF4CFAD6246BEE57246BCE5BD
:10FEA800012303FA00F9099B23EA090309B209931C
:10FEB80061E5A95ABFE743F04002934222807FF4EC
:10FEC800C9AEFEF72BBFDFED987AFFF7ADB9F4EEB8
:10FED800C77AF1EE10FA40F39483DFED945A9FED60
:10FEE800946A01E0F0EE476AF4EEC66AF1EE10FAA1
:10FEF80036EEE57AF6DCDFED8F6AB4EEE67AF1EEFF
:10FF080010FA40F18583DFED895A9FED8B6A01E095
:10FF1800B0EE667AB4EEC67AF1EE10FA77EE256A9C
:10FF2800F6D49FED867AF4EEC76AF1EE10FA40F344
:10FF38008D809FED837A77EE666A66EEA65A9FED0E
:10FF4800815A9FED816A9FED817AA5EE856A26EE3A
:10FF5800A55AA5EE867AE5EE076AFFF70EB97C4941
:10FF68007C4A0B917C4D012111701B217B48039326
:10FF7800F3F76EFA039B00287FF418ADDFF8F0B1B1
:10FF8800774FDBF80C203B68CBF808309B1AC82B5E
:10FF980000F24183049B1F6807F4805753E53946F4
:10FFA8006E48F3F755FA00283FF49CAE84F8A77022
:10FFB80001F0BEF9FEF7CABDC1B2022940F2BF8204
:10FFC80003297FF476AF0E9B19460F9B002B08BFC1
:10FFD800394630E700210FE0627802EB820202EB3B
:10FFE800820202F2EE2292B20131994220F8022BEB
:08FFF80004F102043FF427ADFF
:020000040801F1
:1000000016F811201AB1022AEAD00288F0E7CAB223
:10001000032AFAD87246EBE700230393FFF7D1B91E
:10002000B2F5FA7FFEF69BAD94F8A630002B7EF475
:1000300096AD059B1B78012113EA010084F8A610F8
:1000400000F0FB8201F0C4FF049B1B6803F0040373
:10005000FEF789BD9FED457AF4EEC76AF1EE10FA1E
:1000600044BF9FED367A77EE666A6AE7404A4149B7
:100070001068B4F9A420C76981FB07018911FF1733
:10008000781A00F5FF407F3082423EF756ADC91B1B
:100090000A4412B2A4F8A420FEF74FBDC8398A4220
:1000A0006CDA9AF8E0109A7841FA06F3DB073FF52C
:1000B000C9AB52420120099218F034F87B1E099A0C
:1000C000162B00F22C81DFE813F0B501CB019C0167
:1000D000FD01E1011102870172015B0144012D0163
:1000E0002A01FD011A011102870172010401EE00CB
:1000F000D8002602C000AA000126FEF759BC3A68C3
:10010000DBF81C301344CBF81830FFF703BA05F0C6
:1001100011FD032240F6B8338BF82020CBF81C30B9
:10012000FFF73CBAAC32002056555555402100200F
:1001300000000000DB0FC940E4CB1641DB0F49C0D3
:10014000E4CB16C1DB0FC93FDB0F494092E741B951
:100150009730083C15A82ABE05320020E432002062
:10016000684300209843002028710020DB0FC9BF9E
:1001700060450020D34D6210843F00209AF8E030A3
:100180000122B24023EA020309F5FA728AF8E0304C
:10019000A260FFF757BB0021C648F3F75DF90028BE
:1001A0007FF466AB322384F8AA00A4F8AC30FFF7E2
:1001B0005FBBC14B1B78002B3EF4D1AC9BF80330E6
:1001C000002B7EF4CCAC94F8A7300133DBB2032BC8
:1001D00084F8A7307EF6C3ACB84B5B7813B9002E19
:1001E0007EF4BDAC01F0F4FEFEF7B4BC002A0CBFF7
:1001F000012002205FE707231A4602EB8202174420
:1002000089F80030B97878780DF042F8059B1E78AF
:1002100006F00106FEF724BE08231A46EDE7DAF8D9
:10022000E400DFF89C8290F8361098F80230114410
:100230006429A8BF642121EAE17180F83610002BFF
:1002400040F08A831CF0E4FD3BE5DAF8E400DFF8D7
:10025000708290F8371098F802301144FE29A8BF38
:10026000FE2121EAE17180F83710002BEAD0162038
:100270000BF0CCFEDAF8E400E4E7DAF8E400DFF8AB
:10028000408281781144C829A8BFC82121EAE171C0
:10029000817098F80230002BD4D014200BF0B6FEF9
:1002A000DAF8E400CEE7DAF8E400DFF81482417807
:1002B0001144C829A8BFC82121EAE171417098F80A
:1002C0000230002BBED013200BF0A0FEDAF8E400C1
:1002D000B8E7DAF8E400DFF8E88101781144C829CA
:1002E000A8BFC82121EAE171017098F80230002B03
:1002F000A8D012200BF08AFEDAF8E400A2E7DFF8BB
:10030000C081089898F80230417911446429A8BF47
:10031000642121EAE1714171002B40F04183DAF858
:10032000E4008FE7DAF8E400DFF89481017A98F8C6
:1003300002301144C829A8BFC82121EAE171017225
:10034000002B3FF47FAF0B200BF060FEDAF8E400E7
:1003500078E7DAF8E400DFF86881C17998F80230CC
:100360001144C829A8BFC82121EAE171C171002B3D
:100370003FF468AF0A200BF049FEDAF8E40061E7C9
:10038000DAF8E400DFF83881817998F80230114416
:10039000C829A8BFC82121EAE1718171002B3FF46F
:1003A00051AF09200BF032FEDAF8E4004AE7DAF840
:1003B000E400DFF80C81417998F802301144C82933
:1003C000A8BFC82121EAE1714171002B40F0898268
:1003D000112F7FF456AF35E7DAF8E400DFF8E0805C
:1003E000017998F802301144C829A8BFC82121EA30
:1003F000E1710171002B40F0D982102F7FF457AFCB
:1004000020E70899DFF8B8800F791744642FA8BF58
:10041000642727EAE7770F710BF012FE98F8023095
:10042000002B3FF47CAF032039460BF0EFFDDAF8E8
:10043000E40007E70898DFF8888001781144FA297A
:10044000A8BFFA2121EAE171017098F80230002B6F
:100450003FF465AF01200BF0D9FDDAF8E400F1E6D6
:100460000898DFF85C80817811446429A8BF642172
:1004700021EAE171817098F80230002B3FF44FAF10
:1004800002200BF0C3FDDAF8E400DBE60898DFF8A1
:100490003080C17998F80230114481F30801C171AC
:1004A000002B3FF43CAF05200BF0B0FDDAF8E40080
:1004B000C8E600BF9843002021410020507800206A
:1004C00040430020089BDFF88084997998F8020067
:1004D00011446429A8BF642121EAE17199710028BF
:1004E00040F034820D2F7FF40CAF18E7DAF8E40007
:1004F000DFF85484C17898F802301144C829A8BFA5
:10050000C82121EAE171C170002B40F029820F2F30
:100510007FF4E3AE96E60898DFF82C844178114426
:10052000B1F5967FA8BF4FF4967121EAE171417051
:1005300098F80230002B3FF4F2AE15200BF066FD68
:10054000DAF8E4007EE60E9979E435F9122099781C
:10055000B2F5617F4FF4966393FBF1F33ADB40F61B
:1005600033019142A8BF11460C2FA1F5617191FB97
:10057000F3F100F00D81182F7FF4A3ABC9B2C829A5
:100580000B46A8BFC823DAF8E400C27DDFB2974269
:100590003FF497AB9A1ADFF8B083C77548BF0732AC
:1005A000D71098F802300137FFB23BB9002F3FF463
:1005B00088AB384617F0B6FDFFF783BB18200BF069
:1005C00025FDF3E7B0EE677AFEF7F9BDF0EE477A66
:1005D000FEF70BBE0C2F40F0D18000273946C54BEB
:1005E00009915B78BB423FF46CABDFF85C83384623
:1005F00002F04CFC98F8023009991BB1C9B20C20EA
:100600000BF004FD0137FFB2D0E7B0EE667A76E476
:10061000B94A0292FFF743B9F0EE476A85E4B74A58
:10062000049B1F68138823F004031380012307F43D
:1006300080578BF82130FFF70ABAB14B1B6813F4CF
:10064000003340F0A7801846AE490E5C0F2E00F133
:100650000C000ED00133152BF7D1049B1B68FA3A1E
:100660000021A4F8A42003F0040384F8A610FEF7E8
:100670007ABAA54FD7F800E05800BEF1000F07D0B6
:10068000C61801EB86069EF801E076787645E4D23E
:1006900018449E4E9E4B01EB800100203960308053
:1006A0001860DAE79B4B9C491A684FF47A73B3FBE6
:1006B000F2F3C3EB431203EB8202049B1B68D200EC
:1006C000A1F8B42003F00403FEF74DBA01231A4643
:1006D00093E502231A4690E503231A468DE5042389
:1006E0001A468AE505231A4687E506231A4684E555
:1006F000049B8A491B680A6003F00403FEF733BABF
:100700000021BB2A10917CD0B72A76D0BE2A72D0A5
:10071000BD2A59D09E2A00F0C1809D2A00F0B780E2
:10072000AE2A00F0AD80AD2A00F0A380EF2A00F0E1
:100730003181FD2A00F02881FB2A00F01F81FE2A6A
:1007400000F01681F72A00F0C2807B2A7EF407AA07
:100750004FF4FA61022002F0BFFAFEF700BA704BC4
:10076000002201206F49634C0B60227017F0DAFC05
:10077000049B1B6803F00403FEF7F5B9182F7FF400
:10078000A0AA00210B46FEE6674B01220220E9E702
:10079000CFB224E7654B1B78032B65D0034653E7A4
:1007A000634B02220320DDE7002E3EF451A9614C89
:1007B00094F8A130002B3EF47DA917F0B7FB00237D
:1007C00084F8A130FEF776B94FF6FE735A4AD08905
:1007D0009689014433449381D18108F0A3F9F2F75B
:1007E0000BFA08F087F9F5F7F9F8012017F09AFCF1
:1007F000B4F8A42031E70223E8E70B464FF6FE7178
:10080000E4E70B460221E1E7049B4C4A1B684FF4E6
:10081000C871118003F00403FEF7A5B994F8A8206D
:10082000002A40F0D48094F8AA3083F0010384F8C1
:10083000AA30002B40F0C2800C2017F093FB049BE1
:100840001B6803F00403FEF78EB908F06BF9F2F7AA
:10085000D3F908F04FF9F5F7C1F8012017F062FC61
:1008600094F8A220FFF76FBA17F060FBB4F9A42048
:10087000F3E6FF2100201FF089FB94F8A22055E742
:10088000012100201FF082FB94F8A2204BE70021F9
:10089000FF201FF07BFB94F8A22041E701201FF00E
:1008A00075FB94F8A22038E7002B80D02449254A14
:1008B00009684FF47A7000FB0313136077E71D4C4F
:1008C00001F086FB002384F8A130FEF7F3B8002185
:1008D000042002F001FAFEF742B903230393FEF766
:1008E0001DBE112009920BF091FBDAF8E400099A81
:1008F0006EE500BF744100200C500020A44300208E
:10090000FC2A0020A02E030870200020C420002014
:10091000C8200020684E0020047E0020C021002056
:100920000481002070410020528100209443002067
:10093000A0810020D02000203478002006870020ED
:1009400028710020BC210020404300200D20099286
:100950000BF05CFB099AC5E517200BF057FBDEE4B2
:100960000F2009920BF052FBDAF8E400099ACEE569
:100970000021032002F0B0F9FEF7F1B800210220B7
:1009800002F0AAF9FEF7EBB80021012002F0A4F969
:10099000FEF7E5B80021084602F09EF9FEF7DFB841
:1009A0000E200BF033FBDAF8E4004BE41020099240
:1009B0000BF02CFBDAF8E400099A1EE50B2017F087
:1009C000D1FA049B1B6803F00403FEF7CCB884F84B
:1009D000A80084F8A910FEF7C6B800BF426A806A72
:1009E000101AB0FA80F04009704700BF417170479B
:1009F00043799B070AD5436A8269D154436A0169E6
:100A00000133B3FBF1F201FB12334362704700BFC5
:100A1000437913F0010317D0016AC369C26810B4A7
:100A20005B1A541E23400BD043694C1C5B5CB4FB27
:100A3000F2F102FB114202625DF8044BD8B270473A
:100A400018465DF8044B704718467047437913F019
:100A5000020308D00369426A816A581E531A034090
:100A6000DBB2C01A70471846704700BF437913F0D5
:100A7000010306D0C369C268016A581A531E1840A0
:100A800070471846704700BF10F8113C0133DBB2C5
:100A90000A2B00F8113C07D9044A10F8131C002354
:100AA00022F8113000F8113C704700BF38300020A8
:100AB000F0B55C4F5C4B3C785C4A0134A2FB04020D
:100AC00093E86000120902EB8202D86BA4EB820269
:100AD000A9423A7001EB000233D293F84500002896
:100AE00055D0534802F580320478B2FBF4F29642B6
:100AF00030D3901B4FF4803595FBF4F4204498607C
:100B000040F68C240025A04283E8060083F8455077
:100B100028D993F8406093F9422096424AD00021A8
:100B200093F9412083F843104FFA86FE964250D045
:100B30000022012183F842E083F8402083F844102A
:100B4000F0BD3B480478B2FBF4F29642D1D293F860
:100B5000450010B34FF4803090FBF4F4901B001B61
:100B60009860CDE793F8442082B1A0F2EF2140F2E3
:100B7000DA52914213D893F840200B2A0FD803EB96
:100B80008201013283F84020C860F0BDF0BD284CDE
:100B90002478B2FBF4F29642ABD20446DEE7254A53
:100BA000002102F1300083F8441042F8041F824211
:100BB000FBD1F0BD321F082AB1D893F84320182A80
:100BC0002AD8013283F843204FFA86FE93F9412058
:100BD000ACE793F844100029AAD0174894466AB1AC
:100BE0000FFA86FC134C014600EB4C0754F8045FE7
:100BF00021F8025BB942F9D10B2E08DC00EB4C0165
:100C00000239002001320C2A21F8020FFAD10B49D7
:100C10000A7801320A708BE74FFA86FE83F841E0CA
:100C2000724683E7B82100206C4F0020CDCCCCCC9D
:100C30003C060020744F0020383000203130002066
:100C400030B40E4D0E4B2A780E4C0132A3FB02033A
:100C50001B09E06B03EB8303A2EB83034FF6FF72E8
:100C6000914200F101002B70084408BF0123E063AA
:100C700008BF84F8453030BC704700BFB821002061
:100C8000CDCCCCCC6C4F002000284DD0C14B1A7C71
:100C9000F0B4002A49D11A6800210128116042D01D
:100CA00093F82820002A40F04D819A6900210228FB
:100CB000116038D093F84020002A40F01B811A6B55
:100CC0000021032811602ED093F85820002A40F00C
:100CD000E8809A6C00210428116024D093F87020D9
:100CE000002A40F0B5801A6E0021052811601AD044
:100CF00093F88820002A40F082809A6F002106280D
:100D0000116010D093F8A020002A4ED1D3F8902083
:100D100000210728116006D093F8B820DAB9D3F87B
:100D2000A83000221A60F0BC70475F689A49BA0A7E
:100D30008A4200F0C28140F2718198498A4200F0F3
:100D4000928105318A4200F08C8107398A4200F095
:100D50008281FE216AE1D3F8AC608F48B20A8242F8
:100D600000F0AF8140F249818C48824200F08381DB
:100D70000530824200F07D810738824200D0FE219A
:100D8000EFF31182502080F31288854C756A7069E8
:100D900001EB810104EBC101013540F001004D621E
:100DA000D2B2706182F31188B9E7D3F894607A4CBB
:100DB000B20AA24200F0838140F20481774CA24241
:100DC00000F055810534A24200F04F81073CA24259
:100DD00000D0FE21EFF31182502484F31288704D6D
:100DE000776A746901EB810105EBC101013744F0B9
:100DF00001044F62D2B2746182F3118886E7DE6F1C
:100E0000654CB20AA24200F0648140F2E480634C77
:100E1000A24200F042810534A24200F02081073C4A
:100E2000A24200D0FE21EFF31182502484F31288F5
:100E30005B4D776A746901EB810105EBC1010137F4
:100E400044F001044F62D2B2746182F3118854E716
:100E50005E6E514CB20AA24200F0358140F2C4806D
:100E60004E4CA24200F021810534A24200F01781CD
:100E7000073CA24200D0FE21EFF31182502484F3FC
:100E80001288474D776A746901EB810105EBC10156
:100E9000013744F001044F62D2B2746182F31188C9
:100EA00021E7DE6C3C4CB20AA24200F0148140F211
:100EB00081803A4CA24200F0FE800534A24200F04C
:100EC000F880073CA24200D0FE21EFF311825024AB
:100ED00084F31288324D776A746901EB810105EB66
:100EE000C101013744F001044F62D2B2746182F350
:100EF0001188EEE65E6B284CB20AA24200F0E78051
:100F000050D9264CA24200F0A8800534A24200F03D
:100F1000CE80073CA24200D0FE21EFF31182502484
:100F200084F312881E4D776A746901EB810105EB29
:100F3000C101013744F001044F62D2B2746182F3FF
:100F40001188BCE6DE69144CB20AA24200F0BD80F2
:100F50005CD9124CA24200F0A6800534A24200F0F7
:100F6000A080073CA24200D0FE21EFF31182502462
:100F700084F312880A4D776A746901EB810105EBED
:100F8000C101013744F001044F62D2B2746182F3AF
:100F900011888AE6644A0020020010004D0010000B
:100FA00030710020B2F5801F69D04C498A42B3D11C
:100FB0000221B2E7B2F5801F5FD048498A4283D14F
:100FC000022182E7B2F5801F5DD044498A427FF456
:100FD00000AF0221FEE6B2F5801F52D03F498A429F
:100FE0007FF420AF02211EE7B2F5801F4FD03B49AE
:100FF0008A427FF440AF02213EE7B2F5801F44D021
:1010000036498A427FF4BBAE0221B9E6B2F5801FB1
:1010100041D032498A42A7D10221A6E7B2F5801F0A
:1010200037D001398A427FF494AE0221EFF3118266
:10103000502484F312882A4D7E6A7C6901EB810179
:1010400005EBC101013644F001044E62D2B27C616D
:1010500082F311881FE60021E8E704215DE70521FE
:10106000E1E60521E2E70421E0E70521B2E60421FB
:10107000B0E6052184E6042182E6012125E701216D
:101080004BE70121CFE60121A4E6012178E6012109
:10109000F2E60121CAE7012167E70421C3E6052141
:1010A000EAE6052161E704215FE70421E4E6052182
:1010B00033E7052109E7042107E70321B6E7032108
:1010C00088E603215CE60321D6E603214DE70321F0
:1010D00023E70321A7E60321F7E600BF0100100084
:1010E00030710020704700BF10B4C1F303220C0B15
:1010F000C1F3031301F00F0104EB440402EB4202BD
:1011000003EB430301EB4101183418321833183153
:10111000046142618361C1615DF8044B0620704740
:1011200011F4004F2DE9F04714BF4FF00E0A4FF0B5
:10113000070A11F4804F14BF4FF00E094FF0070952
:1011400011F4005F14BF0E26072611F4805F14BF50
:101150004FF00E084FF0070811F4006F14BF0E2572
:10116000072511F4806F14BF4FF00E0C4FF0070CE1
:1011700011F4007F14BF0E24072411F4807F14BFE4
:101180000E22072211F0800F14BF0E23072311F047
:10119000400F14BF4FF00E0E4FF0070E11F0200F4E
:1011A00014BF0E27072711F0100F866114BF0E26FB
:1011B000072611F0080F056214BF0E25072511F050
:1011C000040F846214BF0E24072411F0020FC262C0
:1011D00014BF0E22072211F0010F036314BF0E2368
:1011E0000723C0F810A0C0F81490C0F81C80C0F805
:1011F00024C0C0F834E08763C66305644464826435
:10120000C3641220BDE8F087F8B5A0F517746379C0
:10121000A179DB0711D594F840327BB994F84332B9
:10122000012B4FD06BB3002384F84332A06B01F045
:101230000101BDE8F84015F0E5BFF8BDA06B0268FC
:10124000D36A5B08536294F85132012B07D094F8AB
:10125000453223B1B4F84C320133A4F84C32C943BF
:1012600001F0010115F0CEFF0023012284F8432292
:1012700084F8413284F8423284F84032A4F84A3289
:10128000F8BD94F8426294F84122B24210D9551E3A
:10129000AD1BEDB2B4F84A2201350127F01807FA68
:1012A00000F0013302439D4292B2F7D1A4F84A22E2
:1012B0000123C94384F843321940A06BBDE8F840CC
:1012C00015F0A0BF94F8413284F84232ABE700BF7A
:1012D00070B5164E0546582404FB05641FF0DCF873
:1012E000636813B3DB6803B31149237B114A01EA36
:1012F0004001194389B20B1283EA11134B4003F0EA
:101300000F0305EB850043EA011105EB40000025C2
:101310001368257389B206EBC00098476368DB68E1
:1013200058601A6842F001021A6070BD4C4B0020F0
:10133000FEFF0100404B00202DE9F04F804B1B7851
:1013400085B0002B40F0DB807E4B1B78D80767D43C
:101350001DF0E8FE7C4B1B88002B6DD1794B187873
:10136000C10702D505B0BDE8F08F784F3B78002B60
:1013700040F0E280DFF82082754C7249754B40F0F6
:1013800003020A7002E0043398450AD01A78242A2E
:10139000F9D19978DA789142F5D26A4B40F007009A
:1013A00018706D4B6649B3F904206C4B6C4D88780E
:1013B00026681B686B4985FB02544FF47A77D21775
:1013C000C2EBA40207FB0060002413F40033486062
:1013D0004A808C6040F0A9806349C85C05281A46A1
:1013E00007D00132152A03F10C03BBD0C85C0528D5
:1013F000F7D15E4C2568530035B1981801EB800099
:101400006D784078A842ADD213445948594A01EB4F
:101410008301002321600380136005B0BDE8F08FD5
:10142000554A564B1178186801F00101F0F700FF9A
:10143000454B1B88002B91D0514A127822B1514A5A
:10144000B2F8B420002A8DD1464C002B93FAA3F2B7
:10145000B2FA82F308BF4FF0FF33A2680133934220
:1014600080D0DAB29200402A47494848A360A8BF1A
:101470004022042A086040F30784082A486040F2AA
:1014800001840C2A886040F2FB83102AC86040F275
:10149000F583142A086140F2EF83182A486140F26C
:1014A000E9831C2A886140F2E383202AC86140F264
:1014B000DD83242A086240F2D783282A486240F25A
:1014C000D1832C2A886240F2CB83302AC86240F252
:1014D000C583342A086340F2BF83382A486340F248
:1014E000B9833C2A886340F2B383C8634023FF2258
:1014F0000E20CA5405B0BDE8F04F16F033BD204AA7
:101500001378002B7FF420AF214B1E4819684FF44D
:101510007A73B3FBF1F3C3EB431103EB8103DB00FD
:101520000121A0F8B43011700EE71A4B1B78032B81
:1015300000F0898323464FE7064B03F1500831E062
:10154000507800209C450020A4430020484B0020F8
:1015500028710020AC34002050410020FC2A0020DB
:1015600067666666B8210020A02E03087020002060
:10157000C4200020C8200020F3700020F470002058
:101580006C200020047E0020FC2C0020140A050A98
:10159000684E002094430020FC340020043343456F
:1015A00000F023811A78232AF8D19978DA789142C9
:1015B000F4D28F4B1A680AB1002111609A690AB1FE
:1015C000002111601A6B0AB1002111609A6C0AB1F6
:1015D000002111601A6E0AB1002111609A6F0AB1E0
:1015E00000211160D3F890200AB100211160D3F8D6
:1015F000A8300BB100221A607E4B7F495B68002245
:10160000C3F308030A70002B40F0BE81EFF311838F
:10161000002B40F0B981794C79492268886800BF75
:1016200023689A42F9D1774E31684FF47A7909FBF1
:1016300001F31B1AB3FBF1F309FB02397048DFF821
:10164000E4E14FF47A754FF0100C4FF0010A694B4A
:101650005B68C3F30803002B40F05581EFF311835F
:10166000002B40F050812368816800BF22689342BC
:10167000F9D1D6F800B005FB0BF2521AB2FBFBF21F
:1016800005FB0323A3EB0903B3F57A7FDFD3232103
:101690005D48F1F7E1FE3B785C4A002840F0A88104
:1016A0001070002B00F00981594B5A4A1B780193A6
:1016B000534D00920A230293CDF80C80019B8BB30B
:1016C000DFF854A11F464FF0000B4FF058094FF0C0
:1016D0000108514B09FB0B3080F80C80DAF804301C
:1016E000C3B1DB68B3B1037B4C4A83F02A0101F03C
:1016F0000F0143F0280341EA03110023037312682A
:1017000050469047DAF80430DB6858601A6842F0B7
:1017100001021A600BF1010B5FFA8BF39F420AF191
:10172000580AD6D8009B1B78002B7DD03C4A116804
:10173000908800224A62D1F80CE0012B40EA0E00AA
:10174000C86071D036493648896880894A62D1F8C4
:101750000CE0022B40EA0E00C86065D030493048EA
:101760000969808A4A62D1F80CE0032B40EA0E0036
:10177000C86059D02A492A488969808B4A62D1F8C1
:101780000CE0042B40EA0E00C8604DD024492448E8
:10179000096A808C4A62D1F80CE0052B40EA0E0001
:1017A000C86041D01E491E48896A808D4A62D1F8BE
:1017B0000CE0062B40EA0E00C86035D018491848E6
:1017C000096B808E4A62D1F80CE0072B40EA0E00CC
:1017D000C86029D012491248896B808F4A62CA6852
:1017E000082B42EA0002CA601ED0044CC5E500BFC7
:1017F000644A002000ED00E0504E002028710020D7
:1018000010E000E02C71002098430020A42000206C
:10181000AA4500200C4E00204C4B0020404B0020DD
:10182000104E002024710020694B5B68C3F308034D
:10183000002B40F08680EFF31183002B40F0818075
:101840002368A96800BF22689342F9D130684FF439
:101850007A7202FB00F8A8EB0108B8FBF0F802FB73
:101860000388DFF86CA1DFF87CE14FF47A704FF069
:10187000100C4FF00109DAF80430C3F308033BBB46
:10188000EFF3118323BB2268A96800BF236893424A
:10189000F9D1376800FB07F2521AB2FBF7F200FBEE
:1018A0000323A3EB0803B3F57A7FE4D3029B013B48
:1018B00002937FF403AFDDF80C80464B464A1B6869
:1018C00046499B1A464A087818BF0123137054E50D
:1018D000EFF311828CF31288AF682B68D90302D51D
:1018E000CEF80090AF682368D1B2DEF8002081F313
:1018F000118831681A4400FB01F3DB1BB3FBF1F3E1
:1019000000FB0233CDE7EFF311838CF31288D0F89C
:1019100008B00268D20303D5CEF800A0D0F808B012
:101920002268D9B2DEF8003081F3118831681A4498
:1019300005FB01F3A3EB0B03B3FBF1F305FB023350
:10194000A0E6EFF31183102282F31288D5F808E0A5
:101950002A6812F4803F234A03D001211160D5F890
:1019600008E0D4F800801268DBB283F31188306895
:101970004FF47A71904401FB00F3A3EB0E03B3FB29
:10198000F0F301FB08386CE7EFF31183102282F3C8
:10199000128802F1E0229168106810F4803F11482B
:1019A00002D00121016091680F4CDBB2D4F80090A5
:1019B000026883F311880D4E35684FF47A709144B4
:1019C00000FB05F35B1AB3FBF5F300FB093935E6C1
:1019D00000ED00E03C4B00200D2501089C45002057
:1019E000504E002024710020287100202C7100200E
:1019F00001211170002B3FF460AFA44BA44A1B7867
:101A00000293A44D00920A230193CDF80C80029B0F
:101A10008BB3DFF884A21F464FF0000B4FF058093C
:101A20004FF001089C4B09FB0B3080F80C80DAF872
:101A30000430C3B1DB68B3B1037B984A83F028015B
:101A400001F00F0143F02A0341EA0311002303735D
:101A5000126850469047DAF80430DB6858601A681C
:101A600042F001021A600BF1010B5FFA8BF39F4207
:101A70000AF1580AD6D8009B1B78002B5FD0884A01
:101A80001168908800224A62D1F80CE0012B40EAEC
:101A90000E00C86053D082498148896880894A62B3
:101AA000D1F80CE0022B40EA0E00C86047D07C4918
:101AB0007B480969808A4A62D1F80CE0032B40EA2E
:101AC0000E00C8603BD0764975488969808B4A62B0
:101AD000D1F80CE0042B40EA0E00C8602FD070490A
:101AE0006F48096A808C4A62D1F80CE0052B40EA05
:101AF0000E00C86023D06A496948896A808D4A62AD
:101B0000D1F80CE0062B40EA0E00C86017D06449FB
:101B10006348096B808E4A62D1F80CE0072B40EADB
:101B20000E00C8600BD05E495D48896B808F4A62A9
:101B3000CA68082B42EA0002CA607FF456AE594BCD
:101B40005B68C3F30803002B5AD1EFF31183002B1A
:101B500056D12368A96800BF22689342F9D1306842
:101B60004FF47A7202FB00F8A8EB0108B8FBF0F81A
:101B700002FB0388DFF82CA1DFF82CE14FF47A7028
:101B80004FF0100C4FF00109DAF80430C3F30803EA
:101B9000DBB9EFF31183C3B92368A96800BF2268DA
:101BA0009342F9D1376800FB07F2521AB2FBF7F201
:101BB00000FB0323A3EB0803B3F57A7FE4D3019B77
:101BC000013B01937FF423AF75E6EFF311828CF3B1
:101BD0001288AF682B68DB0302D5CEF80090AF689F
:101BE0002368D1B2DEF8002081F3118831681A44ED
:101BF00000FB01F3DB1BB3FBF1F300FB0233D9E77E
